:020000040800F2
:20000000F0FF0120BD5E0608C9F4000811B70408355F0608355F0608355F06080000000028
:20002000000000000000000000000000C5F40008C1F4000800000000BDF40008657A04089E
:20004000355F0608355F0608355F0608355F0608355F0608355F06083DDA040805DA0408C6
:20006000CDD9040895D904085DD90408511306084113060831130608211306080D1306087C
:20008000F9120608E5120608355F06080000000000000000000000000000000025D9040896
:2000A000DD6204082D630408CD620408556304081D6304080D630408FD620408355F060845
:2000C000355F0608355F0608355F0608355F0608355F0608417C0408857B04080000000021
:2000E000EDD80408355F0608810D010800000000000000000000000000000000D112060805
:2001000000000000FDEE0508ED620408355F060800000000000000000000000000000000EA
:20012000BD120608A912060895120608811206086D12060800000000000000000000000036
:2001400000000000000000000000000051EE0008591206084512060831120608C97A0408DA
:20016000355F0608355F06080000000000000000000000000000000000000000000000003B
:2001800000000000355F06080000000000000000355F0608355F06085C5A060001000000BC
:2001A0000E020100020000001C6E0020806E002000000000B09107087C6E00201402010003
:2001C00005000000503C0020886E002000000000B2910708846E00201302010004000000DA
:2001E000382E0020946E002000000000B8910708906E0020031101000A000000646D0020D1
:200200009C6E002000000000D1190108986E00200D1001004C000000FC680020AC6E002073
:2002200000000000D5DF0308A86E0020090201000100000064680020FC6E00200000000046
:20024000BC910708F86E0020FD0101002400000028680020046F002000000000C353040834
:20026000006F0020FB01010001000000386300202C6F00200000000029610508286F00202D
:20028000FC0101000900000004620020346F00200000000031610508306F0020F7010100B7
:2002A00006000000F8610020446F002000000000BE910708406F0020F901010004000000C0
:2002C000F4610020506F0020000000006D5404084C6F0020160215003F000000EC2F00207B
:2002E000586F0020000000004D610508546F00203400010010000000246100209C6F002064
:2003000000000000618A0208986F00201102010008000000FC600020B06F002000000000EA
:20032000C4910708AC6F00201212010004000000F4600020BC6F002000000000CC910708CA
:20034000B86F00201830010038000000BC600020C46F002000000000916D0508C06F0020EC
:20036000000201000B000000405D0020007000200000000071610508FC6F0020FF21010097
:2003800005000000E85C00201070002000000000196105080C700020081203000F00000005
:2003A000F45C00201C70002000000000A561050818700020FA01010003000000545600209D
:2003C00030700020000000008D6105082C7000202A02010008000000CC4A00203870002073
:2003E00000000000D0910708347000202052010008000000284900204470002000000000E9
:20040000858A0208407000200610010024000000082F002050700020000000000D62050805
:200420004C7000200C02010004000000D44100207870002000000000956105087470002089
:20044000FE01010014000000843D00208070002000000000DD6005087C700020FD0701003C
:200460007C0000000EE7002090E7002000000000BD7F01088CE70020F59101006C00000089
:20048000CCE5002010E8002000000000DD9001080CE8002023200100100000004AE6002045
:2004A00080E80020000000001D0902087CE80020123001001000000088DB002094E800208E
:2004C00000000000D891070890E800200B3001001A000000ECD50020D8E8002000000000F5
:2004E000E8910708D4E800201F50010024000000ACD50020F8E800200000000004920708BE
:20050000F4E80020050201000400000000DA002020E9002000000000289207081CE90020C2
:20052000010201000B000000A8ED0020D4F600200000000061610508D0F600200202010053
:2005400003000000A0ED0020E4F600200000000000000000E0F600201B02010010000000CD
:200560008CED0020ECF600200000000079610508E8F600201B2001000C00000004EB0020A4
:2005800000F700200000000039860108FCF6002021020100F00000003CE9002010F70020EA
:2005A00000000000799D01080CF700203710010030000000E8EF002004F80020000000006E
:2005C0002C92070800F80020161001000600000028ED002038F80020000000005C92070887
:2005E00034F800202F10010022000000ACF6002044F80020000000006292070840F80020D4
:200600002322010010000000B4EC00206CF80020000000008492070868F800201E0001007C
:2006200009000000A8EC002080F8002000000000949207087CF80020052001000C0000006A
:20064000FCEC002090F8002000000000A09207088CF80020F62101000C0000000C1801209C
:20066000B818012000000000AC920708B41801201C0202001C000000241801200C19012070
:2006800000000000296B0508081901201400010005000000DC1701202C19012000000000E3
:2006A000B892070828190120012001000C000000840E01203819012000000000BE920708CD
:2006C000341901200C400600E4000000A80C0120481901200000000035DB03084419012086
:2006E0000A90010024000000640C0120301A012000000000D50802082C1A01200E300300B0
:20070000BC010000A00A0120581A0120000000009D8A0208541A01201310010004000000D6
:2007200084150120181C012000000000CC920708141C01200101010004000000E4090120D7
:20074000201C012000000000000000001C1C01200001010004000000DC090120281C012072
:2007600000000000D0920708241C01200201010003000000D8090120301C01200000000031
:2007800075DB03082C1C0120220201001C0100006C130120381C012000000000496D05087B
:2007A000341C01201900010005000000542801209428012000000000D492070890280120E1
:2007C000150010007000000048260120A028012000000000000000009C2801200300010023
:2007E0000100000040260120142901200000000000000000102901202A0008006000000027
:20080000FC2101201C29012000000000398A0208182901202C0004001000000090290120EB
:200820008029012000000000018802087C29012029201400780000003C230120A429012052
:200840000000000000000000A02901201A0001000E000000A0210120202A01200000000038
:20086000DA9207081C2A01202B001200240000007C210120342A012000000000D587020892
:20088000302A012019020100100000001C2101205C2A01200000000051610508582A01204A
:2008A00025201E002C0100000C310120C03801200000000000000000BC3801200312010006
:2008C0003D000000A4330120F039012000000000E8920708EC390120F8310100060000009A
:2008E000E42D0120343A01200000000026930708303A012010100100020000007C2C0120F8
:20090000403A0120000000002C9307083C3A0120020001000C000000A83C0120403D012025
:2009200000000000000000003C3D01202902010040000000243B0120503D01200000000083
:200940002E9307084C3D01202C020100040000005C3C0120943D0120000000006E9307082F
:20096000903D01200A02010014000000803B0120BC3D01200000000001DB0308B83D012075
:20098000280204000400000008450120D04601200000000009620508CC46012027020400A8
:2009A0000400000004450120D846012000000000FD610508D44601201F02080010000000AB
:2009C00040420120E046012000000000F5600508DC4601201A0201003C000000E83D0120E9
:2009E000F446012000000000ED6D0508F04601203820010003000000DC3D012034470120AC
:200A000000000000729307083047012004000800800000000048012080490120000000004B
:200A200000000000004A01202B0201000C000000A44B01205C560120000000007693070816
:200A4000585601201D020200060000003C5601207056012000000000000000006C56012023
:200A60002700010004000000E04F0120FC6601200000000082930708F866012010020100C1
:200A800001000000149801201098012000000000869307080C9801200403090412010002A9
:200AA000EF0201408304563200020102030100001201000202020040830440570002010270
:200AC00003010000FFFFFFFF00000000000000000100000000000000000000004C3C00206D
:200AE0000000000001000000000000000000000000000000000000000000000000000000F5
:200B0000000000000000000000000000000000000000000000000000006002401060024081
:200B2000000000000000000000000000000B00000000000000000000000000000060024008
:200B400028600240010000000000000000000000060C0000000000000000000000000000B8
:200B60000060024040600240020000000000000000000000100D00000000000000000000D2
:200B8000000000000060024058600240030000000000000000000000160E00000000000092
:200BA00000000000000000000060024070600240040000000000000000000000200F00004E
:200BC000000000000000000000000000006002408860024005000000000000000000000044
:200BE0002610000000000000000000000000000000600240A06002400600000000000000D5
:200C0000000000003011000000000000000000000000000000600240B86002400700000090
:200C20000000000000000000362F00000000000000000000000000000064024010640240F3
:200C40000000000000000000000000000038000000000000000000000000000000640240B6
:200C6000286402400100000000000000000000000639000000000000000000000000000066
:200C80000064024040640240020000000000000000000000103A000000000000000000007C
:200CA000000000000064024058640240030000000000000000000000163B0000000000003C
:200CC00000000000000000000064024070640240040000000000000000000000203C0000F8
:200CE00000000000000000000000000000640240886402400500000000000000000000001B
:200D00002644000000000000000000000000000000640240A0640240060000000000000077
:200D2000000000003045000000000000000000000000000000640240B86402400700000033
:200D40000000000000000000364600000000000000000000000000007D0000000985000804
:200D60000585000801850008F5840008F1840008FD840008F9840008000000007196000838
:200D8000A9A90008D58F000805AB0008419700088D8500086585000849850008F9A2000870
:200DA00075880008658A000861900008DD900008A5910008798500085185000841850008D9
:200DC000010000000000803FC53E0108C9430108413F0108D5120108B9140108E5120108E3
:200DE00001130108AD1201089D120108000000000000000009022000010104C03209040026
:200E0000000208065005070581024000000705010240000009026400030100C032090400DD
:200E20000001030000000921110100012236000705830309000A080B01020202010009044C
:200E400001000102020100052400100105240100020424020205240601020705820308002E
:200E6000FF09040200020A000000070501024000000705810240000009024300020100C029
:200E80003209040000010202010005240010010524010001042402020524060001070582BE
:200EA000030800FF09040100020A000000070501024000000705810240000000FF000000F1
:200EC000140000FF0000000000000000AA550701000001AA55050100002D202D2D202D2DD1
:200EE0002D2D202D2D2D2D000000000000000000000000000000000008000000FC8506082D
:200F0000FF1FFF1FFFFFFFFF05010905A101A1000501093009310932093309350934093698
:200F200009371581257F75089508810205091901290815002501950875018102C0C00000F0
:200F400009022200010100E03209040000010301020009211101000122360007058303090C
:200F6000000A000000000000010203040102030406070809AA550B010000AA550501000025
:200F8000AA550902000000AA5503009F01000000C0120000CCE8002000000000A4E8002053
:200FA000000000007EFF010000000100E0010000FFFFFFFFFF000000FFFFFFFF08FF0101D1
:200FC000FF0100000100000025FE01080000000000000000448B06081C1001207010012019
:200FE000000000000000000000000000DCA2060800000000000000000000000094A3060820
:2010000000000000000000000000000040A30608000000000000000049130208A2110120A5
:20102000FF0101004934020800000000000000005CA40608A9370208000000000000000030
:2010400014A406082D202D2D202D2D2D2D202D2D2D000000000000000000000000000000A8
:2010600000000000FFFFFFFF6118020800000000000000006CA2060801000000FA000000DA
:201080000100000001000000010100000001010100000000EE0D01200000F4010100000037
:2010A000EC0D01200000F40101000000EA0D01200000F40101000000E80D01200000F40107
:2010C00001000000E60D01200000F40101000000E40D01200000F40101000000E20D0120ED
:2010E0000000F40101000000D106020895060208000000000C8D0608D20D01200532010095
:20110000E00D01206400F40101000000DE0D01206400C40901000000D00D0120E803D00769
:2011200001000000CE0D0120E803D00701000000CC0D0120E803D00701000000CA0D01203A
:201140001E00B80B01000000D80D012005000F0001000000DA0D012003000A00010000007C
:20116000C80D01201E00F40101000000DC0D012002000000988D0608C60D012014006400BA
:2011800001000000D40D01203200E80301000000C40D01200000C80001000000A50C0120A1
:2011A00000C80100A40C012000500100A30C0120005A0100A10C012002000000008D0608AE
:2011C000D00A0708D80A0708A01101200100C409000000009E1101200100C40900000000F7
:2011E0009C1101200100C409000000009A1101200100C40900000000961101200100C40923
:2012000000000000981101200100C40900000000941101200100C4090000000092110120DE
:201220000100C40900000000030A012000C80100020A012000C80100000A01200000FFFFCA
:201240000A000000FE0901200100C80001000000FC0901203200307532000000FA0901203F
:201260007EFF140005000000F809012005002C0105000000F7090120055A0500F4090120DC
:2012800000FF0100F609012002000000C0080020F209012003000000B4870608F3090120BF
:2012A00000FF0100F509012002000000C0080020F109012003000000B48706085009012044
:2012C000FF7F01004C09012000000000FFFFFFFF010000004809012000000000FFFFFFFFAE
:2012E000010000004409012000000000FFFFFFFF0100000025060208B50502080000000089
:20130000E88D0608940E0120EE02CA0801000000920E012000C8010064000000910E012016
:2013200002C8010064000000900E012002000000A48D0608EA0901200000803E05000000A7
:20134000E809012080C1803E05000000E20901200083007D05000000E009012080C1803E5D
:2013600005000000DB09012000FF0100D40901206400F40101000000D20901206400F401B6
:2013800001000000D00901206400F40101000000CE09012004000000F48E0608CD09012075
:2013A00002000000088F06088F0A01200D000000148F06088C0A0120006401008A0A01203D
:2013C000320010270A000000880A01200D000000148F0608870A01200D000000148F0608B9
:2013E000860A012002000000B08D06080000000000000000000000004C8F0608990E01203E
:2014000046000000848F0608970E012003000000A0900608980E012004000000BC8D06083C
:20142000910A012003000000B0900608900A012003000000B0900608920C0120000A0100C9
:20144000900C01200000E803010000008E0C01200000E803010000008C0C0120000A010078
:201460008A0C01200000E80301000000880C01200000E803010000005C0C0120C800E803EC
:2014800001000000620C01203C00FA0001000000600C01200100E803010000005E0C012080
:2014A00000050100A00C012002000000D08D06089E0C01200000F401010000009C0C012062
:2014C0000000F401010000009A0C01200000F40101000000980C01200000F401010000009E
:2014E000960C01200000E80301000000940C01200000E80301000000B20D0120006401004B
:201500000A000000B10D0120006401000A0000009F0D0120196401009E0D0120020000005A
:20152000DC8D06089C0D0120E803D0070A0000009A0D0120006401000A0000008F0D0120AA
:20154000006401008E0D012000640100960D0120006401000A000000950D012000640100AA
:201560000A000000940D0120006401000A000000990D012000FF01000A000000980D012099
:2015800000FF01000A000000970D012000FF01000A000000930D012001FF01000A000000A6
:2015A000920D012001FF01000A000000910D012001FF01000A0000009A0A01200000F401DC
:2015C00001000000980A01200000E80301000000960A01200000E80301000000940A0120EF
:2015E0000000E80301000000920A01200000E80301000000F311012000960100EA1101207E
:2016000000C80100E911012000640100E811012000640100E711012000640100E61101206C
:2016200000640100E5110120FF080100E411012001640100A5040208690402080000000080
:20164000C0900608ED11012001320100EC1101200100000030910608EB11012004000000CA
:2016600038910608E311012000960100E211012000640100E01101201400E803010000005C
:20168000DE110120000030750A000000DC11012000C80100DB11012000C80100DA110120D2
:2016A00000C80100F011012000320100F211012000140100F1110120004B0100EF11012043
:2016C000040000004C910608EE110120006401000A000000BE0D01200AC805000A000000BF
:2016E000BD0D0120010000005C910608C00D01200AC805000A000000BF0D01200100000046
:201700005C910608B50D012000C805000A000000BC0D012000C805000A000000B60D01206F
:2017200000C805000A000000B70D012000C805000A000000BA0D012000C805000A00000057
:20174000BB0D012000C805000A000000B90D012000C805000A000000B80D012000C8050058
:201760000A000000B40D01200200000064910608021201200000D00701000000FC1101203D
:2017800000C80100FB11012000C80100FA11012000C80100001201200000D007010000008A
:2017A000F911012000C80100F811012000C80100F711012000C80100FE1101200000D00749
:2017C00001000000F611012000C80100F511012000C80100F411012000C80100081C070805
:2017E0000000000000009A180120141C0708070800000000D40E00201C1C07080708000070
:201800000000CC0E0020241C0708070800000000C40E00202C1C0708080800000000B80E51
:20182000002000070708070800000000B00E002008070708070800000000A80E002010076B
:201840000708070800000000A00E0020BC070708080800000000940E0020341C0708071082
:20186000000000008C0E00203C1C0708071000000000840E0020441C0708071000000000F8
:201880007C0E00204C1C0708081000000000700E0020380A0708010000000000000000001F
:2018A00000000000100000000000000000000000390202081D0202083D180208709106083C
:2018C000830A0120005A0100820A012000C80100800A0120E803D00701000000000000001B
:2018E00000000000891302080C920608F00901200300000054920608EF0901200003010068
:20190000EE09012000030100590102080D0102080000000064920608CD00020885000208C5
:201920000000000000930608A5010208211802080000000080930608EC09012001030100D7
:20194000F1FD0108D1FD010800000000F496060891070208650702080000000074970608F0
:20196000F5FF01089DFF010800000000E497060849020208AD3F0208000000009C980608AF
:20198000A91D0208BD0702080000000044990608990202080000000000000000E099060892
:2019A0007D0302081D03020800000000449A060825040208E103020800000000FC9A0608C2
:2019C00049770208E104020800000000889B0608C20D012001060100E1020208AD0202087F
:2019E00000000000A09C060865760208E919020800000000109D060811050208091B0208A3
:201A0000000000008C9E06088D770208C91A020800000000DC0E0020C10D01200103010095
:201A2000ED010208BD01020800000000989F0608C11702080000000000000000FC9F060816
:201A40004D000208091802080000000098A0060800000000000000000000000034A10608DB
:201A60008D050208551C020800000000B4A10608000000000000000000000000DCA306085F
:201A800084D500209CFF2C01000000001C150120E0150C17000000001E1501200200000045
:201AA00014A70608C809012088136F1701000000CA09012088136F1700000000986D00200F
:201AC0000000000000000000966D00200000000000000000946D00200000000000000000C2
:201AE000926D00200000000000000000906D002000000000000000008E6D0020000000008F
:201B0000000000009006002000000000000000005109012003000000F8A40608C0090120FD
:201B200088136F1701000000F6D9002088136F1700000000DDFE010800000000000000008F
:201B400008A506085D110120010000005CA50608F8D900200100000068A50608EED9002037
:201B60000200000070A506080000000000000000000000007CA50608C5FE01080000000045
:201B80000000000018A606080000000000000000000000006CA60608000000000000000059
:201BA00000000000DCA60608CC0901200200000014A70608F2D90020E0150C1700000000D1
:201BC00001F11F3FD60100003986020894A00020FFFFFFFF0000803F000000000000000006
:201BE000000000000000000000000000000000000000000000000000000000000000803F26
:201C00000000000000000000000000000000803F0000000000000000000000000000803F46
:201C2000000000000000000000000000010000000000FA430000FA43C5CE0408000000008A
:201C400000000000000000000000803FFFFFFFFFFF00000060FECD0000000000A83D012099
:201C60000800000000000000983D0120080000001D3E0108C9130108B53D0108000000001A
:201C8000991201089D460108053D01085139010800000000000000005912010819850008AC
:201CA0000D850008618F00087D8F0008458F0008298F00080D8F0008D53D0108A513010862
:201CC000093D0108000000007112010855390108D93C0108B1380108000000000000000082
:201CE00065120108C9E20308000000000000000000000000995004080000000000000000B9
:201D000000000000E83C0708B800070800000000FDDB0308A086010004000000E83C070888
:201D2000F03C07080000000079540408E803000004000000E01007080000000000000000A1
:201D40004D4703087D000000FF000000E40E07080000000000000000195F03087D00000067
:201D6000FF000000101407080000000000000000E57F03087D000000FF00000078110708AE
:201D8000000000000000000059CF0408E803000003000000F83C07080000000000000000DE
:201DA000E51C0308102700000300000040870708000000004986020875B704085F76000021
:201DC00005000000F48A0708000000000000000091E004081027000002000000043D07086B
:201DE000000000000000000059520408E803000005000000103D07080000000000000000E0
:201E000049DE0308204E000003000000203D0708000000000000000045DC0308204E000019
:201E200003000000303D07080000000000000000F9D40408400D030003000000282E070892
:201E4000000000000000000041CC04081027000002000000E400070800000000000000003D
:201E60006DE301081027000003000000380D07080000000000000000F1500408A861000025
:201E800002000000442E0708000000000000000085810408A00F000002000000403D070870
:201EA0000000000000000000C1CC01081027000002000000281E070800000000797F0108FD
:201EC00015C001088545010002000000F80C07080000000000000000091A010810270000E1
:201EE00002000000CC0007080000000000000000A148020850C30000020000004C3D070865
:201F0000000000000000000049240108400D030001000000543D070800000000000000005A
:201F2000AD500408400D0300020000005C3D07080000000000000000E1F2010850C30000AF
:201F400003000000683D070800000000000000006DED030840420F0001000000743D070813
:201F60000000000000000000DDE4030850C3000001000000803D07080000000000000000B5
:201F8000A16A0108102700000200000001000000A00F0000B80B00000102FFFF010000007F
:201FA000FFFF00001C87070800000802050303000000000028870708010008020504030087
:201FC00000000000348707080000080205030300000000003C870708010008020504030039
:201FE000000000005C2D07080200FE0101100300000000002C0E07080300140200030000CF
:020000040800F2
:20200000000000004487070804001F0202000800000000004C87070805001F0202010800A4
:2020200000000000FFFFFFFF1A030000000000000000000000000000000000000000000087
:20204000000000000403090412010002000000408304205700020102030101005D74050831
:2020600031740508D5730508B5620508F173050895730508B1620508B41B002051750508CD
:20208000717505084175050895620508FD740508B574050885620508901B0020696E05082F
:2020A0009D6205089962050891620508B96E05088D6205088962050840FA06083946010814
:2020C00085130108194501080000000000000000B13C0108C13B01080000000000000000FD
:2020E000000000004D1201083D63050831630508C1750508DD750508E9620508A575050809
:202100008975050802000000000000008C1B0020685601200200000001000000A9640508EF
:20212000881B0020000000000100000001000000E16405080418002000000000000000004C
:2021400000000000000000000000000000000000000000000100000000000000000000007E
:2021600000000000000000000100000000000000000000000000000000000000010000005D
:2021800000000000D8000000000000000500000006000000FFFFFFFF03000000000000005D
:2021A00005000000050000000000185006000000D007000001040C0001011860070000003E
:2021C000A00F000002040E0002031870070000000A1A000003040C000305189006000000BB
:2021E000204E000000020C000000000097FFFFFF81060000C4090000C409000003000000AB
:20220000881300000101000094FFFFFFE40C0000B80B0000C409000006000000881300006F
:202220000203000090FFFFFFEF160000AC0D0000C40900000A0000008813000003050000D4
:202240008BFFFFFF0B480000A00F0000C4090000000000008813000000010000204E00001D
:202260000000000000000000841B0020000000000400000000000000F98305080000000012
:2022800000000000000000000100000000000000801B002000000000020000000000000080
:2022A00000000000000000000000000008000000010000004983050800000000000000003C
:2022C00000000000010000000000000086000000CC1900200000000004000000000000006E
:2022E0002985050800000000000000000000000001000000000000006C1B00204C560120B8
:2023000004000000000000009D83050800000000000000000000000001000000000000008B
:202320007C1B0020000000000400000000000000F983050800000000000000000000000059
:202340000100000000000000781B002054560120040000000000000009890508000000005B
:20236000000000000000000001000000000000001B000000701A0020000000000300000094
:2023800000000000000000000000000000000000080000000100000059830508000000004B
:2023A00000000000000000000100000000000000741B0020505601200400000000000000A2
:2023C000698305080000000000000000000000000100000000000000701B00200000000058
:2023E0000400000000000000F983050800000000000000000000000001000000000000004F
:2024000097000000001B00200000000003000000000000008D8305080000000000000000CA
:20242000000000000100000000000000010101001F0000001C0000001F0000001E00000020
:202440001F0000001E0000001F0000001F0000001E0000001F0000001E0000001F00000087
:202460000068214C0100000064FA0608150000008200FFFF170000001D0000008200FFFFD1
:202480001A0000008300FFFF0600000005000000008002021F00000053544D20202020205F
:2024A00050726F64757420202020202020202020302E3031008002021F00000053544D20E8
:2024C0002020202050726F64757420202020202020202020302E30312AFF000000000000D6
:2024E0000000000000000000010000000000000000000000000000000000000001000000DA
:2025000000000000FF000000F4010000A4000000000000000000000000000401000002001C
:2025200001000002100000000700000000000000000000000102030406070809C700000092
:202540000500000006FF00004C1C00200000000000000000000000000000000000000000E9
:2025600000000000000000000000000000000000000000000000000000000000000000005B
:2025800000000000000000000000000000000000000000000000000000000000000000003B
:2025A000000000000000000000000000FFFFFFFFFFFFFFFFFFFFFFFFFFFFFFFFFFFFFFFF2F
:2025C000FFFFFFFFFFFFFFFFFFFFFFFFFFFFFFFFFFFFFFFFFFFFFFFFFFFFFFFFFFFFFFFF1B
:2025E000FFFFFFFFFFFFFFFFFFFFFFFFFFFFFFFFFFFFFFFFFFFFFFFFFFFFFFFFFFFFFFFFFB
:20260000FFFFFFFFFFFFFFFFFFFFFFFFFFFFFFFFFFFFFFFFFFFFFFFFFFFFFFFFFFFFFFFFDA
:20262000FFFFFFFFFFFFFFFFFFFFFFFFFFFFFFFFFFFFFFFFFFFFFFFFFFFFFFFFFFFFFFFFBA
:20264000FFFFFFFFFFFFFFFFFFFFFFFFFFFFFFFFFFFFFFFFFFFFFFFFFFFFFFFFFFFFFFFF9A
:20266000FFFFFFFFFFFFFFFFFFFFFFFFFFFFFFFFFFFFFFFFFFFFFFFFFFFFFFFFFFFFFFFF7A
:20268000FFFFFFFFFFFFFFFFFFFFFFFFFFFFFFFFFFFFFFFFFFFFFFFFFFFFFFFFFFFFFFFF5A
:2026A000FFFFFFFFFFFFFFFFFFFFFFFFFFFFFFFFFFFFFFFFFFFFFFFFFFFFFFFFFFFFFFFF3A
:2026C000FFFFFFFFFFFFFFFFFFFFFFFFFFFFFFFFFFFFFFFFFFFFFFFFFFFFFFFFFFFFFFFF1A
:2026E000FFFFFFFFFFFFFFFFFFFFFFFFFFFFFFFFFFFFFFFFFFFFFFFFFFFFFFFFFFFFFFFFFA
:20270000FFFFFFFFFFFFFFFFFFFFFFFFFFFFFFFFFFFFFFFFFFFFFFFFFFFFFFFFFFFFFFFFD9
:20272000FFFFFFFFFFFFFFFFFFFFFFFFFFFFFFFFFFFFFFFFFFFFFFFFFFFFFFFFFFFFFFFFB9
:20274000FFFFFFFFFFFFFFFFFFFFFFFFFFFFFFFFFFFFFFFFFFFFFFFFFFFFFFFFFFFFFFFF99
:20276000FFFFFFFFFFFFFFFFFFFFFFFFFFFFFFFFFFFFFFFFFFFFFFFFFFFFFFFFFFFFFFFF79
:20278000FFFFFFFFFFFFFFFFFFFFFFFFFFFFFFFFFFFFFFFFFFFFFFFFFFFFFFFFFFFFFFFF59
:2027A000FFFFFFFFFFFFFFFFFFFFFFFFFFFFFFFFFFFFFFFFFFFFFFFFFFFFFFFFFFFFFFFF39
:2027C000FFFFFFFFFFFFFFFFFFFFFFFFFFFFFFFFFFFFFFFFFFFFFFFFFFFFFFFFFFFFFFFF19
:2027E000FFFFFFFFFFFFFFFFFFFFFFFFFFFFFFFFFFFFFFFFFFFFFFFFFFFFFFFFFFFFFFFFF9
:202800000828000800400008232042657461666C69676874202F2053544D33324634313157
:202820005358313238302028533453582920342E332E30204A756E202037203230323220A2
:202840002F2032313A31363A353320286E6F7265766973696F6E29204D5350204150493A82
:2028600020312E34340A2320636F6E6669673A206D616E7566616374757265725F69643AE1
:2028800020424546482C20626F6172645F6E616D653A2042455441465056463453583132C5
:2028A00038302C2076657273696F6E3A2037646636363039332C20646174653A2032303223
:2028C000322D30362D31325431333A34313A34325A0A0A626F6172645F6E616D652042458F
:2028E000544146505646345358313238300A6D616E7566616374757265725F69642042457D
:2029000046480A0A23207265736F75726365730A7265736F75726365204245455045522092
:2029200031204131340A7265736F75726365204D4F544F522031204230380A7265736F752A
:20294000726365204D4F544F522032204130300A7265736F75726365204D4F544F52203303
:20296000204231300A7265736F75726365204D4F544F522034204230370A7265736F7572AA
:202980006365204D4F544F522035204130380A7265736F75726365204D4F544F5220362007
:2029A0004131300A7265736F75726365204C45445F53545249502031204230310A726573B5
:2029C0006F757263652053455249414C5F54582031204130390A7265736F757263652053EE
:2029E000455249414C5F54582032204130320A7265736F757263652053455249414C5F5445
:202A000058203131204130380A7265736F757263652053455249414C5F52582031204131D5
:202A2000300A7265736F757263652053455249414C5F52582032204130330A7265736F75BD
:202A40007263652053455249414C5F5258203131204130380A7265736F75726365204C45E5
:202A6000442031204331340A7265736F75726365205350495F53434B2031204130350A72A8
:202A800065736F75726365205350495F53434B2032204231330A7265736F757263652053F7
:202AA00050495F53434B2033204230330A7265736F75726365205350495F4D49534F2031BF
:202AC000204130360A7265736F75726365205350495F4D49534F2032204231340A726573AD
:202AE0006F75726365205350495F4D49534F2033204230340A7265736F75726365205350C7
:202B0000495F4D4F53492031204130370A7265736F75726365205350495F4D4F5349203255
:202B2000204231350A7265736F75726365205350495F4D4F53492033204230350A7265734A
:202B40006F75726365204144435F424154542031204130310A7265736F75726365204144BB
:202B6000435F435552522031204230300A7265736F75726365204F53445F43532031204244
:202B800031320A7265736F757263652052585F5350495F43532031204131350A7265736F7B
:202BA000757263652052585F5350495F455854492031204331330A7265736F75726365200E
:202BC00052585F5350495F42494E442031204230320A7265736F757263652052585F535031
:202BE000495F4C45442031204331350A7265736F757263652052585F5350495F4558505219
:202C00004553534C52535F52455345542031204230390A7265736F757263652052585F53EC
:202C200050495F455850524553534C52535F425553592031204131330A7265736F757263BC
:202C400065204759524F5F455854492031204230360A7265736F75726365204759524F5FCA
:202C600043532031204130340A0A232074696D65720A74696D657220423031204146320A5F
:202C8000232070696E204230313A2054494D33204348342028414632290A74696D6572201C
:202CA000423038204146320A232070696E204230383A2054494D34204348332028414632DC
:202CC000290A74696D657220413030204146310A232070696E204130303A2054494D32201C
:202CE0004348312028414631290A74696D657220423130204146310A232070696E20423102
:202D0000303A2054494D32204348332028414631290A74696D657220423037204146320A2F
:202D2000232070696E204230373A2054494D34204348322028414632290A74696D65722076
:202D4000413038204146310A232070696E204130383A2054494D3120434831202841463144
:202D6000290A74696D657220413130204146310A232070696E204131303A2054494D31207A
:202D80004348332028414631290A0A2320646D610A646D6120414443203120300A23204170
:202DA000444320313A20444D41322053747265616D2030204368616E6E656C20300A646DFD
:202DC000612070696E2042303120300A232070696E204230313A20444D41312053747265A6
:202DE000616D2032204368616E6E656C20350A646D612070696E2042303820300A2320700B
:202E0000696E204230383A20444D41312053747265616D2037204368616E6E656C20320A9C
:202E2000646D612070696E2041303020300A232070696E204130303A20444D41312053744F
:202E40007265616D2035204368616E6E656C20330A646D612070696E2042313020300A2369
:202E60002070696E204231303A20444D41312053747265616D2031204368616E6E656C20F5
:202E8000330A646D612070696E2042303720300A232070696E204230373A20444D41312069
:202EA00053747265616D2033204368616E6E656C20320A646D612070696E2041303820306C
:202EC0000A232070696E204130383A20444D41322053747265616D2036204368616E6E65E8
:202EE0006C20300A646D612070696E2041313020300A232070696E204131303A20444D41DF
:202F0000322053747265616D2036204368616E6E656C20300A0A2320666561747572650A27
:202F20006665617475726520534F465453455249414C0A666561747572652052585F5350C7
:202F4000490A666561747572652054454C454D455452590A66656174757265204C45445F0D
:202F600053545249500A66656174757265204F53440A0A23206D61737465720A736574206A
:202F800072785F7370695F627573203D20330A7365742072785F7370695F6C65645F696E6E
:202FA00076657273696F6E203D204F4E0A736574206473686F745F6275727374203D20410C
:202FC00055544F0A736574206473686F745F62697462616E67203D204F46460A736574205D
:202FE00063757272656E745F6D65746572203D204144430A73657420626174746572795F3D
:203000006D65746572203D204144430A7365742069626174615F7363616C65203D2038308B
:20302000300A736574206265657065725F696E76657273696F6E203D204F4E0A73657420AB
:203040006265657065725F6F64203D204F46460A7365742073797374656D5F6873655F6DED
:20306000687A203D20380A736574206D6178373435365F7370695F627573203D20320A73A7
:203080006574206779726F5F315F62757374797065203D205350490A736574206779726FDB
:2030A0005F315F737069627573203D20310A736574206779726F5F315F73656E736F725FBE
:2030C000616C69676E203D20435739300A736574206779726F5F315F616C69676E5F7961FB
:2030E00077203D203930300A73657420657870726573736C72735F646F6D61696E203D201E
:2031000049534D323430300A0A00FFFFFFFFFFFFFFFFFFFFFFFFFFFFFFFFFFFFFFFFFFFF02
:20312000FFFFFFFFFFFFFFFFFFFFFFFFFFFFFFFFFFFFFFFFFFFFFFFFFFFFFFFFFFFFFFFFAF
:20314000FFFFFFFFFFFFFFFFFFFFFFFFFFFFFFFFFFFFFFFFFFFFFFFFFFFFFFFFFFFFFFFF8F
:20316000FFFFFFFFFFFFFFFFFFFFFFFFFFFFFFFFFFFFFFFFFFFFFFFFFFFFFFFFFFFFFFFF6F
:20318000FFFFFFFFFFFFFFFFFFFFFFFFFFFFFFFFFFFFFFFFFFFFFFFFFFFFFFFFFFFFFFFF4F
:020000040800F2
:20400000AEBE08000E02000000000B0014020000000000FF000A00130200000000010010CC
:20402000000301010004040200A8160000000052000D000100010000001405040500000030
:2040400000000000000005040500000000000800000105040500000000000000000505042D
:204060000500000000000000001E05040500000000000000001F050405000000006400522C
:2040800000070009020000002A00FD0100001912000000000000000018001A130000000076
:2040A0000000000018000000000000000000000000000700FB010000000F00FC01000000D9
:2040C00000000000000000000C00F70100001E01000000000A00F90100003E000000450036
:2040E000160200002102002801001001002A01002701001801001A010000000000000000C4
:2041000000000000000000000000000000000000000000000000000000000000000000009F
:20412000000000160034000000DC0532000000000000000000000001040E001102000000FC
:20414000000000010101010A0012020100FFFFFFFF3E0018000300000103020405060709C2
:20416000000000000001006400DC051A04D0070019750343080E000001000000001E1E1EBF
:204180000101000000000000000000000000001100000200000000000000FF00000000000B
:2041A0000B00FF0102000000000000150008020100151617FFFF2D2E2FFFFF232425FFFFA0
:2041C0000900FA0100000000000E002A02000078005802F40101000E00200205000364320B
:2041E00000F40196002A0006000100E001060000020128102A27181A00000001000001025A
:20420000030405060758022E04D007E8030C000A000C020000012C02001A00FE01000001CA
:2042200011000001200000010000000000000000FFFF008200FD070000E4008209ED084E15
:2042400000CE00EA00970958098B092209EA007601EA00EA00EA00EA00EA00EA00EA00EA35
:2042600000EA002939EA00EA00EA00EA00EA00EA00EA00EA00EA00EA00EA00EA00EA00EA26
:2042800000EA00EA00EA00EA00B600EA00EA00EA00EA00EA006209EA00EA00EA00EA00EA31
:2042A00000EA00EA00EA004209EA002300EA00EA00CD00EA007200F50109009808640014D4
:2042C00001000A010A00007F1F0000142800002C3700008000FFFFFFFF46000102000000C6
:2042E0000000000000000000000000000000000000000000000000000000000000000000BE
:2043000000000000000000000000000000000000005000C4FF00FFFFFFFF01000000051870
:204320000B0C00000000001600230002000A000000FCFFFCFF0C00010000000000160012F6
:204340000003000000000100010553345358000008020020000B000300AE014A015E012C64
:204360000164010100000001000A019A01001E0A0000022A001F00050000000000000100B6
:2043800001000500000102030000000000000000000000000000000000008017000A00056B
:2043A0000200000000000011000102000000000000020000000000000900020200000000D8
:2043C0000016001B02000006000000E8030000000000000000000012001B00020000210069
:2043E000020301F40132000164F600210200000002000010020000000000000000000000FE
:2044000000000000000000000000000000000000000000000000000000000000000000009C
:2044200000000000000000000000000000000000000000000000000000000000000000007C
:2044400000000000000000000000000000000000000000000000000000000000000000005C
:20446000000000000000000000000000000000000000000000FFFF000000FF1E0000FF3CE6
:204480000000FF5A0000FF780000FF960000FFB40000FFD20000FFF00000FF0E0100FF2C0B
:2044A0000100FF4A0100FF0000000000000000010B020D0A03050B030D0A030A0B040D0A2D
:2044C00003080B040D0A03070B030D0A03000000000000060A010000020306000000033624
:2044E000003700010020003200C800D00796001400320028004C0440060005500014000F81
:2045000000080064000100000005000A000000F40196000F000C0016000100C4090000B4E1
:204520000028002F0001004D6574656F72383500000000000000000000000000000000004A
:20454000000000000000000000160023020200000000000000000000000000FF0000000F10
:20456000001E000000000501000000000000120005000200020300000000000000000000F9
:204580001200F601020000000000010000000000000022001C020000000201140000260290
:2045A00000000000840301020000000000010000000000000B001400000003010023001218
:2045C0000001000200E80364000F0A00010A001E00EA000C00040032000307070700000003
:2045E000414141440046050064CE07CE07CE07010000000000000000000000000032000350
:20460000070707000000434343410046050064CE07CE07CE0701000000000000000000004C
:20462000000000320003070707000000434343410046050064CE07CE07CE070100000000F7
:20464000000000000000000000320003070707000000434343410046050064CE07CE07CEDF
:20466000070100000000000000000000000000320003070707000000434343410046050093
:2046800064CE07CE07CE070100000000000000000000000000320003070707000000434366
:2046A00043410046050064CE07CE07CE0701000000000000000000000000002A000A00090A
:2046C00000300000000000F40100000000000000000000020000029E077D00FA00F40100A0
:2046E0000105016400C2010E00030064004B00000000002D341F0084002F36230089002D8A
:20470000340000840032324B0000002800000000000055F401900101374B000000FA00AC06
:204720000D00000000320090015E01F40100000A64C8009001960000050F00010F031400BD
:204740004B3200005A140B00004B009600001400280100C8001E22002514640000000000A0
:20476000000000000000003232329600001E070F5A0500000264644164640F6E01646464FD
:20478000004B00000000002D50280078002F542E007D002D500000780032324B00000028B7
:2047A00000000000000055F401900101374B000000FA00AC0D00000000320090015E01F4D2
:2047C0000100000A64C8009001960000050F00010F0114004B3200005A140B00004B00966B
:2047E00000001400280100C8001E22002514640000000000000000000000003232329600AB
:204800000019070F5A050000026464646464646401646464004B00000000002D50280078B7
:20482000002F542E007D002D500000780032324B0000002800000000000055F401900101A2
:20484000374B000000FA00AC0D00000000320090015E01F40100000A64C8009001960000AF
:20486000050F00010F0114004B3200005A140B00004B009600001400280100C8001E2200E3
:2048800025146400000000000000000000000032323296000019070F5A0500000264646493
:2048A000646464640164640A0013000100000444120A0001010000000000000A0000010010
:2048C00000200300000900020100006E0A012201220200000508E916D516C116AD169916A9
:2048E000851671165D16651678168B169E16B116C416D716EA164916351621160D16FD1620
:204900001117251739176C1680169416A816BC16D016E416F8161A163F1664168916AE1641
:20492000D316F8161D1700000000000000000000000000000000000000000000000000004C
:2049400000000000000000000000000000000000000000000000424F5343414D5F410042C0
:204960004F5343414D5F4200424F5343414D5F4500464154534841524B00524143454241D8
:204980004E440042414E44362020200042414E44372020200042414E4438202020004142FE
:2049A0004546523637383100320033003400350036003700380001010101010000000400C8
:2049C00000000100020003000000000000000000323520003130300032303000333530008F
:2049E0004C5634004C5635004C5636004C5637000B00190000000000280100760015000081
:204A0000000000000000000000000000000000000000000000000000000000000000000096
:204A2000000000000000000000000000000000000000000000000000000000000000000076
:204A4000000000000000000000000000000000000000000000000000000000000000000056
:204A600000000000000000000000000000000000000700030000000066002A00000000009C
:204A80000000E803D007DC0564FF00000000E803D007DC0564FF00000000E803D007DC0567
:204AA00064FF00000000E803D007DC0564FF00000000E803D007DC0564FF00000000E8039C
:204AC000D007DC0564FF00000000E803D007DC0564FF00000000E803D007DC0564FF160099
:204AE0002C000000E803D007E803D007E803D007E803D0077E002900020000002030000089
:204B00000101001000000201102000000B03203000001B0220300000000000000000000085
:204B2000000000000000000000000000000000000000000000000000000000000000000075
:204B4000000000000000000000000000000000000000000000000000000000000000000055
:204B600000000000000000000000000000000000000014001A0000007E05EA05B4053200AA
:204B8000E803D00700002A002B000000001E001E001E0005011E011E011E011E011E011EE5
:204BA000011E011E011E011E011E011E011E011E1600190200001300000000000000001F9A
:204BC00003223F013D003201250002000000000000000000000000000000000000000000D9
:204BE0000000000000000000000000000000000000000000000000000000000000000000B5
:204C0000000000000000000000000000000000000000000000000000000000000000000094
:204C2000000000000000000000000000000000000000000000000000000000000000000074
:204C4000000000000000000000000000000000000000000000000000000000000000000054
:204C6000000000000000000000000000000000000000000000000000000000000000000034
:204C8000000000000000000000000000000000000000000000000000000000000000000014
:204CA0000000000000000000000000000000000000000000000000000000000000000000F4
:204CC0000000000000000000000000000000000000000000000000000000000000000000D4
:204CE00000000000000000000000000000000000000000000000000043000302010000006B
:204D0000000000000000000000000000000000000000000000000000000000000000000093
:204D20000000000000000000000000000000000000000000000000000000010C00F801036A
:204D4000000101F40114000800100001000005120002000000000000000000000000000016
:204D60000046002902000000000000000000000000000000000000000000000000000000C2
:204D8000000000000000000000000000000000000000000000000000000000000000000013
:204DA000000000000000000A002C020000010001001A000A02000000004A01B400D60100BD
:204DC00000C2010E019600440000000A0028020000000000000A00270200000000000016AA
:204DE000001F020000FFFFFFFFFFFFFFFFFFFFFFFFFFFFFFFF42001A020000000000000044
:204E000000000000000000000000000000000000000000000000000000000042454648007D
:204E20004245544146505646345358313238300000000000000100090038000200000A0725
:204E40008600040000000000000000000000000000000000000000000000000000000000C8
:204E6000000000000000000000000000000000000000000000000000000000000000000032
:204E8000000000000000000000000000000000000000000000000000000000000000000012
:204EA0000000000000000000000000000000000000000000000000000000000000000000F2
:204EC00000000000000012002B020000291D0000D1D8EA58000001FF0C001D020000000037
:204EE000000000000A0027000000200300000700100200000000000113000000FFFFFFFF35
:204F0000FFFFFFFFFFFFFFFFFFFFFFFFFFFFFFFFFFFFFFFFFFFFFFFFFFFFFFFFFFFFFFFFB1
:204F2000FFFFFFFFFFFFFFFFFFFFFFFFFFFFFFFFFFFFFFFFFFFFFFFFFFFFFFFFFFFFFFFF91
:204F4000FFFFFFFFFFFFFFFFFFFFFFFFFFFFFFFFFFFFFFFFFFFFFFFFFFFFFFFFFFFFFFFF71
:204F6000FFFFFFFFFFFFFFFFFFFFFFFFFFFFFFFFFFFFFFFFFFFFFFFFFFFFFFFFFFFFFFFF51
:020000040800F2
:020000040800F2
:20800000134B0268196821EA02011960596821EA0201596019680A431A609968026821EA4A
:2080200002019960D96821EA0201D9604179102907D001F1804303F59E3319680A431A602C
:208040007047996811439960D9680A43DA607047003C0140024B9A6D136A002BFCD170479F
:20806000B01C0020F0B401292D4C2E4D4FF0000694BF00230123EE62C4F81861C4F81C61B5
:20808000C4F82831D4F82871D4F8F43047EA4207C4F82871EE63EC6B002A38D144F495748B
:2080A000EC631C6824F001041C601C68E407FCD4490289085960D8601968EAB921F04001D6
:2080C000196019498B421DD018494FF47410C860196841F01E011960596941F08001596143
:2080E000196841F00101196022B90E4AD36A43F00803D362F0BC704741F0400119600A49CF
:208100008B42E1D14FF0746041F8500CE0E744F01A04EC63EC6A44F00804EC62C1E700BF85
:20812000B01C0020002C014058640240006402401248002302461178032902F1060218D0E5
:208140000133062BF7D10E4AD2F85031052B0FD0591C03EB4303C2F8501100EB4303032028
:2081600040F2EB3140F2FF32187059809A807047704703EB430300EB4303F0E7DC1D002010
:20818000B01C002030B5134A134B8DB0082102F1580082F8F0100693694400230DF10705B5
:2081A0000124CDE9073302938DF8143009938DF828300B93CDE9035445F0BEFDFFF74AFFF9
:2081C0009DF80700A0F1FF00B0FA80F040090DB030BD00BFB01C0020DD810008826D136AE9
:2081E0005B681B78FF2B08D090F8F030013BDBB280F8F0301BB10120704700207047126A27
:20820000526802201370704770B4C3080D4CE25C00F00706B24004EBD004D2B20020C6F1B5
:2082200008038B4228BF0B46C3F108052A419840C91A40EA02004FF0000614F8012FEED1DB
:2082400070BC7047F01C0020084AD2E9553199420AD0D118013391F85C110170C3F30A0380
:20826000C2F854310120704700207047B01C0020064BD3F86009D3F85C29D3F85C3982422B
:2082800098BF03F50063181A704700BFB01C0020012380F85130704707B501A8FFF7D4FF96
:2082A0000028FAD09DF8040003B05DF804FB044BD3E95503984288BF03F50063181A704764
:2082C000B01C002001207047024BC3F86429C3F868197047B01C0020024BC3F86C29C3F80E
:2082E00070197047B01C00207047704730B4134DD5E955239A4286BF03F50064A21A9A1A7D
:208300000A44B2F5006F13D8A9B101444A1E013810F8014FE918824203F1010381F85C41A3
:20832000C3F30A03F4D1C5F85831002030BC7047022030BC70470846F8E700BFB01C00200F
:2083400041B370B5144C0144D4F860394E1E451E1A4604E001203FF0E5FAD4F86029D4F897
:208360005C19531CC3F30A038B42F3D0D4F85C19B1F5006FEED094F874190029EAD115F8A8
:20838000011FC4F860392244B54282F87819DFD1002070BD00207047B01C002010B5094C26
:2083A000D4F88030084611465BB1D4F88030052B07D1002AD4F8843003DDFFF7C1FFD4F800
:2083C000843010BDA82D002010B590F85010002380F8503081B10B4CD4F8802072B1D4F87B
:2083E0008020052A0CD13C30D4F88430FFF7A8FFD4F88430012010BD0120FCE71046FAE79F
:208400001846F8E7A82D0020002280F85120DBE790F85020531C0244DBB280F8503082F8B1
:208420003C1090F851200AB1132B00D9CCE77047212838B50C4605D022282FD0202813D0EA
:20844000002038BD0029FBD0072AF9D11A4BD3F8880093F88C1093F88D2093F88E30206038
:2084600021716271A371EBE70029E9D0072AE7D1124AD2F868391BB1D2F8640909689847CC
:208480000D4B256820796179A279C3F8885083F88C0083F88D1083F88E20D1E70029CFD00E
:2084A000022ACDD1054AD2F87039002BC8D00988D2F86C099847C3E7A82D0020B01C002033
:2084C000024B0020C3F88000704700BFA82D0020054B064A00200521C2F88010C3F8700925
:2084E000C3F86809704700BFB01C0020A82D0020704700BF704700BF704700BF704700BF21
:20850000704700BF704700BF704700BF042301480B8070479801002010B4074A074B92F89D
:208520009000122403F114020C8001280CBF184610465DF8044B7047A82D00209C0100202A
:2085400000487047D81C002000487047D81C0020034B93F82400032894BF00200120704782
:20856000B01C0020034B93F82400032894BF002001207047B01C0020034B93F8240000387B
:2085800018BF0120704700BFB01C0020034B93F82400003818BF0120704700BFB01C0020F2
:2085A000A0B182680D4B12B107229A7070471978DA6003294FF004000CBF80214FF48071A1
:2085C000C3E901111A611A7598707047034B41F2E47101225A545A70704700BF44B7002012
:2085E0000378022B10D0006908B9012070470C4B1B78032B0EBF0B4B80B24FF6F7739842FB
:2086000094BF0020012070470549436841F650028A58B3EB422F2CBF01200020704700BFFA
:2086200044B70020F7FFFF0F0378022B14D030B4104A4368006941F6480402F5C251155942
:20864000096841F63C042B4012595B0A023801FB0030104430BC7047064B426841F6340133
:2086600041F630005958185800EB410000EB5220704700BF44B7002030B593B040F04002BE
:208680000B0E0D0C04468DF80810080A8DF80420952101AA8DF805308DF8065000230625C2
:2086A0008DF807008DF809100DF1030001210392134A0493CDE90733CDE90D33CDE909013E
:2086C0008DF818308DF82C300F938DF84030119305950C92FFF756FD00B974B9094B0822CC
:2086E00003F1580003A983F8F02045F025FBFFF7B1FC9DF8030013B030BDFF2013B030BDE8
:2087000009870008B01C0020836D1B6A5B681B78FF2B0AD190F8F030002B03F1FF3380F894
:20872000F03014BF0120022070470020704700BF30B5104A104B8DB0014682F8F01002F12B
:208740005800069302A900230DF107050124CDE9073302938DF8143009938DF828300B93C6
:20876000CDE9035445F0E8FAFFF774FC9DF807000DB030BDB01C00200987000870B51C4D17
:2087800090B00024FD220DF1030305F15800012601A98DF803200693CDE90144CDE90A44F3
:2087A000CDE90C442C628DF81040059407948DF824408DF838400F940396089645F0BCFA71
:2087C000FFF748FC3046FFF7B3FFFF2809D0094BD3F884306B612046092385F8243010B07F
:2087E00070BD0423022085F8243010B070BD00BFB01C0020A82D002070B5064690B00820CC
:208800000D46FFF795FFFF2821D0FE2802D0022010B070BD002402230E48089301A9CDE9C2
:208820000265CDE90544CDE90A44CDE90C4401948DF8104007948DF824408DF838400F943A
:2088400045F07AFAFFF706FC204610B070BD012010B070BD081D002008B5FFF7FBFB0A20FE
:208860003EF024FF024B186EBDE8084042F028BFB01C002070B50379254C002B14BF0122AF
:2088800000228AB084F8502003D184F824300AB070BD054690F9001004F1580045F0C2FBE2
:2088A000AD784DBB01261B482566C4F8EC4084F8646046F0A3F903464FF47A70A4F85C30DE
:2088C0003FF030F8206E42F0FBFE2822684600215FF009FC0A2310480293694645F02CFAF7
:2088E000FFF7B8FB0D4B84F82460D3F884306361002323760AB070BD284642F013FC054697
:2089000008B11E23C380092128463EF09FFAC9E7B01C0020801A0600081D0020A82D002045
:208920002DE9F84F494B98420ED003F56853083398424ED0464B0020C3E94000A3F8FC0074
:20894000A3F80801BDE8F88F414C424FDFF810810223C4F8943004F198060025FB6AAB4212
:20896000294605F1010503D0D4F8180153F09EFA94F81C31D4F8182186F82430326230463F
:20898000414653F0A7FCD4F894309D4206F13006E4DB002384F80A31D4E92803D4F89410DD
:2089A000B4F89C20B4F8A850C4F8283112FB01F203FB01F3A4F8FC20B4F89E10264AA4F886
:2089C0000851C4E94003A4F8FE10C4F8F8200120B8E71F4C1F4F0223C4F8943004F1980500
:2089E0004FF0000B4FF4806A4FF040094FF40068FA6A01265A455946B34403D0D4F8180155
:208A000053F054FAD4F8181194F81C21296285F824204FF400314FF00062C5E90212A5F847
:208A200004A0A5F81090A5F80680AE74FFF780FB28466E7653F09AFBD4F89420074B45F866
:208A4000303B9345D4DB84F80A61A5E71971EF00A82D002098010020B48106088881060830
:208A60001940EF002DE9F843194C94F82460042E0546894690461F4608D0082E02D0002061
:208A8000BDE8F883FFF77AFE0228F8D1206E42F011FEA37E9BB969021120FFF7EDFDA0B93C
:208AA0000C4BC4F80090D3F8842065600523C4E90387626184F824300120BDE8F88329463D
:208AC0001120FFF7D9FD0028EAD0FFF7C5FED6E7B01C0020A82D00202DE9F04FCF4ED04DD1
:208AE00086468C4617460FCE05F596742DED068B0FC40FCE0FC496E8070089B095F862318E
:208B0000039784E80700CDE904EC042B00F24881DFE813F0B401460141010500C4019FED5A
:208B2000C18ADFEDC18AC149C5F84811C049C14BC14AC5F844110399002918BF134638EE66
:208B4000887AF5EE006AC6EE879ABC4EC5F85031A6F1120B06F1C0080027DFEDB97A9FED84
:208B6000B99A28EE278AB0EE67AA059BBB4200F00C811BF8013BEA1892F86741002C00F073
:208B80001481002202E0152A00F00F8102EB42014FEA420918F80100A04202F10102F2D11D
:208BA000294491F84512002900F06681204602933DF0FAFE029B8246504602933DF014FF78
:208BC0000178002940F0F180029BA9440133DBB2032289F8853289F88422BAF1000F00F0D9
:208BE000E4804FEA141909F1FF39B9F1040F04F00F0000F20881944C04EB4901B1F884C038
:208C00004CFA00F111F0010100F0FD80012101FA00F0013800EA0C00A14402935CF0D6FFD6
:208C200099F890C0DFF838E2029B60440EEBC00C03228CF807308CF806205EF83000C6F88E
:208C400014C000F13F4303F57E0304EB9324012194F898309AF8082003F01F045B09032BD6
:208C600001FA04F100F00381042B00F0FB80022B00F0CF80BCF804300693B3FA83F3C3F132
:208C80001F03C3F3CC0100EB810103F007030C6A9B004FF00F0C0CFA03FC24EA0C040C62C9
:208CA0000C6A02FA03F323430B62022306A907930CF004F8039B002B00F08380B5F8603119
:208CC000D5F8301507EE903AF8EEE77AFCEEE77A17EE900AB1FBF0F202F57F42FF32120CFD
:208CE000B1FBF2F295F86211B2FBF0F0042983B27ED007EE902AF8EE676A66EE887A29EED4
:208D0000677A95F8630104990091A8EEA67A019051463046C6ED027A86ED037A35F0F2FBCE
:208D2000002F72DD7368D5F8882193426FD0012F6BD0D5F8A021934269D0022F65D0D5F816
:208D4000B821934263D0032F5FD0D5F8D02193425DD0042F59D0D5F8E821934257D0052FAF
:208D600053D0D5F80022934251D0062F4DD0D5F81822D31A18BF012301370122082F337471
:208D8000727406F118067FF4F0AE304809B0BDEC068BBDE8F08F9FED2E8AF0EE488AC2E69C
:208DA0009FED2C8AF0EE488ABDE62B4A224BC5F848210020C5F8503109B0BDEC068BBDE820
:208DC000F08FB0EE690A5DF0FBFDFCEEC07A4FF6FF7317EE902AD5F83015B1FBF2F21A4424
:208DE000120CB1FBF2F295F862110429184680D107EE900A07EE102AF8EE677AF8EE476ACD
:208E000067EE8A7A7BE7716154E70123B4E70023B2E7124B5C6C214359642BE7E081060848
:208E2000A82D0020ACC5A737ACC5A7361942030859540408ED3E03084D5404082C2F002023
:208E40006F12833A00007A4488810608D42E0020282930386F1203393D4003080038024065
:208E6000583000200F4B1C6B2143196302E70D4B1C6C21431964FDE68A469DE69FED0A8A89
:208E80000A4A0B4BC5F84821C5F8443100220123CDE90332F0EE488A064B50E69FED068A4C
:208EA000EEE700BF003802406F12833A19420308595404084D54040800000000F8B5104E8F
:208EC000D6F83045054600680F4664080BF0FAFDB4FBF7F1B1F5803F03D3012CFAD96408AB
:208EE000F6E72246284689B23DF068FB054BC6F8983D28460449BDE8F84000223DF032BA3E
:208F0000A82D002001390208403B002010B5044C04480A4621460AF04FFC204610BD00BF2E
:208F2000483B002034FE060810B5044C04480A4621460AF041FC204610BD00BF483B00206A
:208F400044FE060810B5044C04480A4621460AF033FC204610BD00BF483B002050FE06088F
:208F600010B5044C04480A4621460AF025FC204610BD00BF483B00205CFE060810B5044CAC
:208F800004480A4621460AF017FC204610BD00BF483B002068FE060810B50C4C94F8F220FD
:208FA0000023236212B10A4AC2F8A03E56F006F820B10423022084F8243010BD044BD3F845
:208FC00084306361092384F8243010BDB01C0020A82D002070B50D4D95F82430042B044696
:208FE0000E460AD0082B06D1EB6983420CD0FFF7D3FF022801D0012070BD0823C5E907460D
:2090000085F82430022070BD022070BDB01C002010B50AF0A5FB0F4C48B194F82430032B34
:2090200011D8237E0133DBB2072B237603D9002384F8243010BD084A0123D2F884206261D7
:2090400084F8243010BD054845F0D8FDA4F85C00E7E700BFB01C0020A82D0020801A060016
:2090600070B51D4C94F82430042B06460D4608D0082B20D1E36983422BD0FFF77FFB022812
:2090800019D1206E42F016FB00213720FFF7F4FA29461720FFF7F0FAA8B9A37E6BB971021A
:2090A0001920FFF7E9FA70B90823C4E9076584F82430022070BD012070BD31461920FFF71E
:2090C000DBFA0028F0D0FFF7C7FBFFF7A1FF032070BD022070BD00BFB01C00202DE9F041F4
:2090E0002B4C0546884617461E4694F82400042834D0082806D1E369AB4206D0FFF73EFBFA
:209100000228F2D00120BDE8F0814FF0FC0CA26D2048117B204B80F8A4CEC3F8588051B1F8
:20912000526942B194F8E020002A0CBF4FF480724FF4007201E04FF480721A6617491848C0
:2091400044F0FAFD01220623C4E90085C4E90376227284F824300020BDE8F081206E42F0E6
:20916000A9FAA37E5BB969021820FFF785FA40B994F82430082BC8D04FF0FE0CC7E72946F5
:20918000F2E7FFF769FBFFF743FF0320BBE700BFB01C0020A82D002098010020C80100205D
:2091A000081D00202DE9F04FC64C94F8506095B0002E00F0818194F82420C34F04F158082B
:2091C00004F14009531E082B00F29680DFE813F034005A00200194008300A50019009400C3
:2091E0000900FEF7CFFF002840F01A826369D7F88420FA3393427CD2FFF70AFF94F8242051
:20920000E0E7FEF7BFFF0028F0D0236A0022012B227640F21B82E269013B511CC4E90713EF
:20922000082284F82420A2F10806B6FA86F67609304615B0BDE8F08F206E42F03BFA002183
:209240000846FFF719FA0546FFF706FB012D50D1206E4FF0000A84F819A042F02BFA40F291
:20926000AB110820FFF708FA052800F07A81012800F04281FFF7F0FA627E002AD1D002236E
:2092800084F82430206E42F015FA637E022B0CBF4FF08045002500213720FFF7EDF929466A
:2092A0002920FFF7E9F90546FFF7D6FA0DBB637E022B00F06981A576206E42F0FBF90021DC
:2092C0000920FFF7D9F9002873D0FFF7C5FA94F82420531E10E020684FF40071FFF78CFA94
:2092E000012800F02681022800F02A81002800F03A8194F82420531EDBB2022B0AD8724B7C
:209300006169D3F884305B1AC82B8CD9FFF780FE94F82420042A86D18AE7A26D117B136AE5
:20932000002900F0D5805269002A00F0D18094F8E020002A00F0CC80B3FA83F35B09002BF5
:20934000D7D004A900250DF10F0302220591404605A94FF0010ACDE90B3A0792CDE90955A4
:20936000CDE90E55CDE91055ADF8105006958DF820508DF834508DF84850139544F0DCFC4A
:20938000FEF768FE9DF80F3003F01F03052B00F05081FFF73DFED4F80CB0BBF1000F00F034
:2093A000DD802A46236961685046D84794F8242008E710214846FFF71FFA8246002884D104
:2093C00001217F20FEF720FF012805467FF47DAF50460221FEF718FF002800F0038101281B
:2093E0007FF473AF16213A20FEF70EFF01308002A062FFF731FA206E42F05CF900210A200F
:20940000FFF73AF9002840F0E680032384F82430102105A8FFF7F0F900287FF46AAF9DF869
:2094200021309DF822109DF81C209DF815009DF816501B01DBB243EA111303F5FA63638765
:20944000DDF81D3001F00F0184F83C101BBA110902F00F0245EA002084F8381084F8392047
:209460009DF814109DF817206363069B2363A08584F82E1084F82F20FFF7EEF9A37E6BB9AE
:20948000206E42F017F94FF400711020FFF7F4F80546FFF7E1F9002D7FF4AEAE0B4845F097
:2094A000ADFB00220423A4F85C003046226284F8243015B0BDE8F08F304684F8246015B0D5
:2094C000BDE8F08FB01C0020A82D002040787D012268217A4FF4807302EB0121404600223F
:2094E00045F0B6FC237A0133DBB22372A3F10203B3FA83F35B0922E7042304AA05A9404660
:2095000007930692CDE909AACDE90BAACDF814A08DF820A08DF834A0CDF838A044F00CFC55
:20952000FEF798FD9DF81330AB2B04BF02236376A0E66369D7F8842064339342BFF4D9AEC7
:20954000FFF78AF9FFF764FDE5683DB10022104623696168A84794F8242033E694F824208B
:2095600030E6657686E60190FFF776F9E56801982076042384F82430002D3FF459AED4E901
:2095800000212369A847B4E6206E42F093F829463A20FFF771F804AA8246042305A9404651
:2095A00006920793CDE90955CDE90B5505958DF820508DF834500E9544F0BEFBFEF74AFDEB
:2095C000BAF1000F07D1FFF747F9049B1BBAC3F38073A37670E6FFF73FF9FFF719FD94F871
:2095E0002420EFE504212C20FEF70EFE032182464E20FEF709FE0C2183463620FEF704FE48
:209600000BF1020B421C02FA0BF205FA0AF5A2FB0501420A42EAC152A262FFF71DF9EAE6DE
:209620000190FFF719F901980423064684F82430FEE50E4BE568D3F884306361072284F844
:209640002420002D3FF4EFAD504698E708D0042384F82430FFF700F994F82420531E4BE685
:20966000FFF78CF802287FF444AE2EE6A82D002070B50379204C002B14BF0123002384F80A
:20968000503003D1002384F8243070BD1B4D002195F9AB2E03203EF005FD0028F2D046687B
:2096A00030463EF0EDFC84F8F1000028EAD095F8A93E003B18BF0123304684F8F23056F0CA
:2096C000D7FB0AF04DF828B9237E84F824000133237670BD55F05CFD30B1237E00220133E7
:2096E000237684F8242070BDD5F8843063610123207684F8243070BDB01C0020A82D002007
:2097000010B555F045FD48B10B4C237E0133DBB2072B237603D9002384F8243010BD0AF0EA
:209720001FF80028F7D0054A0123D2F88420626184F8243010BD00BFB01C0020A82D002042
:209740002DE9F041844C94F85050002D00F0F28094F82420814E0227531E082B3FD8DFE8ED
:2097600003F035379C3E694F153E050055F026FC002840F0E6806369D6F88420FA3393423B
:209780002AD2FFF7BDFF94F82420E5E755F016FC0028F0D0236A0022012B227640F2D58046
:2097A000E16994F8F200013B0131C4E9071310B16A4BC3F8A02E082284F82420A2F1080523
:2097C000B5FA85F56D092846BDE8F08184F8247055F0F4FB002844D194F82420531EDBB217
:2097E000022B0AD85D4B6169D3F884305B1AC82BE4D9FFF785FF94F82420042ADED1E2E754
:20980000D4F82431002BD9D1544BE668D3F884306361072284F82420002ECFD0D4E900218E
:2098200023690120B047D7E76369D6F8841064338B42C3D2D4F82081B8F1000FF4D155F070
:20984000BDFB00289FD0E66884F81880042384F82430002E73D0D4E9002123694046B04708
:20986000BAE755F051F80028B6D196F8AD3E002BA3F10203B3FA83F314BF022201225B092C
:209880006276A37655F040F800287FF47AAF344A0323926CA26284F8243055F035F8002886
:2098A0009AD12E4B206293F8DC6EB3F8DE0ED3F8E0EED3F8E0CED3F8E07ED3F8E02E84F846
:2098C0002E6093F8E41EA08593F8E56E84F8322093F8E50ED3F8E82E6263B3F8EE8EB3F8A6
:2098E000EE2E84F83310B3F8EE1EC2F30B1343EA182303F00F0301F00F024FEA1E6E4FEA96
:209900001C4C3F0A360900F00F0003F5FA63042184F8390084F82FE084F830C084F8317015
:2099200084F83860638784F83C2084F824102846BDE8F08184F824502846BDE8F08105465E
:2099400041E7042384F824303DE7FAD1FFF724FB94F82420531E42E7B01C0020A82D002099
:20996000583C00202DE9F84FBA4C94F8081F0546C1F34001D4F8100F41F0A8FE94F8081F68
:20998000D4F80C0FC94301F0010141F09FFE002D00F0CD806E1EB04FB04D5FFA86FB4FF008
:2099A0001008D4F8100F41F075FED4F80C0F41F071FEB4F8183F002B40F0438194F81A1F92
:2099C000D4F81C0F41F082FE4FF0FA094FF47A704FF0010C7B68C3F30803002B40F008819C
:2099E000EFF31183002B40F00381D4F88420A968D4F884309A42F8D1D4F8403F9942F4D87A
:209A0000D4F83C6F00FB06F35B1AB3FBF6F300FB02327B68C3F30803002B40F0A880EFF397
:209A20001183002B40F0A380D4F88430D5F808A0D4F884108B42F7D1D4F8401F8A45F3D865
:209A4000D4F83C6F00FB06F1A1EB0A01B1FBF6F100FB03139B1AB3F57A7FDAD3B9F10109AB
:209A6000B8D1D4F8100F41F015FED4F80C0F41F011FEB4F8183F002B40F0D78094F81A1F8D
:209A8000D4F81C0F81F0010141F020FE4FF0FA0C4FF47A704FF0010E7B68C3F30803002B7E
:209AA00040F08680EFF31183002B40F08180D4F88420A968D4F884309A42F8D1D4F8403FAD
:209AC0009942F4D8D4F83C9F00FB09F35B1AB3FBF9F300FB02327B68C3F308034BBBEFF377
:209AE000118333BBD4F88430D5F808A0D4F884108B42F7D1D4F8401F8A45F3D8D4F83C9F8E
:209B000000FB09F1A1EB0A01B1FBF9F100FB03139B1AB3F57A7FDED3BCF1010CBCD10BF1C8
:209B2000FF365FFA86FBBBF1FF0F7FF43AAFBDE8F88FEFF3118988F31288AE682B68DB03BC
:209B400044BFC4F838EFAE68D4F88430D4F8381F5FFA89F989F31188D4F83C9F0B4400FB85
:209B600009F1891BB1FBF9F100FB0313D0E7EFF3118E88F31288D5F808A02B68D90344BF6C
:209B8000C4F838CFD5F808A0D4F88430D4F8381F5FFA8EFE8EF31188D4F83C6F0B4400FB2A
:209BA00006F1A1EB0A01B1FBF6F100FB031351E7EFF3118188F31288D5F808902B68DA03DD
:209BC00044BFC4F838EFD5F80890D4F88430D4F8382FC9B281F31188D4F83C1F1A4400FB7F
:209BE00001F3A3EB0903B3FBF1F300FB023272E7EFF3118188F31288AE682B68DB0344BFAA
:209C0000C4F838CFAE68D4F88430D4F8382FC9B281F31188D4F83C1F1A4400FB01F39B1B06
:209C2000B3FBF1F300FB0232F3E6D4F8343F002B3FF42CAFD4F8203FC3F8009084F8319F50
:209C400024E7D4F8343F002B3FF4BEAE3DF02AFFBAE600BFA82D002000ED00E010E000E0A9
:209C60002DE9F84FB74CB84F94F8081FD4F8100FB64DC1F3400141F029FD94F8081FD4F811
:209C80000C0FC94301F0010141F020FD4FF0050B4FF01008D4F8100F41F0FCFCD4F80C0FBB
:209CA00041F0F8FCB4F8183F002B40F0438194F81A1FD4F81C0F41F009FD32264FF47A70E5
:209CC0004FF0010C7B68C3F30803002B40F00781EFF31183002B40F00281D4F88420A968DC
:209CE000D4F884309A42F8D1D4F8403F9942F4D8D4F83CEF00FB0EF35B1AB3FBFEF300FB4B
:209D000002327B68C3F30803002B40F0A780EFF31183002B40F0A280D4F88430D5F808A001
:209D2000D4F884108B42F7D1D4F8401F8A45F3D8D4F83CEF00FB0EF1A1EB0A01B1FBFEF146
:209D400000FB03139B1AB3F57A7FDAD3013EB9D1D4F8100F41F09EFCD4F80C0F41F09AFCC2
:209D6000B4F8183F002B40F0DA8094F81A1FD4F81C0F81F0010141F0A9FC4FF0320C4FF466
:209D80007A7001267B68C3F30803002B40F08780EFF31183002B40F08280D4F88420A96858
:209DA000D4F884309A42F8D1D4F8403F9942F4D8D4F83C9F00FB09F35B1AB3FBF9F300FBE4
:209DC00002327B68C3F308033BBBEFF3118323BBD4F88430D5F808A0D4F884108B42F7D177
:209DE000D4F8401F8A45F3D8D4F83C9F00FB09F1A1EB0A01B1FBF9F100FB03139B1AB3F567
:209E00007A7FDED3BCF1010CBCD10BF1FF3616F0FF0B7FF43FAFBDE8F88FEFF3118988F38C
:209E20001288D5F808A02B68DB0344BFC4F8386FD5F808A0D4F88430D4F8381F5FFA89F949
:209E400089F31188D4F83C9F0B4400FB09F1A1EB0A01B1FBF9F100FB0313CFE7EFF3118E8D
:209E600088F31288D5F808A02B68D90344BFC4F838CFD5F808A0D4F88430D4F8381F5FFAB2
:209E80008EFE8EF31188D4F83CEF0B4400FB0EF1A1EB0A01B1FBFEF100FB031352E7EFF37E
:209EA000118188F31288D5F808902B68DA0344BFC4F8386FD5F80890D4F88430D4F8382FA8
:209EC000C9B281F31188D4F83C1F1A4400FB01F3A3EB0903B3FBF1F300FB023271E7EFF3F1
:209EE000118188F31288D5F808E02B68DB0344BFC4F838CFD5F808E0D4F88430D4F8382F67
:209F0000C9B281F31188D4F83C1F1A4400FB01F3A3EB0E03B3FBF1F300FB0232F1E6D4F842
:209F2000343F002B3FF429AFD4F8203F1E6084F8316F22E7D4F8343F002B3FF4BEAE3DF074
:209F4000B1FDBAE6A82D002000ED00E010E000E000F01F0240090123032803FA02F304D0B2
:209F600004280CD0022805D07047074A116C0B4313647047044A516C0B4353647047024AC6
:209F8000116B0B4313637047003802400E4B30B4DB68427801780D4CDB43C3F30223C3F197
:209FA0000403DBB202FA03F360181B0101F01F050122490903F0F003AA4080F8003344F846
:209FC000212030BC704700BF00ED00E000E100E0002879D02DE9F0418388B3FA83F3202B1F
:209FE000174684B00446C3F11F0256D0374DDFF8E8804FF0004008EB020605EB820205F6DF
:020000040800F2
:20A00000847C30FA03F396F8A060C2F844CF05D02F4A106820EA03001060536120463CF03C
:20A0200015FFA2882168B2FA82F2C2F11F0303F0FC0000F1804000F59C3003F003039C006E
:20A040004FF00F0C01F13F4381680CFA04FC21EA0C01816003F57E0308EB8707D0F808C0C0
:20A06000D7F8B0108DF80D10C3F38723A34043EA0C034FF00041354421FA02F28360002124
:20A08000012302A88DF80E3002928DF80C10FDF7B7FF95F8883FF02B02D804B0BDE8F0813D
:20A0A0000C4B9B5D8DF80430F02103224FF4807301A885F8881F8DF80520ADF80630FFF7E4
:20A0C00065FF04B0BDE8F081704700BFA82D0020003C0140D4FE06088881060800286BD010
:20A0E000F0B58388B3FA83F3202B85B00446C3F11F024CD0314D32484FF00041104405EB16
:20A10000820205F5796731FA03F390F8A060C2F8447F05D02B4A116821EA030111605361C4
:20A12000204600213CF092FEA3882268B3FA83F4C4F11F0303F0FC0101F1804101F59C31C6
:20A1400003F0030398000F2702F13F438A68874022EA070203F57E038A60C3F3872383406F
:20A1600088684FF000420343354422FA04F48B604FF44062012302A88DF80E300294ADF8FF
:20A180000C20FDF73DFF95F8883FF02B01D805B0F0BD0D4B9B5D8DF80430F02103224FF437
:20A1A000807301A885F8881F8DF80520ADF80630FFF7ECFE05B0F0BD704700BFA82D0020AD
:20A1C00088810608003C0140D4FE0608002869D0F0B58388B3FA83F3202B85B00446C3F159
:20A1E0001F024AD0304E314D16444FF0004005EB820230FA03F396F8A060C2F8441F05D03B
:20A200002B4A116821EA030111605361204600213CF01CFEA3882268B3FA83F4C4F11F039F
:20A2200003F0FC0101F1804101F59C3103F0030398000F2702F13F438A68874022EA0702AE
:20A2400003F57E038A60C3F38723834088684FF000420343354422FA04F48B604FF40062A4
:20A26000012302A88DF80E300294ADF80C20FDF7C7FE95F8883FF02B01D805B0F0BD0D4B2B
:20A280009B5D8DF80430F02103224FF4807301A885F8881F8DF80520ADF80630FFF776FEE5
:20A2A00005B0F0BD704700BF88810608A82D0020003C0140D4FE060810B4B8B10D4CD4F80B
:20A2C000943F102B05D15DF8044B052100203DF0A5B803EB4302224482F8991F01210B44EA
:20A2E00082F8980F82F89A1FC4F8943F5DF8044B704700BFA82D002080782021DCE700BFB1
:20A300002DE9F04FDFF8ACA32DED028B9AF8DC1F002297B0CAF8CC2FCAF8D02FCAF8D42FE2
:20A32000CAF8D82FCAF8C82F19B19AF8DD2F8AF8C82F9AF8DE2F1AB19AF8DF2F8AF8D72F28
:20A340009AF8E22F1AB19AF8E32F8AF8D22F9AF8E02F1AB19AF8E12F8AF8CD2F9AF8E43F27
:20A3600005935A1ED3B257B203937B1C00F0AA80C54AC64E52F83790029602EBC702002353
:20A380001279019308EE102A1D463446984626783946304644F0D4FF83463046BBF1000F1F
:20A3A0001ED040F0BFFEEA1D1321D2B220B14FF0000E827180F807E03CF048FD207844F056
:20A3C000E9FF4FF0070308F1010223714FF0010384F802806070CDF804B05FFA82F8E3700C
:20A3E0000135042D04F10504D1D118EE100A029ECDF81080FFF7ACFDA549A64A48680240D2
:20A4000042F440324A600FB9019B5BB9A24C4820FFF79EFD204602215BF0F8F9A26842F08A
:20A420000102A2609A489C4A4168BAF8E64F41F400014160516821F480515160916B21F487
:20A44000401141F480119163D16841F46001D160956B85F44011C1F3015101EB81011F2074
:20A4600000FA01FC25EA0C0C112505FA01F141EA0C019163D16841F0E061D160956BC5F3D7
:20A480000151C1F10401C9B201EB810188404FF0120C25EA00000CFA01F108439063E4B1CB
:20A4A000BAF8E81FCAF8F04FA1B1BAF8EA2FCAF8F41F62B1019B7948521A90FBF2F2CAF8E3
:20A4C000F82F6BB917B0BDEC028BBDE8F08F744A1288EFE7734A1188E7E7734A1488DFE79F
:20A4E000484604995BF092F9684B012003F114080723F278441CE4B252B375783279A5F1BA
:20A500000A0101EB410105EB450C092D03FA01FE03FA0CFB02FA01F140F2A080D9F80C204E
:20A5200022EA0E0E41EA0E01C9F80C10421E02EB82021F21062801FA02FC05FA02F273D866
:20A54000D9F8341021EA0C010A432046C9F834200536B045CDD1D9F80820039942F40072FB
:20A56000C9F80820D9F8082042F48072C9F80820D9F80820574442F00102C9F8082097F9A6
:20A58000EC2F02203DF08EFD044600289AD0466830463DF075FD454A431E242101FB0323D0
:20A5A00093F89C50002D8DD1059983F89D10062283F89C20002885D030463DF061FD55F0B1
:20A5C00083FB60680AF0D8F907A80AF097F9049EA26837480792012E8CBF4FF480630023AA
:20A5E0000D9309F14C034FF48072CDE90A56089309904FF4003360680C9507A94FF40067BA
:20A600004FF40056CDE91023CDE90E760AF088F96268136843F001031360D9F8083043F0D8
:20A620008043C9F808304DE7C11FA0F10D0201EB81014FF01F0E02EB82020C280EFA01FC26
:20A640000EFA02F005FA01F113D8D9F8302022EA0C0211432046C9F8301079E7D9F81010DD
:20A6600002FA0CF221EA0B0B42EA0B02C9F810205CE7D9F82C1005FA02F221EA00010A43F9
:20A680002046C9F82C2063E744820608703D002000230140E030FCFF0020014080380100D3
:20A6A0002E7AFF1F2C7AFF1F2A7AFF1F98010020A43D0020A82D002000285FD00368374A5C
:20A6C0002DE9F04103F13F4404F57E0402EB9422012492F8982002F01F055209032A04FA9B
:20A6E00005F456D0042A4FD0022A48D08588B5FA85F0C0F11F00C0F3CC0603EB860600F0BA
:20A70000070082000F24306A944020EA04003062306A01FA02F20243002132624FF0010E9E
:20A720000A464FF0030C02270EFA02F838EA050002F101021CD118680CFA01F420EA0400BD
:20A740001860186807FA01F606431E609E6826EA04069E6098689860586820EA08005860A2
:20A7600058685860D86820EA0400D860D868D860102A01F10201D7D1BDE8F0817047084A6D
:20A78000556C2C435464B1E7054A156B2C431463ACE7034A156C2C431464A7E78881060897
:20A7A0000038024070B5464E16F8F44C04EB440306EBC303650013F8F03C032B6ED8DFE854
:20A7C00003F059291E02254406EBC50555F8EC0C002870D116F8903C9C425FD0013404F002
:20A7E0000302934206F8F42C58D002EB420406EBC404022344F8EC0C04F8F03C70BD2B195B
:20A8000006EBC30353F8EC2C72B1013A43F8EC2C002070BD2B1906EBC30353F8EC2C002A98
:20A82000F3D1022203F8F02C254406EBC50515F8E43C013BDBB205F8E43C8BBB214B16F822
:20A84000906CD3F8C01255F8E80C621C02F003024B1E0324B242034405F8F04CB3FBF1F016
:20A8600045F8EC0C1AD0994218D8013845F8EC0C012070BD44F05AFC80B1124B2C44D3F8DF
:20A88000C02206EBC404012102F51C5304F8F01C0F33B3FBF2F344F8EC3C70BD012070BDD9
:20A8A000084BD3F8C022012002F2E733B3FBF2F345F8EC3C70BD013845F8EC0C002070BD89
:20A8C000A03E0020980100202DE9F84F3249DFF8D4B091F8AD1E01240229074619461046E8
:20A8E000CBF820414FF000022C4C1D4618BF7F02FDF7B8FB2A4B63626B02A362E36A40F2EE
:20A90000FF5943F093034FF400704FF48A62E3620121C4F83890A0601020E26054F040F95A
:20A92000012D40F251434E46C4F83890CA4640F252488EBF4FF0120998464FF011090A2522
:20A94000C4F838A00121A7604846C4F80C8054F027F903464FF0000C40F277420121372008
:20A96000A6632BB900231846CBF81C31BDE8F88FA663C4F808C0E26054F012F9013DA663C8
:20A980000028EFD015F0FF05DAD10346CBF82051CBF81C31BDE8F88FA82D0020002C014001
:20A9A00000E1F505B01C00202DE9F843DFF8748098F82450042D0446894617461E4608D0CD
:20A9C000082D02D00020BDE8F883FEF7E5FA0228F8D101234A4620460021FFF775FF68B1AB
:20A9E000FEF78EFED8F80C40002CEBD00022D8F81030D8F804101046A047E3E7084BC8F8A3
:20AA00000090D3F88420C8F804400523C8E90376C8F8142088F824300120BDE8F88300BF19
:20AA2000A82D0020B01C00202DE9F84F3149DFF8CC9091F8AD1E1E4602292F4B07464FF042
:20AA4000010418BF4702012E40F25948C3F8244198BF4FF48B683B469346474640F2FF55B5
:20AA6000B0468CBF4FF0190A4FF0180A0A241E4640F2FF53C9F838300121C9F808605046B2
:20AA8000C9F80C7054F08CF803464FF0000C40F2774201213720C9F83850ABB958464146E7
:20AAA0000122FDF7DFFA4646144A154B536276029662D36A43F09103D3620F4B0021084635
:20AAC000C3F81C11BDE8F88FC9F83850C9F808C0C9F80C2054F064F8013CC9F83850002855
:20AAE000DCD014F0FF04C3D1034BC3F82441BDE8F88F00BFA82D0020B01C0020002C014068
:20AB000000E1F5052DE9F047364C82B005460E461746984694F8240004280CD0082806D1C0
:20AB2000E369AB4207D0FEF737FA0228F2D0012002B0BDE8F087DFF8B4A02660DAF8A09E43
:20AB40006560C9F34F210F294FEA592222D8236A0193FBB194F8F200E0B1B9F5005F13D052
:20AB6000214831464FF4007248445DF05BFA09F50072C2F34F211029CAF8A02E4FEA522207
:20AB800002D0019B012B20D192B2013A164EAD1A0B4600E0012332462846062601250021D2
:20ABA000E760C4F81080257284F82460FFF73CFF0028BDD0FEF7A4FDE66886B12846236970
:20ABC00061680022B0470320B2E7E269013B01320421C4E9072384F824100220A8E703209D
:20ABE000A6E700BFB01C002094700020A82D00202DE9F04FB44CB54E95B0002305464FF4B6
:20AC0000F0728B46A4F18C00202104F88F3C04F88E3C01955DF067FA202104F5AA704FF437
:20AC2000F0725DF060FADFF8BCC2A94932274FF0100E4FF47A704FF00108DCF80430C3F3DB
:20AC40000803002B40F0BA80EFF31183002B40F0B580D6F884208D68D6F884309A42F8D1C0
:20AC6000D6F8403F9D42F4D8D6F83C9F00FB09F35B1BB3FBF9F300FB0232DCF80430C3F33F
:20AC80000803002B79D1EFF31183002B75D1D6F88430D1F808A0D6F88450AB42F7D1D6F835
:20ACA000405FAA45F3D8D6F83C9F00FB09F5A5EB0A05B5FBF9F500FB03539B1AB3F57A7FB5
:20ACC000DBD3013FB9D194F83523002A50D094F83633013B022B4BD803EB830004EBC0012C
:20ACE0007C4D91F8D07305EBC0004FF0010C022FC4F8380384F8C0C300F0C182DBB204EBED
:20AD00000313D3F84834C1F8D4338BB3022381F8D033A5F188034C3DC1E9FA354FF4807081
:20AD2000A1F8DC031509013D042D02F00F0200F28982694F07EB4503B3F8840040FA02F3BE
:20AD4000DB0740F17F82012303FA02F2013A10403D445AF03BFF95F89020604B104403EB10
:20AD6000C000C4F840038379002B47D0412B45D06FF0010015B0BDE8F08FEFF311898EF30F
:20AD80001288D1F808A00B68DD0344BFC6F8388FD1F808A0D6F88430D6F8385F5FFA89F99A
:20ADA00089F31188D6F83C9F2B4400FB09F5A5EB0A05B5FBF9F500FB03537EE7EFF3118502
:20ADC0008EF31288D1F808900B68DB0344BFC6F8388FD1F80890D6F88430D6F8382FEDB267
:20ADE00085F31188D6F83C5F1A4400FB05F3A3EB0903B3FBF5F300FB02323EE72323C3807B
:20AE000009213CF023F8D4F8403313B11A689B881383D6F83025324BB3EB920F80F035827D
:20AE2000B3EBD20F80F03382B3EB121F80F03382B3EB521F80F03382B3EB921F80F03382D2
:20AE4000B3EBD21F80F03382B3EB122F80F031824FF4807200230DF10D01FF20A4F83C23BE
:20AE60000122CDE90413CDE90833CDE90A33D4F838138DF80D000D9306928DF81C208DF8D7
:20AE80003020EFF31180102383F31288D4F838331B6A002B00F0DA81069B04AD2A461BB1EC
:20AEA000D3691432002BFBD10B6A002B00F01782996839B99A421AD01968A9B15B68996898
:20AEC0000029F7D01433F3E7A03E0020A82D002010E000E07042002088810608583000200D
:20AEE000404B4C0000ED00E0B84AC3E90025C0B280F31188D4F838130B6A002BFCD18C222B
:20AF00000120CDE908330DF10E080DF10F0A05938DF81C300D93109312938DF80E200023CD
:20AF20000022CDE90E23CDF8108006900B908DF830008DF84400CDF828A0EFF311801023D1
:20AF400083F31288D4F838331B6A002B00F08781069B2A461BB1D3691432002BFBD10B6A37
:20AF6000002B00F0BC81996839B993420AD0196829B15B6899680029F7D01433F3E7934ACA
:20AF8000C3E90025C0B280F31188D4F83823136A002BFCD19DF80F301B2B40F09081D4F89F
:20AFA0004033012204F88F2C0BB12322DA80DFF81C92402248460A2143F0F4FE8A21002356
:20AFC00001228DF80E1000200021CDE90E01CDE90833D4F83813CDF81080CDF828A0059323
:20AFE0008DF81C300D931093129306920B928DF830208DF84420EFF31180102383F31288EF
:20B00000D4F838331B6A002B00F03181069B2A461BB1D3691432002BFBD10B6A002B00F0C1
:20B020005B81996839B9934209D0196829B15B6899680029F7D01433F3E7C3E90095C0B2B0
:20B0400080F31188D4F83823136A002BFCD19DF80F2094F83413C2F3801284F87824002929
:20B0600000F0D480022900F0B980D6F830355849B1EB930F80F01F81B1EBD30F80F009819E
:20B08000B1EB131F80F00981B1EB531F80F00981B1EB931F80F00981B1EBD31F80F00D810C
:20B0A000B1EB132F34BF4FF48076802694F87C14A4F87A64182914D1464F474800215B087C
:20B0C000B3FBF6F3A7FB03730F465B0B66F30F076BF30F0163F31F4762F31F41C4F8801468
:20B0E00047603A48A4F83C630222002143F05AFEC8203CF0DBFAD4F838034FF0800B00263C
:20B10000002700230122CDE90E67CDE908338DF80EB0CDF81080CDF828A005938DF81C3018
:20B120000D931093129306920B928DF830208DF84420EFF31182102383F31288D4F8383345
:20B140001B6A002B38D0069B002B3DD02B46D96914330029FBD1006A002800F0BA808168CA
:20B1600039B9834209D0016829B1406881680029F7D01430F3E7C0E90095D2B282F311888D
:20B18000D4F83803036A002BFCD19DF80F3013F00203B6D1019841788278007884F8880414
:20B1A000C1F12001C2F11002184684F8891484F88A2415B0BDE8F08F0562D2B282F3118874
:20B1C000024856F07FF9DBE72B46C4E7D8410020809698005917B7D120430020D6F83035F4
:20B1E0004048B0EB930F72D2B0EBD30F51D2B0EB131F52D2B0EB531F53D2B0EB931F54D210
:20B20000B0EBD31F34BF802640264FE7D6F830353549B1EB930F4ED2B1EBD30F39D2B1EB38
:20B22000131F3AD2B1EB531F3BD2B1EB931F3CD2B1EBD31F41D2B1EB132F34BF4FF48076AE
:20B24000802633E70020C4F84003D9E504ADC0B20D6280F31188254856F034F94AE60D6234
:20B26000C0B280F31188214856F02CF98DE60D62C0B280F31188484656F024F9E2E691F8DA
:20B28000DD33634481F8DD334CE50222E2E50422E0E504260AE70822DCE5082606E7102214
:20B2A000D8E5102602E72022D4E52026FEE64022D0E58022CEE50226F8E64026F6E6D4F80D
:20B2C000400320213BF0C2FD4FF0FF3052E50E46ECE6C0F80090FFDEC3F80090FFDE034A9B
:20B2E0001A60FFDE002D3101404B4C00D841002038B50C4C0546A11CD5224FF0CFFD2B68A6
:20B30000A342C5E90043A3EB04000AD004F14002611C2960237802F8013BD5E90041A142FB
:20B32000F6D138BD2C430020F0B40D6800240CE0BCF1050F18D8A0F137030A2B14D104EB14
:20B34000840415F8010B03EB4404A0F13003DEB2092EA0F16107A0F1410CF0D9052FE7D8F8
:20B36000A0F157030A2BEAD00D601460F0BC704710B5204B84B0C82403F2CC4103F28D4299
:20B380002128CDE9022183F88C4418D00CD802281ED0082825D102A801900BF0A7FA0198C6
:20B3A000FFF7A6FF04B010BD29281AD102A801900BF056F90198FFF79BFF04B010BD02A85C
:20B3C00001900BF097F90198FFF792FF04B010BD02A801900BF0D8FA0198FFF789FF04B0DD
:20B3E00010BD02A801900BF0F7F90198FFF780FF04B010BDA03E0020014488420ED010B41C
:20B400000346074C074813F8012B04FB00F0994280EA0200F7D15DF8044B704701487047B1
:20B4200093010001C59D1C81094B93F86231042B08D9053B032B08D801231A4600B1037000
:20B440001046704700230122F8E700231A46F5E7A82D00209FED727A07EE901A20EE070A30
:20B46000F8EE677A27EE800AFDEEC07A17EE903A2033402B00F2C480DFED6A7AB4EEE70A3B
:20B48000F1EE10FAF0EE407A0CDD9FED676ADFED676AB0EE677AB4EEE67AF1EE10FA77EE79
:20B4A000C67AF6DC9FED627AF4EEC77AF1EE10FA0CD59FED5D6ADFED5F6AB0EE677AB4EE1C
:20B4C000E67AF1EE10FA77EE867AF6D49FED5A7AF4EEC77AF1EE10FA00F38A809FED577A2E
:20B4E000F4EEC77AF1EE10FA44BF9FED517A77EE677A27EEA76ADFED525A9FED527ADFEDDE
:20B50000526AA6EE257A67EE865AE6EE076AB6EE007AE5EEA67A27EE877ADFED476A70EEC0
:20B52000267ABDEEE76A16EE103A2033402B64D8B4EEE60AF1EE10FA0CDDDFED3B5A9FEDD6
:20B540003B6AF0EE676AF4EEC66AF1EE10FA77EEE57AF6DCDFED366AF4EEE67AF1EE10FA6F
:20B560000CD5DFED315A9FED336AF0EE676AF4EEC66AF1EE10FA77EEA57AF6D4DFED2E6A0E
:20B58000F4EEE67AF1EE10FA3DDDDFED266A76EEE77A67EEA75A9FED2A5A9FED2A6ADFEDF3
:20B5A0002A6AA5EE856A27EEA55AE5EE866AB8EE006AE5EE267A67EE867AC7EE206AB7EEE2
:20B5C000006A76EE865A76EE666A86EE257A80ED091A67EE277A66EE876AC0ED017AC0EDD6
:20B5E000037A80ED007A80ED027AC0ED046A70479FED0C7A77EE677A7BE7DFED147ADCE755
:20B600009FED127A89E7DFED0D6AF4EEE67AF1EE10FA44BFDFED066A76EEE77AB9E700BFD1
:20B6200027D4D236DB0F4940DB0FC940E4CB1641DB0F49C0E4CB16C1DB0FC93FDB0FC9BFBE
:20B6400092E741B99730083C15A82ABE000000002DE9F041E14ED6F8103596F8884A07EEE9
:20B66000903AF8EE670A06F684232DED028BC3ED000A002C6FD1DFF8C4C396F8987AC6F87D
:20B68000944A9CF80040002F39D0B6F88E3A9FEDD46A9FEDD47A07EE903AF8EE677A20EE12
:20B6A000877AC6EE276AD04B0022012F1A6076EE876AC7EE267AC3ED017A20D0022F9A606D
:20B6C000C3ED037A1BD0032F1A61C3ED057A16D0042F9A61C3ED077A11D0052F1A62C3EDF0
:20B6E000097A0CD0062F9A62C3ED0B7A07D0072F1A63C3ED0D7A02D09A63C3ED0F7ABB4BB6
:20B700009FEDBB6A93F882319FEDBA7A9FEDBA0ABA4A07EE903AF8EEE77A9CF8583BC6EE45
:20B72000276A1C4414FB07F4E4B207EE904A60EE870AF8EEE77AC2ED006AA7EEA00A5BF0E0
:20B740004BFABDEC028BFCEEC07A17EE903A86F8E83BBDE8F08196F8893A9FEDA96AB6F826
:20B760008A2A9FEDA82ADFEDA86ADFF8D0C296F8987AC6F894CA07EE903AFCEEE05AB6F823
:20B780008C3A8CF8004007EE103A15EE903AF8EE655AF8EE677A86EE255ACCF81430012388
:20B7A00086F8903A06EE102AB8EEC77A27EE822AB8EE466A67EE266A22EE252A8CED025AFC
:20B7C000CCED017A8CED036ACCED046A002F96D0DFED8E7A9FED8E4ADFED8E5AC7EE871A51
:20B7E000C7EB0715A7EB07180CEBC5054FEAC8084FF0000EB1EE611A9FED876A08EB050024
:20B800009FED863ADFED863ADFED866A0346002207EE902AB8EEE77A27EE027AFDEEC77AB6
:20B8200017EE901A2031402900F2D080B4EEC47AF1EE10FAF0EE477A0CDDDFED7B4A9FEDEF
:20B840007B5AF0EE672AF4EEC52AF1EE10FA77EEE47AF6DCF4EEE57AF1EE10FA0CD5DFED7E
:20B86000724A9FED735AF0EE672AF4EEC52AF1EE10FA77EEA47AF6D4F4EEC67AF1EE10FA32
:20B8800040F39A8074EE677A27EEA75AB0EE630AA5EE030ADFED674AE5EE004A65EE272A19
:20B8A000B7EE005AE2EEA47AB0EE458AF0EE454AA1EEA78AE1EE274AC5EE088A84EE880A78
:20B8C00077EE067ABDEEE75A15EE101A203140296FD8B4EEC67AF1EE10FA0CDD9FED525A7D
:20B8E0009FED527AF0EE674AF4EEC74AF1EE10FA77EEC57AF6DCF4EEE57AF1EE10FA0CD504
:20B900009FED495A9FED4A7AF0EE674AF4EEC74AF1EE10FA77EE857AF6D4F4EEC67AF1EE0E
:20B9200010FA3CDD74EE677A27EEA75AF0EE632AE5EE032A9FED3F7AA5EE227A65EE274AE8
:20B94000B8EE005AE4EE877A67EE857A87EE887A0132A24203F1280343ED048A03ED037AE8
:20B9600003ED017A43ED028A83ED000AC3ED056AC3ED026AC3ED016AC3ED046AC3ED036A95
:20B98000FFF646AF783085427FF43AAF0EF5707EBEF5346F05F570757FF42EAF75E69FED95
:20B9A000267AF4EEC77AF1EE10FA48BF75EEE77ABAE7F0EE667AC9E79FED1F5AF4EEC57ADB
:20B9C000F1EE10FA48BF75EEE77A5DE7B7EE000AF0EE408AB0EE408A72E700BFA03E00209A
:20B9E00083F9223EBD3786358C4A0020A82D0020555555406E12833A48E1FA3E844A002006
:20BA00000060EA4827D4D2360AD7233C00004842DB0F4940DB0F49C0DB0FC93F92E741B9FC
:20BA20009730083C00000000DB0FC940E4CB1641E4CB16C115A82ABEDB0FC9BF94A0002011
:20BA40002DE9F04F07EE900A2DED068B9FEDF07AF049DFEDF16AB1F82C3C91F8325CC1F820
:20BA6000840CB8EE679A0AEE103A87EE095AB1F82E3CC1F8405C002283B0C1F8442C08EE99
:20BA8000103AB1F8303CDFEDE57AB8EE4AAA08EE903AB8EEC88A3AEE0A7AF8EEE88AB4EE24
:20BAA000C78AF1EE10FA68EEA77AB4EEE65A01F63443B8BFB0EE478AF1EE10FA83ED028ABA
:20BAC00083ED01AAC3ED007A00F1008307EE905AF8EEE77AB7EE007AC7EE279AD04BDFF800
:20BAE0007CA3184614309C4601909AF8002503F12C04F6EE005A65EE256AF7EE007A86EE44
:20BB0000887ADFEDC83ADFEDC84A9FEDC86AD3ED05AAB4EEE77AF1EE10FAB8BFB0EE677A68
:20BB2000BDEEC77AB0EE004A17EE106AB8EEC77AC1F8E06EC5EE076A87EE875A66EEA36AE9
:20BB4000ACEC015A8AEE267AC8EE267A37EE257A77EEA57AB4EEC47AF1EE10FAB8BFB0EE5E
:20BB6000447AF4EEE47AF1EE10FABDEEC77A88BFF0EE647A17EE107AFDEEE77A07F1FF3BE2
:20BB800017EE900ABBF1230FA8BF4FF0230BCCED006A012E00F1010CB8BF0126BCF1230F87
:20BBA0002BEAEB7BE04629EE066AA8BF4FF02308E345C8BFD846C1F8EC7E83ED046AA8EB2B
:20BBC0000B07C1F8F00E97FBF6F70137002A40F0E380DFED970ADFED975A9FEDA12A9FED1B
:20BBE000965ADFEDA32A9FEDA33ADFEDA33A9FED934ADFEDA21A0AF2045107EE902AB8EE13
:20BC0000E76A66EE207A37EEA57AFDEEC76A16EE903A2033402B00F21282F3EE026AB4EE84
:20BC2000E66AF1EE10FA0CDDDFED8F4ADFED8D6AB0EE471AB4EEE61AF1EE10FA37EE647AED
:20BC4000F6DCB4EEC57AF1EE10FA0CD5DFED864ADFED866AB0EE471AB4EEE61AF1EE10FA85
:20BC600037EE247AF6D4B4EEE57AF1EE10FA40F3FB81DFED736A36EEC77A67EE076AB0EE2C
:20BC8000431AA6EEA21AB0EE630AA1EE260A67EE264AFDEEE76AA4EE807A16EE903A20337F
:20BCA000402B27EE047A00F2D481DFED666AB4EEE66AF1EE10FA40F3FD819FED6B0A9FED8A
:20BCC000691AF0EE676AF0EE664AF4EEC14AF1EE10FA76EEC06AF6DC9FED591AF4EEC14A82
:20BCE000F1EE10FA13D59FED601ADFED604AB0EE660AB4EEE40AF1EE10FA76EE816AF6D457
:20BD0000DFED506AB4EEE66AF1EE10FA0CDD9FED566ADFED546AF0EE674AF4EEE64AF1EE83
:20BD200010FA77EEC67AF6DCF4EEC57AF1EE10FA0CD59FED4D6ADFED4D6AF0EE674AF4EE60
:20BD4000E64AF1EE10FA77EE867AF6D4F4EEE57AF1EE10FA40F38081DFED396A76EEE77A09
:20BD600067EEA76AF0EE434AE6EEA24AB0EE631AA4EEA61A27EEA66AE6EE017A67EE847AFE
:20BD80000132242A81ED007AC1ED017A01F108017FF433AFDFED2CAA4FF0000944E9059B0A
:20BDA00044E902764FF490720021204644F80C8C5CF099F94FF49072A01800215CF093F96A
:20BDC000224B04F51574A342E8D1019BDFED207AC3ED00AA012329EE279A8AF80035002D9A
:20BDE00000F02881DFED1B7A1B4E9FED152ADFED122AC7EEA81AA6F1140406F5117738EE3E
:20BE00004A8AB1EE611A69EE889ADFED0A5A3BE000247449A03E00200000FA440AD7233C13
:20BE2000844D0020398E633C00000C429C534937C3B8B23DDB0FC93FDB0F49C072F97F3F76
:20BE4000DB0F494000001042BC297E3FAC54002027D4D23600004842E84A0020984F002075
:20BE600000000000E4CB1641DB0FC940E4CB16C192E741B99730083C15A82ABEDB0FC9BFAE
:20BE8000000010C20000807F5FED0B6A234630460022B7EE005A07EE902AF8EEE77AB6EE76
:20BEA000007A77EE877AB0EE4A7AA7EEA97AF0EE477A29EE077AE0EC017AFDEEC77A17EED9
:20BEC000901A2031402900F2D780B4EEC27AF1EE10FAF0EE477A0CDD1FED1D4A5FED1F4A3E
:20BEE000B0EE676AB4EEE46AF1EE10FA77EEC47AF6DCF4EEE27AF1EE10FA0CD51FED264A01
:20BF00005FED264AB0EE676AB4EEE46AF1EE10FA77EE847AF6D4F4EEE57AF1EE10FA40F393
:20BF2000B58072EE677A67EEA74A5FED2F3A1FED2F4A1FED2F6AA4EEA34A67EEA43AA4EE22
:20BF4000246AF0EE454AE3EE867AB0EE456AE1EE274AA1EEA76A84EE864AC5EE064A77EE3E
:20BF6000257AFDEEE73A13EE901A2031402900F28A80B4EEE57AF1EE10FA0CDD1FED463A56
:20BF80005FED483AB0EE677AB4EEE37AF1EE10FA77EEC37AF6DCF4EEE27AF1EE10FA0CD5F0
:20BFA0001FED4F3A5FED4F3AB0EE677AB4EEE37AF1EE10FA77EE837AF6D4F4EEE57AF1EE64
:20BFC00010FA6DDD72EE677A27EEA73A5FED580A5FED583A1FED587AE3EE203A63EE270ABF
:20BFE000A3EE237AF8EE003AE0EE877A67EEA37A87EE867A0132AA4203F12803C3ED0B4AFA
:020000040800F2
:20C0000083ED0C7A83ED0E7AC3ED0D4A83ED0F4A83ED145AC3ED116AC3ED106AC3ED136A02
:20C02000C3ED126A7FF437AFC834A74206F114067FF4EBAE03B0BDEC068BBDE8F08FFDEE7D
:20C04000E76AB0EE427A16EE903A2033402B7FF62CAEF0EE427A93E6F4EEE17AF1EE10FA21
:20C0600048BF75EE677A7BE6B4EEE17AF1EE10FA48BF35EE477A00E6B7EE004AF0EE444A02
:20C08000B0EE446A6BE7F0EE667AB1E71FED856AF4EEC67AF1EE10FA48BF72EEE77A42E7B5
:20C0A0001FED8A7AF4EEC77AF1EE10FA48BF72EEE77A89E75FED8E6AB4EEE66AF1EE10FA0D
:20C0C00048BFF0EE676A3FF50EAE2DE65FED939AC1F8402C154601E5084800230246117884
:20C0E000022902F1060204D00133062BF7D10020704703EB430300EB43007047DC1D002010
:20C1000010B582B00A788DF80720040A18238DF804308DF806008DF8054052F065FB01AA56
:20C1200003481146042342F093FE02B010BD00BFBC55002010B582B0040A192200238DF81C
:20C1400001408DF800200C468DF803308DF8020052F04AFB6A4605481146052342F078FEBD
:20C160009DF80430237002B010BD00BFBC55002010B58CB000234CF20502044601A9CDE9E1
:20C180000633CDE90833ADF800208DF8023003220B930123CDE903128DF814308DF82830A1
:20C1A000CDF808D042F09AFE204602A941F0C4FD204642F093FE9DF806000CB010BD00BF09
:20C1C0002DE9F043774D784F83B005F59670242200215BF088FF97F8BD460023C5F850312C
:20C1E000002C3CD1714ED6F8F83063B39B6A53B36F489847836833B303886E4F013B9BB2F8
:20C20000BC46384600210678032E00F106001ED001310629F7D100223978022907F10607BD
:20C2200000F09F800132062AF6D1D5F85011052909D0481C02FB01C2C5F85001022000211B
:20C24000938010705180204603B0BDE8F083062303FB0151B1F82E31013B9BB2DBE797F8EE
:20C26000BC0607F2C463C7F8C03610B94F4E0024B9E73EF057FFC7F8CC0618B183790BB167
:20C28000412BF3D121464C4841F0CCFE04460028ECD0D7F8C036464A9868C3F8942008B1CD
:20C2A0002023C38009213AF0D1FDD7F8C0363F4E98683FF005FA4148D7F8C08642F09EFCEC
:20C2C0004FF00109A8F804003220C6F8188186F81C913BF027FB0423D7F8C0064FF0000C49
:20C2E0000DEB03029F21CDF804C042F007FD9DF805809DF804309DF806104FEA082848EA99
:20C30000034848EA0108414606F1F8004FF0E2FF00287FF468AF4046FCF702FB0346002868
:20C320007FF461AF9DF806009DF805209DF80710000240EA0240224A0843904215D0C6E9EE
:20C340004033A6F8FC30A6F80831FCF7E9FA804600287FF448AF97F8BC0641F0CBFC4446C8
:20C3600041E7062101FB02C268E7164AC6F8FC204FF400334FF00062C6F800314023A6F81E
:20C380000831C6F8042186F80A91FBF7D1FE06F1F80086F811914FF0E9FE0B4BC6F8F83036
:20C3A00021E700BFB01C0020984F0020A82D0020A02E0020DC1D00205C560020404B4C001E
:20C3C00021AAEF0000040008888106082DE9F041C54BC64EC64DC74C0822C3F88820336BC4
:20C3E00082B043F00103336307464FF4C052284640F2023388466946CDE9002308F05EFC1F
:20C400006B6AC4F8408D23F470436B626B6AC4F8487D43F420436B626B6AB749C4F8441D78
:20C4200023F470236B626B6AB448C4F85C0743F420236B62736CB249C4F8601743F4804347
:20C440007364736BAF48B049C4F86C0743F0800302257363AD4F84F86457AD4EAD4DC4F871
:20C46000B0174FF0A043C4F86837AB4AC4F8787703F53463A1F5D071C4F8B457C4F87C670C
:20C48000C4F8B837C4F880170123DFF8BCC2C4F874C707F51077A5F5E465A6F5A066A1F591
:20C4A0008C61C4F8BC77C4F87057C4F8286884F8673705F5A075536106F5B076C4F8EC1714
:20C4C00084F86E381946954B954AC4F8F457A7F5BC67A035C4F80068924EC4F8FC77C4F892
:20C4E000043807F5D45703F56953C4F808584FF050250020DFF854E2C4F82C28ACF5687C93
:20C5000002F5A042C4F83078C4F8346807F5A04706F5A046C4F83838C4F83C58A3F5485313
:20C5200004F25C75C4F84028C4F84868C4F86838C4F8F0E7C4F8F8C70246C4F844782B4609
:20C5400084F87008402683F81C21A3F822210132042AC3E9496083F81D1183F81F01C3F836
:20C56000300103F12803EED1002211462B46402083F87423A3F87A230132042AC3E9DF012B
:20C5800083F8751383F87713C3F8881303F12803EED14FF0A04364489A6822F001029A6080
:20C5A000DA6842F04002DA6007F046FC94F865370022212161F317420BB142F4801294F809
:20C5C0005F17D4F8683701299A6300F0E480DA68D4F86868D4F86C07C2F3076121F0600153
:20C5E00041F0400161F31F620021DA603160026861F3CC22026094F86727012A00F0B8808D
:20C6000010214A4807F06AFF484807F04DFFD4F86C0794F85D3700224FF0FF31026142612E
:20C620008161C26153B305F11407414E114607EB83074FEA830C4FF0FF0E56F8042F13686C
:20C64000002BACBF00234FF09043B74213601161C2F808E0F1D105F1500336496344002737
:20C66000FF2651F8042F1568002DACBF00254FF090459942156017619660F2D1036994F852
:20C680005F1743F480730129036161D0D4F8682729480023936100294FF0FF336FF080419E
:20C6A00051615360516114BF00231023906143F470139069D4F8441D43F4605343F0080341
:20C6C000034393619368096843F00103936088471A4B1B4ADA6068461A4B0093FDF756FCCB
:20C6E00002B0BDE8F08100BF00E100E00038024000000240984F00205C04002008040100A2
:20C700004000400100080050000B00502009005040090050200B0050003C0140C0050050C6
:20C72000001000500030005000570020F456002008570020445700200008008000ED00E0A9
:20C740000005FA05430200010009005020050050D4F86827144B03636FF08041134D0023FE
:20C760004FF0FF30936151615060516195619EE701680F4A0F4E41F00301016080215962B7
:20C780009E62C3F80421E022C3F80821C0F24002C3F80C2134E79A6822F03E0141F02A012D
:20C7A00061F307029A6012E70301810000080080A00040008000200010B5194C94F8510D88
:20C7C000B8B9184B83F85100586594F8543D012B05D0022B20D0D4F8583D1BB910BD124B62
:20C7E000C4F8583D11495B68BDE81040A1F10C0018473EF097FC94F8532D0A49003A18BFA8
:20C80000012281F8512048650028DED01F22C28020213AF01BFBD8E7054BC4F8583DE1E75C
:20C82000984F0020B01C00209C040020F45C00207804002099B10A6B824216D9154BD3F89C
:20C840009C2D914221D34C3991421ED30B6B9842F9D38B6B9842F6D80B46184670470D4B87
:20C86000D3F89C1D0A6B904212D30B680BB9F4E70A6B90420B4602D38A6B9042EDD951F8B3
:20C880004C3F002BF4D1184670470023184670470A46D8E7984F00202DE9F047CC0143D18C
:20C8A0000346224A43F8082B4FF0FF324260022418467E26DFF87880D8F8A09D2644013E96
:20C8C000051D49466FF070474FF0010A08E0A3421CD0631C45F8043C321B1C460435CAB12F
:20C8E0000B6BA34202D88B6BA34204D22046FFF7A1FF014690B10A794B6B002AE7D1A342CE
:20C9000004D0E6D245F8042C631CE5E745F8047C631CE1E7C8F8A01DBDE8F08745F804AC49
:20C92000321B631C4946D8E78026C3E7F8FFFF0F984F002070B4447941BB03684FF40052A4
:20C940004FF40076202502213CBB1A8C22F001021204120C1A841A8B188C22F0F30280B2B0
:20C96000120420F00A00120C014342F0010241F001011A8319841A8B22F00C021204120C8A
:20C980001A831A8B92B270BC1A83704700220368164615461146002CD7D0042C21D0082CCE
:20C9A00038D0198C21F480510904090C19849C8B1D8C45F6FF7040F6FF4128402140024327
:20C9C00042F4805241F4807199831A849A8B22F440621204120C9A839A8B92B270BC9A838F
:20C9E00070471A8C22F010021204120C1A84188B198C89B240F6FF4221F0A00102400D43A6
:20CA000042F4807245F010051A831D841A8B22F44062B3E71A8C22F480721204120C1A84EF
:20CA2000998B1A8C21F0F30192B2090422F42062090C324342F4807241F0010199831A849F
:20CA40009A8B22F00C02C4E738B50E4D0446006808F038F8D5F83025204652084FF6FF712D
:20CA600039F0ACFD20460021FFF764FF064BC5F89C3D05F69C5120460022BDE8384039F067
:20CA800071BC00BFA82D002035140208036870B55E6A26B133460522BDE870401847044695
:20CAA0000D464E1D00E023689B68204698470028F9D0236815F8011B1B6820469847B542A1
:20CAC000F1D170BD0A44914217D010B40139541E11F8013F08225840430010F0800F08BF4B
:20CAE000400083F0D50314BFD8B2C0B2013AF3D1A142EDD15DF8044B704770472DE9F047DD
:20CB0000154B054603F6B454002093F9AD8D84B06F1804F5287A06464FF0B6092368ABB1FC
:20CB200093F83830142B11D018F1020F01D043450CD1002269462046CDE90266CDE9005730
:20CB4000ADF808908DF80D6032F044FFE034A245E4D104B0BDE8F087984F00202DE9F0476D
:20CB60009AB0DDE9226ADDF8909004460D461746984602E020683BF0F5FA20683BF0FAFA21
:20CB80000028F7D10146642201A85BF0ACFA264B8DF80450CDF85CA00293002D3FD0AB1E99
:20CBA000012B3ED9042D14BF002203221F4B0396D3F884308DF805201E440123CDE90594E6
:20CBC00004968DF85B3037B14246394607A85BF029FA8DF85A80164E16F8629C0023189302
:20CBE000B9F1000F18D116F8630C642202FB006001A960385BF016FA012306F8639C06F877
:20CC0000623C236843B143463A46294620461AB0BDE8F04712F040BB1AB0BDE8F087052269
:20CC2000C4E70222C2E700BFEC5F0020A82D0020906000200A480B4B016A10B40A4C0361BC
:20CC40008A1E2231C38F1B01A4FB03C3DB08A3F5B06322F8023F9142F4D15DF8044B70472A
:20CC6000906000200D7A0208CDCCCCCC70B5084C251D2E4614F8010B33F078F828B10378B4
:20CC800005F8013BB442F5D170BDFF23F8E700BFF46000202DE9F0471D4F012607F1080559
:20CCA000B2464FF03C094FF0000817F8010B3EF039FA044690B180F80690C671FB7803F0FF
:20CCC0007F02012A18D013F0800F20460DD185F804803EF0EFFC85F805802C600136052ED8
:20CCE00005F10805E1D1BDE8F08785F804A03EF0E7FC85F805A0F0E71B0605D401212046B6
:20CD00003AF0A4F8FB78DEE73EF0DAFCF6E700BFFC6000202DE9F04FDFF8FC91DFF8FCA1CC
:20CD200083B009F10C06012419F8018BB8F1000F00F0C6804FEA1815013D042D08F00F0226
:20CD400000F2C1800AEB4503B3F8840040FA02F717F0010700F0D28001239340013B184025
:20CD6000554458F033FF95F89030664F184407EBC00704237761FC71BB71002302E0152BAC
:20CD800000F09E8003EB43025F49895C41454FEA430B03F10103F2D15C4B1A4492F8451217
:20CDA000002900F0AD80404639F0FEFD0546284639F01AFE0378002B40F08280534B5B4474
:20CDC000042283F8854283F88422002D78D0002F5DD03B68287A03F13F4202F57E020AEBD3
:20CDE00092224FF0010C92F8982002F01F015209032A0CFA01F171D0042A67D0022A75D048
:20CE0000B7F804E0BEFA8EF2C2F11F02C2F3CC0103EB810102F007020F6A92004FF00F0C21
:20CE20000CFA02FC27EA0C070F620F6A90403843002208624FF0010B11460BFA01FC3CEA3F
:20CE40000E0001F101011ED118680327974020EA07001860D3F800800220904040EA080068
:20CE60001860986820EA0700986098689860586820EA0C00586058685860D86820EA0700E2
:20CE8000D860D868D860102902F10202D5D1204B204AB3F89410B3F8963000910020013491
:20CEA0000190B2FBF3F330469BB22946E4B231F029FB0123092C737406F118067FF434AF96
:20CEC00003B0BDE8F08F0027776156E7DFF850C0DCF830200A43CCF8302091E7DFF840C084
:20CEE000DCF840201143CCF8401089E7DFF830C0DCF844201143CCF8441081E777613CE758
:20CF00000D4654E758300020EC2F0020A82D00209060002040420F0028610020888106084A
:20CF2000003802402DE9F041214E224F96F8673187F8083F06F5B27607F60C7500244FF060
:20CF4000050816F8010B20BB28600134032C05F10405F6D197F8081FD7F80C0FC94301F080
:20CF600001013EF0B3FB97F8081FD7F8100F81F00201C1F340013EF0A9FB97F8081FD7F86F
:20CF8000140F81F00401BDE8F041C1F380013EF09DBB3EF0C7F8013401212860E3B210B145
:20CFA00080F80680C371286839F050FFCEE700BF90600020A82D00202DE9F0412A4C2B4D89
:20CFC000B4F86C61A5F8186F82B0EEB994F868013EF0A8F894F86921C5F81C0F003A18BF09
:20CFE000012285F81A2F48B194F86A112B22002914BF11210121C28039F028FF002002B047
:20D00000BDE8F0413FF096BD94F86881002240462B2139F01FFD074640463EF083F8F8B1E5
:20D02000F7B12B22C5F8340FC280397AFDF744FB4FF000080E4AB2FBF6F3C3F34F00009009
:20D040009BB23946CDF8048005F57260A4F86E6131F058FAD5F8203FC3F8008085F8318F6D
:20D0600002B0BDE8F08100BF90600020A82D002040420F002DE9F84F254C94F87C3184F810
:20D08000703104F27317002604F5C8745FFA86FB0BF101085FFA88F8012117F8010F424693
:20D0A0000E448A4639F0D6FC4FF00009054640B3387804F80E9C04F80D9C04F80FBC04F80F
:20D0C00010AC44F8045C3EF02DF818B180F806A080F80780297AFDF7EFFA0E4A0021284658
:20D0E00039F06CFA0C4B23600C4B221D21462846C4E9013939F036F9697928684A4630F0FB
:20D1000093FC082E04F11C04C0D1BDE8F88F00BF9060002040420F0061DA0308BD3C0308CE
:20D1200070B52B4C2B4B94F8A802C4F8A03200220221C4E99822C4F86822C4F89C22A4F811
:20D14000A42239F087FC002841D0234B0268054603F1C000597C11B159688A422BD01833E3
:20D160008342F7D1002394F8A802C4F88C5184F880313DF0D7FF08B10223C380297AFDF748
:20D180009BFA2846154A002139F018FA144A1549C4F890110026111F2846134BC4F8943115
:20D1A000C4F8986139F0DEF8697928683246BDE8704030F039BC138D0C490D4A9BB2D2F804
:20D1C00030250133B2FBF3F381F82833CAE770BD9060002000FFFF002C2F002040420F0067
:20D1E00024620020E53C0308813E030898010020A82D00202DE9F04FD24DD34C85B00746D0
:20D200000E4605F5C270C02200215AF06CFF94F81433002B00F0E88094F81533002B00F091
:20D22000018195F87031012B72D0022B00F00681C64BDFF83CC303931F46BCE80F000FC7C1
:20D24000BCE80F000FC795F866E195F862319CE80700DFF820C3C4F8F8C2BEF1000C18BF04
:20D260004FF0010C072B87E8070084F81DC300F23881042B00F24681DFF8FCB2ABF1120395
:20D280004FF00008029346454FF003013EDD029B13F801AB029305EB0A030AF1010993F853
:20D2A00067715FFA89F938464A4639F0D3FB034638461F46002B00F01D813DF033FFCBF8AF
:20D2C000140020B14FF00303837180F8079095F8632195F862315FFA88F1002A00F008817B
:20D2E000FA7982F0010200923846524608F1010852F0A2FE002800F0FD804FF00103B8F139
:20D30000080F8BF811300BF1180BBCD1039B69E0DFF868C28E4FDFF86082C4F82063BCE825
:20D320000F000FC7BCE80F000FC79CE8070095F8623195F866C184F860330023BCEB030C38
:20D3400087E8070018BF4FF0010C9B4607F1980019464FF44C7284F81DC384F81E3307F53E
:20D36000727A5AF0C0FEA8F1120902965E46D4F82033B34240F3AC8019F8013B2B4493F80F
:20D380006771384639F0ECFB834638463DF0CAFE95F863310746002B00F09D809BF807307B
:20D3A00083F0010B0BF0010194F81D03013184F81C1308B18BF0010B002F00F0B380B879A5
:20D3C00000285CD041285AD0624B6349634AC4F8C832029EC4F8C412012384F81E33C4F8CB
:20D3E000D0220023C4F81833D4F818335BB10022012183F82C6083F82D101A6383F82E20A5
:20D4000005B0BDE8F08F564E564D0FCE0FC50FCE0FC596E80700A5F1200385E80700C4F81C
:20D420001833EDE795F86421003A384618BF01223146FBF751FBC4F81803D5E795F866319D
:20D44000002B3FF4F5AE95F86231082B7FF460AFDFF81CC1DFF81CE1BCE80F0004F5387713
:20D4600003970FC7BCE80F000FC79CE80700012387E8070084F81D33C4F8F8E234E0B888D8
:20D48000CAF80C704901B0FA80F041F009010136C0F11F004FF00303CAF80400CAF81410B7
:20D4A0008AF810B0FE71BB71384639F0CFFC1BF0010F384612D03EF0FDF8DAF80C30C8F8B1
:20D4C0001430082E0AF1200A08F118087FF44FAF029E1F4B86E79BF807B063E73EF0F0F802
:20D4E000EBE7082B7FF4C8AE1F4BC4F82433C3E6FA79F8E6194B174AC4F80433C4F8FC2235
:20D5000000236FE795F86531184AC4F82423012B05D0022B06BFBEFA8EF35B09002384F8DB
:20D520002833A9E6490141F009014FF0FF33CAF81410CAF80430CAF80C708AF810B0013678
:20D54000B2E700BFA82D002090600020706300203C63002055540408595404084D540408A1
:20D560004C820608BC63002009E3040839E304087882060821D805082C2F0020A4820608B3
:20D580002DE9F84FD54F97F8380097F839503DF0C9FD60B12D23C3802021044639F056FC8E
:20D5A0000A203AF083F8204640F096F918B9D7F89437DE0001D5BDE8F88F013D092DFAD8E6
:20D5C00097F83740CCB9402034F092F90028F2D090F90430797A092BC8BF143B3B440A295B
:20D5E00093F8984700F0B68193F8A43797F83620002A08BF1C46002CDDD020463DF092FD01
:20D600008046002800F09E812D23C380012139F01DFC012108463EF061F8D8F80030B8F86F
:20D6200004201A833C203AF07DF9002101203EF055F897F83930002B00F0D280A84CDFF840
:20D64000A892A84D002694F8081FD4F80C0FC94301F001013EF03AF894F8081FD4F8140FDA
:20D6600081F00401C1F380013EF030F8B8F1000F04D0D8F80030B8F804205A83D9F8043067
:20D68000C3F30803002B40F00581EFF31183002B40F00081D4F88420A968D4F884309A42B9
:20D6A000F8D1D4F8403F9942F4D8D4F83CCF4FF47A7000FB0CF35B1AB3FBFCF300FB023270
:20D6C0004FF0100C4FF47A710120D9F80430C3F30803002B40F0BD80EFF31183002B40F071
:20D6E000B880D4F88430D5F808B0D4F884E07345F7D1D4F840EFF345F3D8D4F83CAF01FB8C
:20D700000AFEAEEB0B0EBEFBFAFE01FB03E39B1A772BDAD994F8081FD4F80C0F01F0010125
:20D720003DF0D4FF94F8081FD4F8140FC1F380013DF0CCFFB8F1000F04D0D8F80030B8F8DE
:20D7400004201A83D9F80430C3F30803002B40F0CD80EFF31183002B40F0C880D4F8842011
:20D76000A968D4F884309A42F8D1D4F8403F9942F4D8D4F83CCF4FF47A7000FB0CF35B1A0E
:20D78000B3FBFCF300FB02324FF0100C4FF47A710120D9F80430C3F30803CBBBEFF3118351
:20D7A000B3BBD4F88430D5F808B0D4F884E07345F7D1D4F840EFF345F3D8D4F83CAF01FB95
:20D7C0000AFEAEEB0B0EBEFBFAFE01FB03E39B1A772BDED997F8393001369E42FFF633AF08
:20D7E00097F83730002B40F0A580BB6B03F0FF13B3F5803F7FF4DFAED7F8943713F08053B1
:20D800007FF4D9AE87F83930BDE8F84F4DF0C0BCEFF3118A8CF31288D5F808B02B68DB03F5
:20D8200044BFC4F8380FD5F808B0D4F88430D4F838EF5FFA8AFA8AF31188D4F83CAF734489
:20D8400001FB0AFEAEEB0B0EBEFBFAFE01FB03E3BDE7EFF3118A8CF31288D5F808B02B682D
:20D86000DB0344BFC4F8380FD5F808B0D4F88430D4F838EF5FFA8AFA8AF31188D4F83CAF22
:20D88000734401FB0AFEAEEB0B0EBEFBFAFE01FB03E33CE7EFF31181102383F31288D5F8E1
:20D8A00008C02B68DA0304D50123C4F8383FD5F808C0D4F88430D4F8382FC9B281F3118830
:20D8C000D4F83C0F4FF47A711A4401FB00F3A3EB0C03B3FBF0F301FB0232F1E69060002071
:20D8E000A82D002010E000E000ED00E0EFF31181102383F31288D5F808C02B68DA0304D501
:20D900000123C4F8383FD5F808C0D4F88430D4F8382FC9B281F31188D4F83C0F4FF47A719B
:20D920001A4401FB00F3A3EB0C03B3FBF0F301FB023229E7322039F0F5FF4046002139F0ED
:20D9400085FA52E7012139F081FA012108463DF0C5FE67E6D7F8BC375D057FF52CAE09F031
:20D9600043FB00287FF427AE002C7FF446AE22E60B6810B414681B1B036054684B681B1B6D
:20D9800043608B6892685DF8044B9B1A836070472DE9F047041E0D4612DB092C26DC824A52
:20D9A0000B468248A0FB0410C00800EB8000A4EB40000021125C1A7059702846BDE8F0872F
:20D9C00064422D23092C01F8013B24D8764A774BA3FB0403DB0803EB8303A4EB4303002078
:20D9E000D35C48700B702846BDE8F0876F4B632CA3FB04264FEAD60621DC6B4A0B466B495E
:20DA0000A1FB0601C90801EB8101A6EB4101515C03F8011BC5E7654A632CA2FB04364FEA93
:20DA2000D60637D8604A614BA3FB0603DB0803EB8303A6EB4303D35C01F8013BC7E7A3FB20
:20DA40000627B4F57A7F4FEAD7070DD2564A0B465649A1FB0701C90801EB8101A7EB4101BA
:20DA6000515C03F8011BCAE7A3FB072842F20F7294424FEAD80836D84B4A0B464B49A1FB9C
:20DA80000801C90801EB8101A8EB4101515C03F8011BDDE7A2FB0637B4F57A7F4FEAD7074E
:20DAA0000CD2414A414BA3FB0703DB0803EB8303A7EB4303D35C01F8013BB4E7A2FB0738BF
:20DAC00042F20F739C424FEAD80821D8364A374BA3FB0803DB0803EB8303A8EB4303D35C96
:20DAE00001F8013BDEE7324AA3FB080994424FEAD90921D82C4A0B462C49A1FB0901C90864
:20DB000001EB8101A9EB4101515C03F8011BB5E7274BA2FB08099C424FEAD90921D8224AE3
:20DB2000224BA3FB0903DB0803EB8303A9EB4303D35C01F8013BCAE71E4AA3FB09039442A0
:20DB40004FEAD30A21D80B461849174AA1FB0A01C90801EB8101AAEB4101515C03F8011B22
:20DB6000CAE7144BA2FB09029C424FEAD20A13D80E4B0D4AA3FB0A03DB0803EB8303AAEBC8
:20DB80004303D35C01F8013BCAE70A22BAFBF2F04DF0EEF80346D7E70A22BAFBF2F04DF03D
:20DBA000E7F80146E4E700BF84FE0608CDCCCCCC9F8601003F420F0070B4344890F8C0371F
:20DBC000A3F13001092957D800F5F864224600F2CF7012F8015FA5F13001092904D8824232
:20DBE000F7D1002070BC7047141B022C4ADD2848002101E010F8013B01EB810103EB410380
:20DC0000161A303B022E044603F0FF01F2DC214B03FB01F1A2424FF000030DD903EB830352
:20DC200014F8016B5B00303B3344A24203F0FF03F4D1194800FB03F32E2D06D01748A0FB14
:20DC4000032301EB930070BC7047013204200024157804EB8404303D6400092D00F1FF3096
:20DC6000A4B202D82C44A4B2013210F0FF00EFD1642202FB0433E1E700211D4600F5F86267
:20DC80000B46D9E7064C0021C4E700BF90600020516800208096980040420F00ABAAAAAAC5
:20DCA0005068002038B504460D460A460068FF215AF019FA21682944216038BD83B50C46D7
:20DCC0001646054632F0C0F8204632F0BDF80021204B0846002E08BF1E463DF0FFFC00210A
:20DCE00001203DF0FBFC28463AF044FAB0B1012100203DF0F3FC28463AF034FA07462046D1
:20DD00003AF034FA0028FAD0394620463AF036FA3846B047002108463DF0E0FC20463AF0FD
:20DD200029FA0028DFD0012100203DF0D7FC20463AF018FA0146284601913AF017FA0199E9
:20DD40000028F8D028463AF019FA002108463DF0C5FCC8E741DC0308F0B50023C1E900334F
:20DD6000C1E902330B610268DFF888C089B004ADC2F385572E4647FA03F0C007344604D592
:20DD800013F80C0004F8010B26460133062BF2D1164CDFF864C0C2F303200023205C337059
:20DDA0008DF81800C2F305370DF1190647FA03F0C007344604D513F80C0004F8010B2646DF
:20DDC0000133062BF2D100233370C2F3834406ABCDE90134084602F00F0305490095C2F353
:20DDE00003124DF04FFD09B0F0BD00BFC4FE0608ACFE0608CCFE0608BCFE060870B5094CBE
:20DE0000D4F8D027054662B10026D4F8D0072D21013641F0D3F8AE42F7DBBDE8704041F04F
:20DE2000ADBB70BD906000202DE9F04F5FFA81F9002185B00746084616463DF04FFC00212F
:20DE400001203DF04BFC3DF039F9022E0AD0042E44F6C01818BF4FF49648B9F1070F07D9E8
:20DE600000200CE0B9F1FF0F4FF41648F5D10326BE4D95F8D4372BB90020C5F8D80705B056
:20DE8000BDE8F08F032EBA4C0DD0A144002299F86701032138F0DEFD0028EDD0C4F8780505
:20DEA000C3799A07E8D495F8D40784F8936D0022032138F0CFFDC4F87C090028DCD0AD4A9F
:20DEC000AD4BC4F8343502F1480003234FF48061A4F83835C4F84805002302F24C404FF0AC
:20DEE000010A032EC4F83C85C4F86035C4F84015C4F85435C4F85035C4F84C05C4F844155F
:20DF0000C4F85C35C4F8583584F8843DA4F880ADC4F88C3DA4F8903D84F8923D91460ED077
:20DF2000D4F878B59BF804003DF0FCF8C4F87405584615F08BFC5146484615F09BFC3220BE
:20DF400039F0F0FC012E09D1D4F87C094146FAF7B5FFD4F87805FEF777FD0AE0022E3BD14E
:20DF6000D4F8780515F061FCD4F87C094146FAF7A5FFC5F8D8974FF0060A022E11D0D5F830
:20DF8000D8073AF0F7F860B1012100203DF0A6FBD5F8D8073AF0EEF8014600287FD13DF0C0
:20DFA0009DFB38463AF0E6F880B1012108463DF095FB4FF0050B4FF0000838463AF0DAF8D5
:20DFC0000146002874D101203DF088FB042ED6D0052039F0A7FCD0E7032E58D14FF0000A99
:20DFE0005146664884F894AD40225AF07CF88DF80FA04FF0010A9DF80F30072B09D95D48F4
:020000040800F2
:20E00000012115F037FCD4F87C094146FAF756FFAFE79DF80F3003EB430304EBC30393F8AA
:20E0200095316BB39DF80F3003EB430304EBC303D3F8983123B39DF80F30234493F86701A7
:20E04000F0B10022032138F005FD8346C0B115F0ECFB9DF80F3094F8942D03EB430304EB45
:20E06000C30305EBC201D3F89831C1F8DC379BF807300132DB0748BF81F8E0A784F8942DA4
:20E080009DF80F300133DBB28DF80F30B3E7042E7FF46FAFD4F8780515F0C7FB54E7D5F8B2
:20E0A000D8073AF05FF8014638463AF067F86FE738463AF057F895F82A3801468BB924289F
:20E0C00003D14FF0010385F82A38012E04D1384601913AF053F80199D5F8D8073AF04EF80B
:20E0E0006BE7012B06D14D280CBF0223002385F82A38EAE7022B06D13C280CBF0323002317
:20E1000085F82A38E1E7032B10D10A2802D985F82A88DAE7042385F81D0885F81C8885F8E5
:20E120001F8885F81E0885F82A38CEE7042B09D195F81E3885F82B08434085F81E3885F892
:20E140002AB8C2E7052BC0D195F81C3895F81D9895F81E084B4513D25A1C2B44484085F83E
:20E160001E0885F81C2883F82018AEE790600020A82D0020DC320020D08206086C680020E9
:20E180008842C4D195F82B3885F82AA8F42B9CD1B9F1000F99D12421384685F82A9839F007
:20E1A000EDFF4D21384639F0E9FF3E21384639F0E5FF4946384639F0E1FFF421384639F0BA
:20E1C000DDFFF421384639F0D9FF032E1BD0D4F87805437901689D080223AB40DB439BB225
:20E1E0000B828D892B408B810079202115F00CFBD4F878054A46494638F0B4F8D4F878358A
:20E20000186806F05FFC0022D4F87C09114638F0A9F8D4F87C39186806F054FC01202EE61E
:20E2200030B583B04D1C009303688572C2729C690023A04703B030BD03685B6C0BB1022174
:20E240001847704770B51D4C0968D4F830581C4ED4F82C48D6EDCB7ADFED1A6A491B00EE01
:20E26000901A0168F8EEE00A091B60EEA70A00EE101A20EEA07AB8EEC00A1C46A0EE007A7E
:20E28000B1EE400AF1EEC77A67EEA67AFCEEE77AC2ED007A4DF0C6FB9FED0B7ADFED0B7A2C
:20E2A000E0EE077AFDEEE77A17EE902A002ABCBF02F50C42A032226070BD00BF90600020CA
:20E2C000980100202C7D8E3FA00CB34500A00C4638B50F4C94F84B1801F03F018B1C024622
:20E2E00001F10A0584F8493884F8465804F6440084F8472808311DF02DFA254485F8420840
:20E3000094F846381C44000A84F8430838BD00BF9060002038B50B4C00250122802120466B
:20E3200033F0D2FA30B194F9040033F001FB08B1006838BD0135062D04F10C04EDD10020FB
:20E34000F7E700BFFC68002038B5041F00F1080554F8043FD81780EA430017F0FFF9A5427D
:20E36000F6D138BDF8B5C44CDFEDC47AD4F8B82894F82039B4F8227907EE102A2DED028B6C
:20E38000B8EE478A28EE278A002B60D1D4F82C3994F83D29002B40F3FC8007EE902A9FEDAB
:20E3A000B86ADFEDB86AF8EEE77AB7EE007AA7EE867AF0EE477A07EE103AF8EEC78AB7EE98
:20E3C000087A87EE270AC6EEA87A20EE270A58F085FB0F28B8BF0F2094F8213985B2A4F8A2
:20E3E0002259002B00F03C81AF4234D0B4F824399FEDA56A94F8BC6807EE103A07EE905A63
:20E40000B8EE477AF8EE677AC6EE076A86EE277A76EE887A37EE087AC8EE276AC8EE077A09
:20E42000B6B39A4B94F82629B4F82859C3ED047AC3ED087AC3ED0C7AC3ED106AC3ED147A88
:20E44000C3ED187A002A49D0BDEC028BF8BD94F82139002B72D094F8BC68002E40F0F88073
:20E46000B4F82439DFED886A07EE907A07EE103AB8EE676AB8EE477AC6EE877A86EE867A90
:20E4800077EE887A37EE087AC8EE276AC8EE077A7E4B94F82669B4F8285900225A609A6009
:20E4A000DA605A619A61DA615A629A62C3ED047AC3ED087AC3ED0C7AC3ED106AC3ED147A7B
:20E4C000C3ED187ADA625A639A63DA635A649A64DA645A659A65DA65002E65D1D4F82C393B
:20E4E00094F83D29002B40F3948007EE902A9FED646ADFED646AF8EEE77AB7EE007AA7EE1A
:20E50000867A07EE903AF8EEE77AB7EE086A86EE070A86EEA77A20EE070A58F0DFFA0F284D
:20E52000B8BF0F2080B2A4F82809002E3BD0A8428AD0002874D1BDEC028BF8BDD4F82C3930
:20E5400094F83E29002B40F38E8007EE903AF8EEE78A3D4607EE902A9FED496ADFED496A56
:20E56000F8EEE77AB7EE007AA7EE867AF0EE477AB7EE087A87EE270AC6EEA87A20EE270A1F
:20E5800058F0ACFA0F28B8BF0F2080B2A4F824092AE794F821390F25A4F82259002B7FF4D5
:20E5A00023AF2846F2E7054694F83C3984F8793C002D3FF449AF07EE905A9FED336A344BE6
:20E5C000F8EE677AD3ED006A86EE277ABDEC028B00220121C3F8082384F8781CC3F80C23DB
:20E5E000C3F81023C3F81823C3F81C23C3F8202337EE267AC3F82823C6EE877AC3F82C23B5
:20E60000C3F83023C3EDC57AC3EDC97AC3EDCD7AF8BD0F20A4F8280946B30F2D3FF414AF37
:20E6200007EE900ADFED186A194BF8EE677ABDEC028B86EEA77AD3ED006A37EE267AC6EE64
:20E64000877AC3EDC57AC3EDC97AC3EDCD7AF8BD94F82639B4F82859002B7FF4F5AE3DE7AE
:20E6600094F83E2976E73D460F208FE794F83C3984F8793C05469EE790600020BD37863561
:20E68000CDCCCC3D002474494E2DA63D4C690020D06900201D4991F8C027A2B3F0B4002676
:20E6A00005463346304637461BB991F8C0472D2C23D02E2A19D0CA1800EB800092F8C047D4
:20E6C000A4F13002092A4FEA40009CBFA0F13002A0180E2B14D80133CA1892F8C027002A1B
:20E6E000E2D106B14042F0BC70470133002DF8D0CA182A4482F8C077DDE701231E46EBE783
:20E700000020F0BC70470020704700BF906000202DE9F0410C4F0124A0231825E6B2FF2B47
:20E720000BDCC5F11B0103F10108D7F8CC0CDBB23246C9B2FFF774FD4346013DEFD10134D9
:20E74000052CEAD1BDE8F081906000201FB503AC8DF80C30009400238DF80D300DF052FAA1
:20E7600004B010BDF8B5054626201BF057FF154C014610BBD4F8D00C90F838301E3B012BE9
:20E7800002D894F8DD3C0BB139F0F8FC0E4F0026AE420ADBB4F8FE3C0133A4F8FE3C0B4B83
:20E7A000D3F88430C4F8103DF8BD17F8011BD4F8D00C39F0E3FC0136EAE7002384F80C3D51
:20E7C000EDE700BF906000206E6D0020A82D002010B58021044605F015F82046002105F078
:20E7E00011F82046BDE8104005F04CBB2DE9F041B14C94F8273DC4F8140D82B088465A2B23
:20E8000000F2B980DFE813F0CC00B700B700DC00B700B700B700B700B700B700B700B70035
:20E82000B700B700B700B700B700B7000F01B700B700B700B700B700B700B70033017400D5
:20E84000B700B7007400B700B700B700B700B801B7006201B700B7007C00B7000902B700C4
:20E86000B700B700B7005B00B700B700B700B700B700B700B700B700B700B700B700B70084
:20E88000B700B700B700B700B700B700B700B700B700B700B700B700B700B700B700B70008
:20E8A000B700B700B700B700B700B700B700B700B700B700B700B700B700B700E40194F8E5
:20E8C000283D9B0700F16982B4F82E3DD4F8292DD4F8681D5BBA9BB212BAD0188842C4F82F
:20E8E000743DC4F8702D03D904F04CFF002854DB0020A4F8600D0546284602B0BDE8F081F2
:20E9000094F86C3D002B40F0FF8094F9243D002B31DAD4F85C3D08469B689847002840F0D7
:20E920001E82B4F82E0DD4F8292DD4F8683D40BA80B212BA15189D42C4F8740DC4F8702D23
:20E9400007D904F01FFF002827DBD4F8702DD4F8740DD4F8643DD4F8206D03FB00F003FB33
:20E9600002F20225B042C4F8702DC4F8740D84F86C5D00F0CF8094F8383D5A1CD2B204EB86
:20E98000C30305204FF40051042A84F8382D83F83C0DC3F8401D00F0A0814FF0FF35ABE7F7
:20E9A000D4F8203D002BE6D1D4F85C3D08469B6898470546002840F0D281A4F8600D9BE736
:20E9C0003E4B002203F1120103F8012F8B42FBD13B4994F8623D94F8380D70250D70984255
:20E9E0004FF00C05CD7110D004EBC300013390F83C5D8D70B0F8400DDBB2042B40BA8881F1
:20EA000014BF84F8623D84F8622D94F82B3D12229342A4F8602D98BFA4F8603D00252846B4
:20EA200002B0BDE8F08194F8283DDA0700F13E81D4F85C3D94F82B0DDA6901EBC10102EB85
:20EA400081010A79531D834228BF0346A4F8603D002BE3D0013B1A489BB201331944034472
:20EA600011F8012D03F8012D8342F9D1D6E7154E154F35460823073EC5F10700A4F8603D42
:20EA8000002202E092F880211D462B46B54203F8012900EB030217FA82F2F3D1D4F85C3DB9
:20EAA0004046DB6898470028B8D0AB7863F07F03AB70002520E700BF9060002093900020AD
:20EAC000949000209B90002088810608D4F85C3DC74A5B680846111D98470546002840F059
:20EAE0003E81D4F8683DC34AD4F8641D013B180E1070180C09BAD37050701B0A0820937070
:20EB00005160A4F8600DF7E6D4F8746DD4F8702DD4F8643DD4F85C5DB2FBF3F24FF48057AA
:20EB2000BE4228BF3E462D69B249A4F8607D4046B6FBF3F39BB2A8470028C0F2BC80334678
:20EB4000AC4AD4F8140D812104F090FED4F8702DD4F8740DD4F8803D3244851B9E1BC4F8E4
:20EB6000702DC4F8745DC4F8806D002D7FF456AF032384F86C3DBFE69E4E0027334606F1AA
:20EB80000C0203F8017B9A42FBD1D4F85C3D40465B686A4601A998470546002840F0E98055
:20EBA000019BBDF80020013B190E52BAF3713171190C1B0A71710820B371022172810C23B2
:20EBC000BDF80220F07031727272A4F8603D93E6894E8A4F30460823073EC0F10705A4F8D6
:20EBE000603D002202E092F8882118460346864203F8012905EB030217FA82F2F3D1D4F8A3
:20EC00005C3D4046DB68984700283FF407AFF37863F07F03F37000256EE694F86C3D002B26
:20EC200061D194F9243D002BFFF6A5AED4F85C3D08469B689847002840F09180D4F85C3DDE
:20EC40004046DB6898470546002840F0BA80B4F82E3DD4F8292DD4F8681D5BBA9BB212BA77
:20EC6000D0188842C4F8743DC4F8702D00F29F80D4F8641DD4F8200D03FB01F302FB01F2E3
:20EC80008342C4F8702DC4F8743D7FF474AEB3F5805F28BF4FF480530121D4F8140D554A22
:20ECA00084F86C1D9BB204F00BFF25E607235449A4F8603DCEE694F8383D5A1CD2B204EB5B
:20ECC000C30304204FF48851824284F8382D83F83C0DC3F8401D7FF460AE002384F8383D18
:20ECE0004FF0FF3508E6D4F8746DD4F85C0DD4F8643DD4F8702D4569B2FBF3F2B6F5805F31
:20ED000028BF4FF480560846B6FBF3F339499BB2A847002862DBD4F8702DD4F8745DD4F819
:20ED2000803D3244AD1B9B1BC4F8702DC4F8745DC4F8803D2DB9D4F8140D294604F014FF7A
:20ED4000DAE5B5F5805F28BF4FF48055ABB2D4F8140D284A012104F0B3FE0025CCE594F887
:20ED6000383D5A1CD2B204EBC30302204FF468510AE694F8383D04EBC3020133DBB20220C9
:20ED80004FF46851042B82F83C0DC2F8401D22D084F8383D4FF0FF35AEE594F8383D5A1C0E
:20EDA000D2B204EBC30305204FF41051ECE504F0E9FC0028FFF6F1ADD4F8702DD4F8743D06
:20EDC00056E794F8383D5A1CD2B204EBC30302204FF41C51D8E584F8387DDEE594F8383DC2
:20EDE0005A1CD2B204EBC30304204FF440716BE7F46D0020949000209B90002088810608D3
:20EE00000083060810B51C203CF08CF91121044638F01CF820463CF04DFCC82038F082FD8D
:20EE20002046BDE810403CF04BBC00BF08B500203CF078F9054BC3F8880D08B12A23C38022
:20EE4000BDE80840402138F001B800BF906000202DE9F04FB34CD4F868375A69D2078BB01E
:20EE600002D50BB0BDE8F08F5A699B6912EA030AF7D0CAF307431AF4002F009340F00281BB
:20EE8000009B5D0743D41AF0020F5FFA8AF503D0D4F8683702225A61BAF1000FC0F211824D
:20EEA0001AF4006FCAF3072740F084812E0708D59D4B9E48D3F83C339847D4F86837082227
:20EEC0005A61ED0600F1E981F80600F1A981B90600F12E81009BDA0609D5934B9348D3F8D4
:20EEE0004C339847D4F868374FF480125A61009B9B06B6D58C4B8D48D3F850339847D4F84D
:20EF000068374FF400125A610BB0BDE8F08FD4F86C279369D26913401FFA83FBBBF1000F28
:20EF2000B1D0DFF80882CDF80CA045464FF0000909E05FEA5B0B09F1010908F1040805F114
:20EF4000280500F0DA811BF0010FF2D0D4F86C175FFA89F708694A6B04EB8703FA40D3F890
:20EF60007437D2019B68D2B202431A40D007D3B216D54B6BD8F81820012000FA09F023EAC7
:20EF800000034B63684B6948D3F83433012191603946984794F85F67012E00F0FC810123A7
:20EFA0001A0703D5D8F8182008239360DE0603D5D8F8182010239360580603D5D8F818200A
:20EFC00040239360990703D5D8F81820022393601A06AED5D5E94C60D5F82431D8F818C06C
:20EFE000311A8B42DCF8182028BF0B46033392B2B2EB930F9DD9D4F86C27323704EB870345
:20F00000CDE9019890469946B04238D2BEB3D5F8241194F85F37D5F82821371AB94228BF12
:20F02000394601F1030E4FEA9E0E83B98FB20337BF10D9F864A70AD0013352F8040BCAF8DE
:20F0400000009F42F8D1D5E94C60D5F82821DCF8183008440A44B042C5F82821C5F83401E6
:20F060000AD195F81C11D8F83420012707FA01F122EA0102C8F834209BB29E45C4D3DDE90C
:20F08000019856E7D4F86C379D69DB691D402D0C3FF4F6AE04F25C76DFF88CB0B046B146AC
:20F0A000002708E06D0807F1010706F1040608F128083FF4E5AEEB07F4D5F9B204EB810204
:20F0C000D4F86C37D2F8B02792685B691A40D007D3B218D594F85F07726D012398429360FD
:20F0E00007D11269D8F87C33C2F312029B1AC8F88C33DBF830334846984794F85F37012B50
:20F1000000F0578101239A0702D5726D022393601B07C7D5DBF8383348469847736D082221
:20F120009A60BFE7984F002098010020F4560020D4F86C37D4F874179A680868C2F34102D5
:20F14000022A08BF03224FF0000514BF65F30A0062F30A0008605A6842F480725A6006A805
:20F1600005F05EFDD4F86827D4F86C07D368BF49079D6FF38D23D3608068C0F34100014458
:20F1800091F89011032900F0CF80B949B9480126294484F85E6781424FF04006A4F8606757
:20F1A00000F215810E2161F38D234FF40051D36051618FE6B04B94F86E28D3F84433AF4850
:20F1C00000218DF817108DF817209847D4F86C17D4F8682794F8663788684FF400615161AE
:20F1E000002B3FF463AEC3077FF560AE94F87138012B7FF45BAE9DF81730032B7FF456AEF6
:20F20000D4F868389E491A6842F001021A601A6842F003021A600B6943F006030B6145E6F0
:20F22000D4F86C27954853684FF0000823F001034146536005F052F994F85D67414656B121
:20F24000904BFF2203EB860653F8045FD86BAA609E428260F8D1D4F86C3788484FF0FF3203
:20F260009A614FF00112DA610B2262F3070162F30708C3F8148019611A686FF30A121A60D5
:20F2800004F000FED4F868277B4B7C48D3F840334FF480515161984719E6D4F868379A6947
:20F2A00022F010029A611A6AC2F34340022802F00F0144D0062823D09A6942F010029A61D0
:20F2C00002E694F866373BB1D4F86828136823F0030161F307031360D4F86C2766495368A9
:20F2E000D1F84813654823F0010353608847D4F868374FF000425A61D2E5DDF80CA0C2E51E
:20F3000001EB8101D4F82C5804EBC1012E68D1F8E80AC4F8286DC2F30A1202442868C4F879
:20F320002C0DC1F8E82AC7E700214FF4007084F85E170921A4F8600761F38D2335E747F6CC
:20F34000F0701042B8D001EB8100C2F30A1204EBC00002F1030C5FEAAC0CD0F8DC5AD4F8B9
:20F360002CE84FEA810818BF002006D00130DEF8006045F8046B8445F8D1414404EBC1010F
:20F38000D1F8DC5AD1F8E80A15440244C1F8DC5AC1F8E82A90E7B9F1000F7FF400AE94F87D
:20F3A0006D38042B7FF4FBAD344804F06BFD3346F6E5002F7FF4A6AE94F86D28052A7FF479
:20F3C000A1AE4846019304F05DFD019B9BE62E48A5F57401A1F51051814203D80D2161F3B5
:20F3E0008D23E2E629492A482944814203D20C2161F38D23D9E62748A5F18C71A1F54341A0
:20F40000814203D80B2161F38D23CEE6224923482944814203D20A2161F38D23C5E620494C
:20F4200020482944814203D2092161F38D23BCE61D48A5F1B771A1F55851814203D208216C
:20F4400061F38D23B1E6194919482944814203D2072161F38D23A8E61649174829448142A1
:20F4600034BF0621052161F38D239EE688810608401E1BFF3F420F0098010020F456002082
:20F4800000ED00E008570020DFC810002013FBFE20D61300FF69180000D3CEFE40771B0043
:20F4A000C05BB3FEC091210040AC2700C01D6AFE40E13300803C36FEE09C4100704700BF3F
:20F4C000704700BF704700BF704700BF2DE9F0414FF0FF35324A33482C46002304E001336C
:20F4E0000B2B02F1100215D0917A0429F7D103F5B17100EB0111C979CF07F0D4661C1168FE
:20F5000001D0A942EBD21C4601330B2B0D4602F11002E9D1631C02D10120BDE8F081214D9D
:20F5200004F5B17705EB07139988F1B9DFF880802601AB19D8F8582D1B4916691B4A41F243
:20F54000186001EB442118580023B047D0B1022808D141F2CC6205EB0717AB58013B012104
:20F56000AB50B9710020BDE8F081DFF8448005EB0413D8F8582D41F21860D26818582601BD
:20F580009047D6E741F2CC6205EB0717AB580321B97141F2D061013B0124AB506C54BCE7F4
:20F5A00060CD002044B700205CB70020CDF50008984F0020044B41F2E472995C09B901212E
:20F5C000995401225A70704744B7002038B5174D174B41F2D0640020285504E001300B2880
:20F5E00003F1100314D053F80E4C8C42F6D11C78032CF3D16AB10F4B03EB40239A4201D0EC
:20F60000FFF7D8FF00F5B17005EB00100123837138BD41F2CC6100F5B1736A5805EB0313B9
:20F620000420013298716A5038BD00BF44B700206ACD00205CB7002038B5134B00209C7BD5
:20F6400014B11D688D4205D001300B2803F11003F5D138BD72B10D4B03EB40239A4210D00E
:20F66000FFF7A8FF0A4B00F5B17003EB00100123837138BD064B00F5B17003EB001082711F
:20F6800038BD022CECD1EDE75CCD00205CB7002044B700202DE9F84F12F0020E9B4606D0F9
:20F6A00028B9FFF787FF02252846BDE8F88F804C41F638056559002D5BD14FF0FF367D4F95
:20F6C000B146B046B24600253B68984200F0B68097F80EC0BCF1000F5BD0BCF1010F15D196
:20F6E00005F5B17C04EB0C1C9CF807C01CF0010F0CD11CF07E0F09D15FEADC1340F0A88075
:20F70000D7F808C0D44501D2E246A94601350B2D07F11007D8D1751C04D1B8F1FF3F00F0EC
:20F720009F80464641F2C86806F5B17754F80850013544F8085004EB061C41F21C694FEA28
:20F7400007184CF8095044F8085041F2186904EB07154FF000084CF80900C5F8048004EBD6
:20F760000715AD79042D9CD8DFE805F01A330F334D0004F5C25741F63C063F68A65907FBD7
:20F780000565A84299D3FFF715FF00252846BDE8F88F2E4601350B2D07F1100794D1BAE7E9
:20F7A00012F0010C70D104EB0710D51090F80780BBF1030F65F3C71880F8078062D94FF68B
:20F7C000FF7083455B4628BF03469BB204EB07108380BEF1000F16D004EB061303F5B05324
:20F7E0001833987B04280ED041F2C8654FF0040C60590130605141F2CC65586083F80EC0F2
:20F80000635901336351500705D504EB0710C37943F00103C371D30608D504EB0714E3794A
:20F82000C3F34502013262F34603E371224B012503EB46260E602846BDE8F88F05F5B1778F
:20F8400004EB07164FEA071CB67986B92E4669E7A84601350B2D07F110077FF435AF5AE70B
:20F86000B9F1FF3F18BF4E467FF45CAF8DE741F2C8682E4654F80850013544F8085044F8C2
:20F880000C506CE76346A1E70C4B0B49D3F8583D0B4AD3F8088001EB46210023C047002830
:20F8A0003FF473AF04EB07140223A371FCE600BF44B700205CCD00205CB70020984F002071
:20F8C00039F60008F0B5124D2B7841F63002022B0BBF070AC0F3D417C4B200F07F04A85852
:20F8E00083B00E4600230122384401A9FFF7D2FE01280AD12B78022B019B16BF53F824306B
:20F9000033F8143023F07043336003B0F0BD00BF44B7002010B5144602070B4610D50B4933
:20F9200041F2C472581C8B58834204D305D100232360012010BDFFF73DFE2060012010BD62
:20F9400021461846BDE81040BCE700BF44B700202DE9F0414268C2F308030B44B3F5007F49
:20F9600082B004460D4657D390F91A30591C0AD0304A03F5B17302EB0313FF21DA796FF3FE
:20F980000002DA71817694F91B305A1C0FD0294A03F5B17302EB0313FF20DA79C2F34501F7
:20F9A000013921EAE17161F34602DA71E0762378022B37D01F4A02F5C2531B68B5EB432F9A
:20F9C0004FEA432824DC41F648036768D6583E407342AB421CDCAB19434511D32169207E94
:20F9E00001AAFFF797FF012812D16768236963614744019B2361A5EB0801BF1B67608D191A
:20FA00002046F8F7EDFD20B93D446560012000E0002002B0BDE8F08115444560012002B0CE
:20FA2000BDE8F081616801202944616002B0BDE8F08100BF44B7002070B5154604460E46D8
:20FA4000FFF786FF50B994F8280028B9022384F82830C4E90B5670BD022070BD1DB12046D6
:20FA6000A847012070BD012070BD00BF10B4D0E9011390F91A208B4238BF0B46511C836083
:20FA80000AD0144B02F5B17203EB0212FF21D3796FF30003D371817690F91B305A1C0FD0DC
:20FAA0000C4A03F5B17302EB0313FF24DA79C2F34501013921EAE17161F34602DA71C476A8
:20FAC0000022436A5DF8044B4261426011460361B2E700BF44B7002038B544220021114873
:20FAE00058F001FB104B41F602011A784FF6FF745C52022A41F2E87118BF032203F5C05079
:20FB000041F64C055A5441F60C0441F6010203215D5900F8181910211D519954FFF7A6FF04
:20FB2000012038BD2CCF002044B700202DE9F041B1F904300F2B82B00C461646054632D0ED
:20FB40002846F8F771FD95F91B80B8F1FF3F074633D02D4B41F2186203EB08118A5890429A
:20FB600011D1183303EB4823A188013109B203EB4113A18028463360F8F756FD20600120A2
:20FB800002B0BDE8F081FFF715FD2846F8F728FD28B100230120336002B0BDE8F08100207B
:20FBA00002B0BDE8F0814FF40071FFF7D1FE0028F5D04FF6FF73A380C2E72846F8F710FD2A
:20FBC0000028E2D10FB9FFF7F5FC38460023112201A9FFF75FFD0128D7D1019B0B4A9A1A55
:20FBE00048BF02F2FF12B2F5B05F4FEA622106D24FFA81F885F81B80002BB5D1C5E7FFF782
:20FC0000D9FC019BF6E700BF44B700205CB7002030B50446C06983B010B9012003B030BD74
:20FC20000D460023032201A9FFF734FD0128F5D1B4F92030002B03DAFFF7BCFC0220EDE7C0
:20FC4000019A012D4FEA431102EB431303D0022D12D1E5255554A268DA612278032A04D192
:20FC600000221A775A779A77DA77626A5A83C2F30F429A8203B030BDE268DA61EDE700BF1B
:20FC800010B50378023B012B0446037E02D913F0060F5AD198063AD494F91A30591C0AD000
:20FCA0002D4A03F5B17302EB0313FF21DA796FF30002DA71A17694F91B305A1C0FD0264AD8
:20FCC00003F5B17302EB0313FF20DA79C2F34501013921EAE17161F34602DA71E076237E23
:20FCE0001B070BD51C4841F2C873C35C072B01D0FFF760FC41F2C8730022C254E26A0023A7
:20FD0000237084F82830FAB1BDE81040104700231249E0691A018A58904206D001330B2BAF
:20FD2000BAD01A018A589042F8D10B4A03F5B17302EB0313DA79C2F34501013921EAE17148
:20FD400061F34602DA71A7E710BD0121FFF760FF0128F9D1237E9DE744B700205CCD00206E
:20FD600030B1027822B190F828201AB1002070470120704710B5D0E90142A242C16238BF4C
:20FD800022460321826080F82810FFF779FF012010BD00BF2DE9F04FDFF868918A4699F8A4
:20FDA0000010DAF800300229174683B0834641F6300240F08B8059F80250DEB2A6EB03083A
:20FDC00005EB1325B8444FF480729044BB4208F1FF38B8FBF2F875D2A844032906EB0704D1
:20FDE000A4EB03040CBF80224FF48072944228BF1446A8EB050366B994422CBF0A220B22E0
:20FE000001A92846FFF746FC012809D003B0BDE8F08F0B2201A92846FFF73CFC0128F5D157
:20FE200099F80020DAF80010022A01F1010321D0A64210D2019906F18042013A081F00EBB2
:20FE4000840001EB820242F8043F824203F10103F9D1DAF80010A61B7318BBF1010FCAF8FF
:20FE600000301BD09F4205F101052BD999F800100026B2E7A642EED2DDF804C006F10042AC
:20FE8000013AACF1020000EB44000CEB420222F8023F904203F10103F9D1DCE7BB42E1D1BD
:20FEA00099F80030022B21D004F18044019B013C4FF0FF3243F82420DAF800309F4205F109
:20FEC0000105D3D8012003B0BDE8F08F59F8022003F07F060329C3F3D415A6EB03081544CE
:20FEE000B84414BF4FF4807280226EE704F10044019B013C4FF6FF72584623F8142003B09F
:20FF0000BDE8F08F44B700202DE9F04190F838300446032B51D8DFE803F002323B462D4BE3
:20FF2000C0681978E76A03F5C252032911680CBF80264FF4807601FB06F141F2C47C00EB0B
:20FF4000412041F2A87841F2AC7E53F80C20E06053F80E0053F808502261A5EB4125A0EBD9
:20FF60004121901943F8085043F80E1043F80C00C4E90C205FBB6262012384F83830164826
:20FF80000021FFF745FE012811D1022384F83830626B04F130010120FFF7FCFE012806D1EF
:20FFA000032384F8383000212046FFF731FE431EDBB2012B02D9BDE8F081022094F828307A
:20FFC000062B04BF002384F82830BDE8F081921B2263D1E744B70020E4CE00202DE9F04FF4
:20FFE000DFF8248198F80060012887B08CBF00230123032E02930C460B68154639D0022E84
:020000040801F1
:2000000062D14FF480724FEA1329DFB201920138012823D8012203929D421AD9384E06F17B
:20002000880A06F11C0B32681AB1DBF8001099424ED0DAF8000000234844092205A9FFF77F
:2000400029FB01281FD002280FD020B123689D42E9D82560032007B0BDE8F08F87B1FFF7AE
:20006000A9FA022007B0BDE8F08F022007B0BDE8F08F80220192C3F3D41903F07F07C6E7E5
:20008000019A0392C8E7DDE902C1059ADDF804E098F80030022B14D0032BE6D152F8273049
:2000A00023F07043B3FA83F35B0963450F44236823D00B4477452360EAD309F10109002704
:2000C000C5E732F81730EDE74FF480720192D2E70C490968013A02EB41224902B2FBF1F282
:2000E00003991344B3FBF1F201FB12320AB10B449B1A9D42236096D8ABE7AB42ABD3A8E721
:20010000ECCE002084CF002044B70020F0B5104D2B7841F63002022B0BBF070AC0F3D417C3
:20012000C4B200F07F04A85883B00E4600230322384401A9FFF7AEFA012807D12B78022B72
:20014000019B0CBF23F8146043F8246003B0F0BD44B700202DE9F04390F83C30002983B0D6
:20016000044614BF02210021042B7BD8DFE803F0030C3C476900FFF74BFD012870D1626B72
:20018000002A75D184F83C00404EDFF80881404D4FF6F7771DE01FFA80F9B94594BF4FF0EA
:2001A00000094FF0010901A9B9F1000F46D1FFF789FB0128494650D1206BFFF7A7FF0128D0
:2001C0004BD1019B2A682363013B934228BF13462B603378206B032BDDD1404594BF4FF04A
:2001E00000094FF00109DEE7426B04F130010020FFF7D0FD012833D1032384F83C30234B89
:20020000E16A41F2C47003F5C2521D581268195041F2A87741F2AC76D8596D1A995902FB7A
:2002200005F200EB422501EB422203F5BD500021DD519A51FFF7ECFC012811D1042384F85A
:200240003C3094F82830042B04BF002384F82830A36B8BB120469847012003B0BDE8F083EA
:200260000228FAD194F82830042B09D00220F4E7022384F83C30B8E7012003B0BDE8F08308
:20028000002384F828300220E7E700BF44B7002088CF0020F7FFFF0F38B590F834300446FF
:2002A000052B46D8DFE803F01F033F101963006B4FF0FF31FFF72AFF01283AD1E06A0028AA
:2002C00039D1032384F8343000212046FFF7A0FC01282ED1042384F8343094F82830082BAF
:2002E0002DD0012038BD41F63803224DEA5800F1300102320120FFF771FE012824D0023895
:20030000C0B2012815D8052384F8343094F82830082B04BF002384F8283041F2E5730122CE
:20032000EA54022038BDC06A216BFFF7EFFE0128C7D0002038BD022384F83430F4E70023F7
:2003400084F82830012038BD05F5C252E3681168D4E90B2003EB412341F644016850C4E9C6
:20036000033002B96062012384F83430A0E7014DCCE700BF44B700202DE9F04F436883B034
:20038000C3F308081646002A00F0E180714B05468946A3F1180B4FF0000AC8F5007495F92B
:2003A0001A70B44228BF3446791C28462ED0F8F73BF90BEB071341F218629B58984205D0D9
:2003C000FFF7F8F8504603B0BDE8F08F614B03EB472022464946404457F024FE002221465C
:2003E0002846FFF729FBA2440028EBD02B7E1B0706D5594B2A691B689A4201D3FFF7DAF8D4
:20040000361BA1444FF00008C7D1DBE7F8F7E8F8002849D12846F8F707F96968C1F3080307
:200420002BBB21F4FF7323F0010303F50072AB689A422CBF062207222B7E03F00C030C2BC1
:200440001CD0002301A9FFF725F90128BAD10198404BC31A48BF03F2FF13B3F5B05F4FEA1C
:2004600063224FD257B2AF760028B2D1AAE72B7E03F00C030C2B4FF00702E2D19BF800C03C
:20048000364BBCF1030F1B680CBF4FF0800C4FF4807C03FB0CF34FEA432C0CF1FF3C0CEAF1
:2004A0000101A3EB5123CDE72B7E1A072ED59BF800102A4B95F828201B6803290CBF8021AF
:2004C0004FF4807103FB01F3062A4FEA43233FF479AF23490868834230D891F83D30002B02
:2004E0007FF470AF002A7FF46DAF6B6985F83820062185F82810EB622846FFF705FD012850
:2005000088D05FE7FFF756F80198ACE7154B1A78002A7FF457AF95F82820002A7FF452AFC5
:20052000082185F8342085F82810D3F85F206B692846C5E90B32FFF7AFFEE0E741F2E573A0
:20054000012250460BF8032003B0BDE8F08F924638E700BF5CB7002008CF002084CF002092
:20056000ECCE002029CF00202DE9F04390F8384083B00546032C00F29F80DFE804F0021AAB
:20058000890BFFF789FE012811D002280BD1032385F838302B6C002085F82800002B00F0B8
:2005A000878098470224204603B0BDE8F08385F838002B78022B77D0404A6F6841F648034F
:2005C000D3581F40C7F34F272846F8F72DF8DFF8F08006463F1A0AE0D8F80030013B9945EF
:2005E0004AD2FFF7B5F908B9FEF7E4FF0136022201A900233046FFF74DF8BC1901281FFAB2
:2006000084F94FF400724FF000010446CBD1019857F069FDEB694FF400712846002BDBD0F0
:200620006B68002BD8D1019B4FF020324FF02E0C1A605A6083F800C0C3F807204FF0100EBF
:200640006C6A1A625A6283F820C083F821C0C3F8272083F80BE0EA6B5C83C2F30F4CC4F372
:200660000F4483F82BE09C825A87A3F834C0D8F80030013B9945B4D3C3EBC35359022846E5
:20068000FFF766F908B9FEF795FF022385F838302B6C002285F8282063B1284698470124AD
:2006A000204603B0BDE8F0836F68C7F34F278BE7022478E7012476E7002474E744B70020EF
:2006C00084CF00202DE9F04F90F8303089B00446042B00F2A880DFE813F0A900B200050074
:2006E0008A00E800B64D41F61003EB5C002B40F09A80B44F04F11C09B84607F1380BBA4629
:2007000001AE324649464046FFF710FA012840F018810198002800F0FA800378E52B01D024
:20072000002BEED1A84A821A48BF02F2FF12B2F5B05F4FEA622380F03C811B01A34A134434
:200740009A7B042A0CD041F2C86104266A5801326A5041F2CC615A609E736B5801336B5068
:2007600041F60202AB565E1C09D003F5B17305EB0313FF26D979AE546FF30001D97141F66B
:2007800003016B565A1C0ED003F5B17305EB0313FF26DA796E54C2F34501013921EAE17152
:2007A00061F34602DA712022002157F09CFC2346019A53F8311F58685060116019899B7AD9
:2007C00093721181019B627EDA7205A84AF0FAFABDF81430002B40F02F8144F28172019918
:2007E00003200A82CB810A83CB8284F83000237E980600F1A9802046FFF738F92369002BDB
:2008000000F0AE80237E03F0F70213F00403227640F0B480122A00F0BA80002384F82830CA
:200820002046E36A984709B0BDE8F08F6548FFF71DF94FF6FF720123228484F83030614F84
:2008400004F11C0801AE04F13109324641463846FFF76CF901282FD00228E4D1584D41F6E6
:200860000202AB56591C09D003F5B17305EB0313FF20D979A8546FF30001D97141F60301AE
:200880006B565F1C0ED003F5B17305EB0313FF20DA796854C2F34501013921EAE17161F308
:2008A0004602DA71042384F830300020E36A2070984709B0BDE8F08F019D0B224946284621
:2008C000002D00F087802B78002B00F0838095F80BA01AF0080FB8D157F031FC0028B4D130
:2008E000637E8AEA0303DB0640F1C780344D41F602016B565F1CC1D003F5B17305EB03139A
:20090000FF26DA796E5460F30002DA71B6E73B782F49022B4FF009025046C3D00B78002BE7
:20092000C0D1C1E905330A708BF800304A6B0B7351F8143CC1E90132FFF716FE01283FF408
:20094000E0AE0228AED06EE7E0690023112205A9FEF7A0FE01283FF44EAF09B0BDE8F08FF6
:20096000237E19077FF559AF154A41F2C873D15C00297FF458AF0721D1544EE70023E26AAC
:20098000A16884F828302046FFF756F84BE7626AE06AA0630421C4E90233C4E90B2284F828
:2009A0003C30636384F8281063622046FFF75EF839E7FEF7FFFD01986FF00F03BEE600BF5C
:2009C00044B700202CCF00205CB700205CCD002054CF0020474D41F60202AB565E1C09D0FF
:2009E00003F5B17305EB0313FF20D979A8546FF30001D97141F603016B56581C0ED003F575
:200A0000B17305EB0313FF20DA796854C2F34501013921EAE17161F34602DA71237EDA0684
:200A20007FF540AF3448FFF721F84FF6FF720223228484F8303056E6304B05A9B3F98C2DA1
:200A400002A84AF0DDF99DF80C309DF80D609DF80A509DF80B20BDF808109DF80E00DB020D
:200A600043EA461342EA4512A1F2BC7143EA500342EA41229BB292B2B1E6A98A6B8B204AE3
:200A800043EA014312686362EB69A3605202B3FBF2F102FB113109B113445B1A154DE36000
:200AA00041F6020184F819A06B565E1C09D003F5B17305EB0313FF20DA7968546FF30002FF
:200AC000DA7141F603016B56581C0ED003F5B17305EB0313FF20DA796854C2F345010139F8
:200AE00021EAE17161F34602DA71032384F830307DE600BF44B700202CCF00209060002048
:200B000084CF00202DE9F04390F82830013B83B00446082B41D8DFE803F048054D525865D1
:200B2000406A4300384B4668056B41F6480103F5C2525F5813683740EA19B2EB432F4FEAA7
:200B4000432816D258E02169207EFEF7E3FE012823D1256B666823696361A5EB08053D4423
:200B60004644F61B019B6660A84525634F46236142D82046F7F734FD01AA81460028E2D0FF
:200B80006668A368E26A9E4238BF1E460023A66084F828300AB12046904703B0BDE8F08335
:200BA000FFF7E2FC03B0BDE8F083FFF78BFD03B0BDE8F083FFF764F803B0BDE8F08300210F
:200BC000FFF7C8FA03B0BDE8F0830121FFF7C2FA0128E2D10023216C84F828302046FFF702
:200BE000BFF8DAE7FFF790F903B0BDE8F083FFF753FB03B0BDE8F0832046F7F7F1FC0028BB
:200C0000BFD12E446660BCE744B700202DE9F04782B0054602AF18461C460E46904654F0A5
:200C20007DFF083020F00700ADEB000D0DF1080A013CD14614F8013F5BB989F80030424647
:200C4000CDF800A0314628463DF008F8BD46BDE8F087184649F08CFEC3B2A3F120023F2A49
:200C600088BF202309F8013BE4E700BF2DE9F04704460D469046002144221E46089F57F08A
:200C800032FA01234FF6FF722676628384F828302B782E2B4CD02E4604F1310A307804F1A0
:200CA000390968B12E280BD049F062FEC0B20AF8010BCA4506F1010607D030780028F1D119
:200CC00020200AF8010BCA45F7D130782E2808BF707804F1380908BF013604F13B0A58B1CB
:200CE00049F046FEC0B209F8010FD14506F1010607D030780028F3D1202009F8010FD1450E
:200D0000F7D118F0100F14BF0323012384F819802370E7622B782E2B26D16B7823BB0323FC
:200D2000204684F83030FFF7CDFC2046BDE8F0876B78002BAFD1114B41F2F47241F60C006A
:200D400041F2F0719A5818585958E26041F601026062A1609A5C627641F2E8729B5C2370C8
:200D6000E7622B782E2BD8D00023204684F83030FFF7A8FC2046BDE8F08700BF44B700202B
:200D800010B5114C94F8663723B9104B4FF480225A6110BD0E4A136823F00603136054F0BE
:200DA00089FE94F86637002BEFD0D4F86C379B68DB07EAD5D4F86828136823F0030161F344
:200DC00007031360E1E700BF984F0020003C014010ED00E008B50121032003F07FFD72B615
:200DE0004AF0B6FE2DE9F04F8DB0CF4CDFF84C93CE4D00904FF0000854F80B0C002800F035
:200E0000FE8037F0B7F90646002800F0DB81D9F8843044F8073CE0260023C54F04F8033C41
:200E2000A4F10B0B06FB08F654F80B0C37F0A2F9002800F0E48054F80B0C37F093F914F845
:200E4000023C5A1E82460B2A0DD8DFE812F01F003A004600530083009B00E30017013701EE
:200E600042017901910124280CD0009A3AB995F8B628824240F08281012204F8032C0D2B86
:200E8000D2D186E0012304F8023CCDE700234D28C4F8C53084F8CD3084F8CE3004D05828A7
:200EA00008D004F8023CBFE7022204F8022C84F8C430B9E7032304F8023C022384F8C43027
:200EC000B2E704233C2804F8023C0BD0BAF13E0F0CD0002304F8023CA6E70A233C2804F88E
:200EE000023CF3D1002304F8013C9DE7012304F8013C99E7D4F8C500BB190344421CC4F86D
:200F0000C52083F8BFAD94F8CD00022A8AEA000184F8CD1088D12378C02BDAD86278FF2A1E
:200F200008D1052BD5D9012384F8C430072304F8023C79E7A4F8C12000229342C4F8C93079
:200F400014BF0523062384F8C320C4F8C52004F8023C69E7D4F8C500BB190344421CC4F81D
:200F6000C52083F8BFAD94F8CD00D4F8C9308AEA00019A4284F8CD107FF456AF062304F840
:200F8000023C51E794F8CD308342A2D10D2304F8023C14F8017C002F40F0F680654B089406
:200FA0000FCB04AE86E80F00D4F8C930D4F8D100ADF82A7023440993B4F8C130ADF82830EA
:200FC00094F8C3308DF82C3001238DF82D30324603AB08A9039730F00BFE48B1049B0593E1
:200FE00094F8C420544B0493314658462EF0F2FC039E002304F8023C002E40F0DB8008F17A
:201000000108B8F1030F04F1E0047FF4F5AE0DB0BDE8F08FD4F8C500BA190244431CC4F877
:20102000C53082F8BFAD94F8CD2094F8CE0001938AEA020284F8CD205146D52249F050FF77
:20104000019B84F8CE00072B7FF4EEAEB4F80530C02B3FF63EAFB4F80320A4F8C120A27815
:2010600084F8C32000229342C4F8C93014BF08230923C4F8C52004F8023CD5E6D522014667
:2010800094F8CE0049F02CFF94F8CD3084F8CE008AEA0303D4F8C50084F8CD30BB19034420
:2010A000421CC4F8C52083F8BFADD4F8C9309A427FF4BAAE092304F8023CB5E694F8CD3044
:2010C000434084F8CD3094F8CE3083427FF401AF54E7D4F8C500BA190244431CC4F8C530AD
:2010E00082F8BFAD94F8CE000193D522514649F0F7FE019B84F8CE00052B7FF495AEB4F8E8
:201100000120B4F80330A4F8C120227884F8C32000229342C4F8C93014BF0B230C23C4F8C1
:20112000C52004F8023C7FE6575D002090600020984F00201C83060818980120A82D0020CD
:20114000D522014694F8CE0049F0CAFE84F8CE00D4F8C500BB190344421CC4F8C52083F886
:20116000BFADD4F8C9309A427FF45EAE0C2398E694F8CE3083427FF4ACAE07E7232804BF1E
:20118000022204F8032C7AE6012F4FF0000602D004F8026C33E7D4F8C93008942344099371
:2011A00008A8B4F8C130CDE90A66ADF828302DF093F8EDE754F80B0C2EF046FE54F80B0C1B
:2011C000B0471CE714F8033C002B3FF418AFD9F8842054F8071C521A632A7FF610AF012B68
:2011E00029D0022B7FF40BAF54F80B3CC5F8903D0122C5F8943DC5F89C3D402385F88E2D9D
:2012000085F8A10D0D4A0E4885F8A03D0D4BC5F8982DC5F8D037C5F8E43D3EF0B3F94FF403
:20122000005034F071FC08483EF0A2F985F8E86D85F8E96DE3E6FFF7CDFD00BFF153040877
:20124000DCFE0608286E002012FF0608202301480B807047F4040020642301480B807047D9
:2012600014050020432301480B8070477805002010B5074CD4F8C800FF2807D0054951F866
:20128000042BF7F7D5F8FF23C4F8C830002010BDF404002098CF0020EAE700BF08B5D0F8ED
:2012A000E4355B6A9847002008BD00BF08B5D0F8E4351B6A9847002008BD00BFD0F8E43546
:2012C00010B504461B689847D4F8E8359B689847002010BD08B5D0F8E435DB6903B1984770
:2012E000002008BD08B5042290F81211D0F8E83580F8131180F81221DB689847002008BD48
:2013000010B5D0F8E83504461B699847032384F81231002010BD00BF0B0630B41CD401EB14
:20132000810200EBC202002300EB810582F8741382F8753301241A4604FA01F16D6D61F321
:201340001F4201696FF3CF332B60CB6923EA0203002030BCCB61704701F07F0101EB8104BC
:2013600000EBC404012200EB8105002384F81C1184F81D2102FA01F11A46AD6961F30F02D7
:20138000DFE700BF10B581210446FFF7C5FF20460121FFF7C1FF024B0020187010BD00BF9E
:2013A000FC6D002010B581210446FFF7B5FF20460121FFF7B1FF82212046FFF7ADFFF7F782
:2013C0007FF8002010BD00BF38B50D4604468321FFF7A2FF29462046FFF7E4FF002038BD62
:2013E000F0B416460A063AD401EB810500EBC5052824002204FB0104022B85F87413C5F848
:201400007C6385F8773385F8752304F55D7448D0154600EB8107012202FA01F17F6D61F3B0
:201420001F45D7F800C01CF4004F11D1E488204946F0805242F4004242EA834204F00F042B
:201440001C4B42EA845211400CEA0303194339600269D3692B430020F0BCD361704701F024
:201460007F0101EB810500EBC5052824012204FB0104022B85F81C11C5F8246185F81F316C
:20148000A5F8221185F81D2104F58E740CD0002500EB8107012202FA01F1BF6961F30F05B1
:2014A000BFE722711546B4E700252571F0E700BFFF87CC13007833EC002310B5194604461F
:2014C0004022FFF78DFF8021204600234022FFF787FFD4F8E835A078012284F812215B688A
:2014E0009847002010BD00BF70B44B78012B26D00B784A6900EB83035C6D25682369D2B14C
:201500008A684A6102F07F0223F4002323F07F0342F4002213432361C378012B04BF0B691C
:201520006361C5F3076363F07B0363F31F652560002070BC70478A6802F07F02E4E7826977
:201540004C691568136944B38E68B4428CBF06F07F0404F07F0423F4002323F07F0344F4B8
:20156000002443EA040388BF4E611361C378012B1DD0C5F3076464F07B0464F31F6515600F
:20158000002BD5D14B69002BD2D002690878516B012383400B435363CAE723F4002323F069
:2015A0007F0343F400231361C378012BE1D10B780C6900EB8300C5F30763816963F07B037F
:2015C00063F31F654C610020156070BC704700BF2DE9F0434B78012B30D00B784C6900EBF2
:2015E00083035E6D356837691CB38B681C44013CB4FBF3F4C4F3090203FB02F3C3F31203E8
:201600004B61144643EAC44363F31C073761C378012B04BF0B697361CB78012B44D0C5F3D2
:20162000076363F07B0363F31F6535600020BDE8F0838A680124C2F31203E3E791F8008014
:201640004E6900EB880EDEF818C0DCF80050DCF8107076B3D1F80890384A06EB0904013CE5
:20166000B4FBF9F402EAC444C6F312022243CC7807F060473A43012C174649D0CCF81020B2
:20168000C278012A55D00269516B03FA08F30B435363C5F3076363F07B0363F31F65CCF80C
:2016A00000500020BDE8F0834B7973B345F00055B5E707F0604747F40027CC78CCF810700A
:2016C000C378012B2FD0012CE3D102699268D20554BF45F0005545F08055C5F3076262F06D
:2016E0007B0262F31F65CCF80050002B9ED1B0B203308010DEF8D04098D0CA6852F8041BD8
:20170000216001339842F9D190E745F0805586E764F35E77CCF81070C378012BD5D10A6992
:20172000CCF81420D1E70A69CCF81420012CB0D1CBE70B69CCF81430ABE700BF0000F81F4A
:201740000E4BDA68D20310D4DA68D1060FD4DA68D20510D4DA6812F0E00F0AD1DB6813F0E8
:20176000020F14BF0820092070470120704706207047072070470220704700BF003C0240D4
:2017800000207047104AD068A8B113699BB188420FD88B4234BF00230123DBB243B193698A
:2017A0005161994204D0094B9161142083F8CC0070470023F1E7A1F59C53083BB3F57A7FEC
:2017C0002CBF00230123E9E798CF0020F4040020054B5A7F19778A4204D0044A59771420BD
:2017E00082F8CC00704700BF98CF0020F4040020704728B1034B987F012894BF00200120DC
:20180000704700BF98CF002008B5FFF7F2FF50B1054AD37F127F5B0003F00203002A18BFA0
:2018200043F001030B6008BD98CF002008B5FFF7E0FF10B1014B1B6A0B8008BD98CF0020BF
:2018400070B5FFF7D6FF50B10A4A958C35B1966A0023B3421C4603DB002000E00D7070BD3A
:2018600002EB44040133A48DAC42DBB2F1D10B70F5E700BF98CF002008B5FFF7BAFF10B1C7
:2018800000230B70137008BD0420704728B1034B93F9CE00003818BF01207047F404002007
:2018A00008B5FFF7F3FF50B1054B93F9CE20012AC3BF93F8D130C3F340030B60002008BD36
:2018C000F404002008B5FFF7E1FF18B1024B93F8D0300B7008BD00BFF404002070B5FFF78A
:2018E000D5FF38B10E4C94F8D130DB0703D500230B70137070BD0B4D94F9CF3095F83C602F
:2019000093FBF6F301330B7094F9CF4095F83C1094FBF1F301FB134301331370EAE700BF20
:20192000F404002098CF00200320704770B50A4A92F8403006255E1CB6FBF5F405FB146404
:2019400092F84150AC4205D002EBC303C3E9110182F8404070BD00BF98CF0020002230B5C4
:2019600004461046914200DC30BDA35C0825584010F0800F4FEA400318BF83F0D503013DFC
:20198000D8B2F5D10132EDE710B5D9B10E4B586F814217DCB2B1DB6B9A4213DC0B4C013AC5
:2019A000013903FB012184F8DC1004F1D8000521FFF7D4FF062184F8DD0004F1D800BDE8B7
:2019C0001040B3E710BD00BF98CF0020F40400200023038083708380C3800381704700BF19
:2019E000074A084992F8783009780133DBB2994282F8783004BF002382F87830704700BF56
:201A000098CF002038490020F8B5794CE36F83B1784B1B6893F82E305BB1774B94F880207D
:201A2000A3FB0013012A4FEA931330D0022A08D002B1F8BD714B9842FBD9012384F88030C5
:201A4000F8BDD4F8842064329A423ED894F8783004EB031393F8F824FF2A06D06849013216
:201A6000012083F8F82481F8DE00FFF7B9FF654B1B780122092B84F88020DAD1B4F87A35ED
:201A8000614A01339BB2A4F87A355380F8BD94F878105C48C4F884308C2303FB01430078B6
:201AA00083F89A20002384F8963004F18C050A2202230928C4F8885084F8972084F8803091
:201AC000B7D1514B01311980F8BD94F8962094F897309A42ADD104F18B0004F19405002342
:201AE00010F8012F082153405A0013F0800F08BF5B0082F0070214BFD3B2DBB20139F3D186
:201B00008542EDD194F895209A4239D194F8786094F8935094F89430B4F88F00B4F891205E
:201B200094F88DC004EB061743EA052394F88E5087F8F81440BA52BA81B292B245EA0C209E
:201B40002F4DC7F8FC141BB294F98C10C7F80025032E4FF00102A7F8FA04A7F8043587F8F9
:201B6000F91485F8DE2008D8264A12780C2A29D00D2A02D1244B23F81610FFF731FF5CE7B1
:201B800094F8783004EB031393F8F824FF2A06D01B490132012083F8F82481F8DE00FFF7CA
:201BA0001FFF184B1B780122092B84F880207FF440AFB4F87835144A01339BB2A4F87835BB
:201BC0009380F8BD1149124A91F822100E4803EB830303EB830349089B0093FBF1F382FBB3
:201BE0000312DB17C3EBA20320F81630C5E700BF98CF0020A8630020D34D62103F4B4C00A8
:201C0000F40400201C43002020430020082F0020676666660B4B93F8961093F8972091421E
:201C20000ED010B493F89620D3F88840511CD2B2C0B2C9B283F89610A0545DF8044B7047E0
:201C4000704700BF98CF0020FD2870B522D0F02804D0EF2822D00224204670BD114D03201C
:201C6000052641282E444FF0000405F1010580F080030DD0042B0BD9FFF7E6FF2044B54206
:201C8000C4B2E9D015F8010B412880F08003F1D10420F3E7044D0B200426E2E7034D0C20F5
:201CA0000626DEE750010708580107084801070800B5062983B00A464FF03203014628BF0A
:201CC00006220DF101008DF8003056F0ABF9044B6846D3F87C35984703B05DF804FB00BF20
:201CE00098CF00205E2810B511D05D2805D00D4BBDE81040D3F8803518470A4CD4F88035D4
:201D00009847D4F880353D20BDE810401847054C5D20D4F880359847D4F880353E20BDE800
:201D20001040184798CF002007B50DF1060211F0A7FA68B1084BBDF80620B3F884159A8460
:201D4000914205D00549A3F88425142081F8CC0003B05DF804FB00BF98CF0020F40400206B
:201D600013B50446FFF792FD08B300230DF106022046ADF8063011F083FAC0B10D4C9DF8CA
:201D8000062094F9CE1084F8E320032908BF62F07F024FF00501084808BF84F8E320FFF79C
:201DA000DDFD062184F8E4000348FFF7BFFD02B010BD00BFF4040020D30500202DE9F04F22
:201DC000204B85B04FF0000804461E2093F800A093F801B09D78B3F80490DF881E7ACDF815
:201DE0000480ADF80C8018F019FC18B117B1B9460125C246144A92F88635D9070AD492F868
:201E00008B253AB9012E1BD0022E03D113F0020F08BF01258DF80C608DF804A08DF805B0AC
:201E20008DF80650ADF80890ADF80A7001AB03CB1B88206020466160238105B0BDE8F08F2A
:201E40003546E7E7646D002098CF0020144B30B4D3F8B04514B300220F2583F8B615090A48
:201E600083F8B50583F8B715C3F8B825C3F8BC25C3F8C02583F8B45503F2B450012110F86B
:201E8000015F01312A440E29D2B2F8D183F8C2252046044930BC102236F03CB930BC7047CD
:201EA00098CF00204CD50020034B002183F8C415C3F8C815CAE700BF98CF002013B50446F6
:201EC0002620019118F0AAFB019920B9204602B0BDE81040BAE702B010BD2DE9F743B74C8A
:201EE000D4F8B0350D464BB14FF0020800264FF00109D4F8B00536F03DF958B90027A37FF3
:201F0000042B00F25781DFE813F08F00E400F7003D014601D4F8B00536F024F9D4F8C83582
:201F20005A1C2344C4F8C82583F8CC0594F8C435012B0AD0022B11D0002B70D10F280CBFC8
:201F400084F8C495C4F8C835D3E7A0F17203012B01D9762863D184F8C485CAE7102AC8D112
:201F600097490023012211F8010F013203440E2ADBB2F8D194F8DA2584F8C4659A42C4F852
:201F8000C865B6D194F8DB35002BB2D194F8CD75732F37D0762F0DD0722FAAD194F8CF25AE
:201FA00094F8CE3553EA0223A3D0E360B4F8D0352361A4E794F8CF2594F8CE3553EA022349
:201FC00097D094F8D11594F8D02594F8D505236242EA012294F8D215E17794F8D31584F8B2
:201FE000DE1594F8D415A4F8DC2541EA0021A4F8E015616901B96361A38C002B7FF47FAFBC
:020000040801F1
:20200000A2847CE794F8D32594F8D23543EA02231AB2002B3FF46DAFA4F8E2256FE784F813
:20202000C465C4F8C86564E7722F44D10123A3770022644B1B78402B2FD1634E94F8DEC5A0
:20204000A08CA37FB4F8DCE5338005024FEA0C33217F778005F4706503F440532B434FEAFD
:202060000E1543EA8133EDB22B43276A65691BB2BD4214BF0825002513432B43704514BFB3
:20208000042000201843514B614514BF0221002193F8CC30F3800143B180636F1BB1A36A2E
:2020A000002B40F09D804A494A481F2203B0BDE8F04356F056B8D4F8E435474AEB1A934213
:2020C00001DC0022B5E77220FFF7EEFEC4F8E455F7E7762F03D10223A3770022A9E7D4F8E8
:2020E000E4353D4AEB1A9342EBDD7620FFF7DCFEC4F8E45500229CE7344ED4F8E43596F8A9
:20210000CC20EB1A82B3344A934230DDE27FD2071BD46169226A91420ED089B24620FFF772
:20212000CDFE96F8CC30C4F8E455013B86F8CC300423A37701227CE7A18CB4F8DC258A4232
:2021400003D05020FFF7BAFEEBE7217F94F8DE258A4206D0B1FA81F149094920FFF7AEFE71
:20216000DFE7142286F8CC201C4A9342BDDC762FA7D17320FFF798FE0323A377C4F8E455B4
:20218000002256E7732F9CD0D4F8E415124B691A9942A0DC95E7D4F8E4350F4AEB1A934242
:2021A0008FDD7620FFF780FE0223A377C4F8E45500223EE70023A3771A463AE798CF0020E9
:2021C00064D500201C43002020430020F404002017FF0608D90500203F0D03003F420F008B
:2021E000334DD4F8E8652A2385F8E5300DF1020220230DF10101304685F8E63011F0D7F849
:2022000030B19DF801109DF8027051EA070339D1552385F8E730462385F8E830202301A9EA
:20222000304685F8E93011F0BCF80346214813B1BDF804209ABB204949F024FBB4F8E07577
:202240001E4D87B30DF10301304611F0ADF850B39DF803100DF10602304611F011F810B3C7
:20226000BDF8062016493B46BA420CBF20222A22284649F007FBB4F8E235A4F8EC3503B072
:20228000BDE8F083304611F077F8394685F8E700304611F05DF8037885F8E830BEE709498A
:2022A00049F0F0FACAE70849284649F0EBFAE2E7F4040020DE05002039FF0608E20500203C
:2022C00031FF0608823E070838FF060838B50B680E4D5A1C0A6005221A700B6895F8CE2072
:2022E0000C46591C21601A70236895F8D120591C21601A70B5F8D410204648F033F923689D
:2023000095F8D620591C21601A7038BDF40400202DE9F0472DED028BFFF7B8FAC8B31E4B2D
:2023200093F9CE00012834DD93F804411B4F9FED1C8A15468E1E02EB44084FF03209454559
:2023400004D1BDEC028B2046BDE8F08737F802AB26F802AF07EE90AAF8EEE70AB2EE040A91
:2023600060EE880A54F096FCBCEEC00ABAF10E0F10EE103A9BB209D91933B3FBF9F39BB2C1
:2023800003EB830303EB83035B009BB225F8023BD5E70024D5E700BFF404002086D5002065
:2023A000CDCCCC3D38B50D46FFF770FA044638B10C4890F8D130DB0704D5B0F8D2002880EE
:2023C000204638BD084A90F9CF3092F83C2093FBF2F102FB11320132013100F5847010F0E3
:2023E00063FFECE7F404002098CF002038B5134C94F8413094F840209A4219D004EBC3035A
:202400000F49D3E911200023984212DC93780D4AC4F800065B081370FCF7A4F994F84130F5
:2024200006210133B3FBF1F201FB123384F8413038BDD55C01F8015B0133E5E798CF002080
:202440006E6D00209C6D00202DE9F04FA94B1B788BB08146002B40F0B580A74ED6F8E855EA
:20246000002D00F0AF80A54AD2F80C4104F0F021B1F1E02F6BD1C2F80C31D6F80426944253
:2024800065D004930593ADF818309D4BC6F804469A881F78ADF8142093F801C01A7A93F8FE
:2024A00002A08DF810700DF110088DF811C08DF812A08DF8182098E807000DF11C0EAEE8D0
:2024C00003009049AEF80020C4F34252895CC4F303428F4202F101021F4601D1944508D07F
:2024E00028468DF81C108DF81D2010F0DDFEADF82000284611F029F9032804F0070B33D096
:20250000042835D000239A4501A9284618BF8DF81E3010F043FF48B1019BC4F3001103F034
:2025200001038B4202D0284610F0E6FF0A2207A9404655F0B0FD50B19DF81E30BDF81C207C
:20254000BB703A80BDF82030BB8048F021FE96F808A6DFF8ACB104AF96F80836032B7BD88F
:20256000DFE803F00A3376A3674B13F80B30CAE7664B13F80B30C6E73946284610F014FFFE
:20258000044658B107A8FFF719FC9DF81E109DF810308B4260D0284611F03AF896F808362C
:2025A000013303F0030386F808360CB99A45D3D196F88635DB0700D524B12B6849461B6870
:2025C000284698470BB0BDE8F08F01A8FFF7F6FB96F886859DF8044008F00108ECB1B8F186
:2025E000000F39D13A460DF10301284610F0DFFE044688B307A8FFF7E1FB9DF81C109DF899
:2026000003309DF81D208B4203D19DF81030934222D0284611F006F8C0E7B8F1000FBDD11E
:202620003946284610F0BDFE0446A8B107A8FFF7C5FBBDF82010BDF810308B420CD086F8E9
:20264000098686F80A862B6828469B699847A5E796F88635D80701D500249FE707A92846A7
:2026600010F09CFE04460028F6D01E2017F0D6FF96F80B3683428046EED086F80B0660B1B6
:20268000BBF80630002BE7D1079BD907E4D40121284610F031FF444680E7079BDA07DBD550
:2026A0000146284610F028FF78E73846FFF786FB97E8070007AB03C31A809DF810309BB131
:2026C0000DF11D0207A9284610F071FE0DF11E01284610F069FE0A2207A9384655F0DBFCE8
:2026E000041E18BF012459E708A9284610F059FEECE700BF1E6E002098CF0020F404002029
:20270000646D0020780107086C01070860010708024B0146D3F80C0635F030BD98CF00204A
:202720002DE9F041FD2984B0044669D0F02949D0EF2900F0BD804AB10346861803AD00204C
:2027400003F8010B9E4205F8010BF9D1B74B0B2003F1090501E013F8010F814255D0AB42BF
:20276000F9D14B1E152B21D8DFE813F0C500D000DA00E700EE00F4001600040100012000AF
:2027800020002301230123011001100110010001200020001B01AD00A54D95F88635DE0751
:2027A00000F16981B5F86036ADF80C303AB1224403AB13F8011B04F8011BA242F9D104B07A
:2027C000BDE8F0819B4F03214FF00508B844002501370CE0FFF738FA064660193246FFF7E9
:2027E0009FFF70194745C5B2E9D017F8011B412981F08003084601D0042BEBD80426ECE75F
:202800008D4F0B214FF00408E0E7894BD3F8E00680060CD4002AD2D0224403AB13F8011BAC
:2028200004F8011B9442F9D104B0BDE8F08193F81006870741D5814D287D052834BF022616
:202840000326142916D97C39C8B20628E2D80629E0D801A050F821F0212A0108212A010883
:202860000B2A010815280108052A0108FF290108F92901080929CDD90A390A29CAD801A7A8
:2028800057F821F0E7290108592A01081528010815280108152801081528010815280108D5
:2028A0001528010815280108DF290108212A0108634F0C214FF0060888E7604B0B29187D18
:2028C000A8D10126C9E05A4BB3F87C16CD055ABFCB4303F00103032311F0440F18BF042365
:2028E00011F0020F18BF072311F4806F18BF0923ADF80C305AE74E4BB3F8403603EB83037E
:202900005B0003F5C873ADF80C304FE74D4BD3ED037AFDEEE77A17EE903AADF80C3045E715
:20292000434B93F81F16002900F09C8001922CF049F8019AADF80C0038E701922CF042F8D0
:20294000019AADF80C0031E7394BD3F87036ADF80C302BE7364BB3F86016002900F085806B
:2029600001922CF03BF8019A80B2E3E7304BB3F8DE3619E72E4B3449B3F9DC3681FB030170
:20298000DB17C3EBA103ADF80C300FE7284B03EB4101B1F8BA3603EB83035B00ADF80C3030
:2029A00004E7234B93F8863503F00103ADF80C30FCE6264BDFED266AD3ED007A0C39C9B2F7
:2029C00003EB810393ED127A67EEA67A67EE877AFDEEE77A17EE903AADF80C30E6E6EB8972
:2029E000ADF80C3016E72B8A03EB830303EB83039B00ADF80C300DE7AB6803930AE76B687F
:202A0000039307E72B68039304E7EB89114903EBC3039B00A1FB03135B09ADF80C30F9E62B
:202A2000B3F81236ADF80C30F4E600BF3C01070898CF00205001070858010708BC6800204A
:202A400048010708DCD500206766666618D6002000007A441F85EB51F6B28DF80C608DF8EA
:202A60000D00D7E6B3F8380664E7D3F8780680F3100080B25EE705F24465019222F046F991
:202A8000D5ED037A019AFCEEE77A17EE903A9BB200287FF489AE0349096811F0100F18BF6F
:202AA000002381E64C68002070B5214D95F8E436EA181C4692F8E8268AB11E4E09225C1C38
:202AC000A6FB04135B0803EBC303E31AE918DCB291F8E81609B1013AF1D185F8E44602684C
:202AE0001549561C06600C2616700268561C0660002616700268561C066003EB430603EB93
:202B00008603147019440D2247F0C0FC95F8E416084B4A1CA3FB02035B08294403EBC303C2
:202B20000120D31A81F8E80685F8E43670BD00BF98CF0020398EE3388CD600202DE9F04F5D
:202B4000C31D85B0544C03F4FC7300AFADEB030DD4F86C3704F27C7B0DEB00025B450646C1
:202B60008A46FA60E9462FD094F8BC1894F8BDC8D4F8705701F00F0040EA4C1001310DF143
:202B800001088DF8000084F8BC18C7F8088007F10800ED1AA2EB0808A845194644DD2A468F
:202BA00047F074FCD4F86C27B968C4F86CB72A44A1EB09014846C4F87027C9B2D047002078
:202BC0001437BD46BDE8F08F94F8BCC894F8BD08B4F976570CF00F0141EA401141F01001DE
:202BE000002DC9B2D4F87057B8BF41F080010CF1010C012884F8BCC889F80010A5EB0B080A
:202C000022D1B8F1FE0F3ADDFF2394F8742789F8013007F1080009F103031FFA88F178608F
:202C200089F80220BB6020E0424647F02FFCD4F86C27424448463146C4F86C27D04701207B
:202C40001437BD46BDE8F08F94F87837B4F8741789F8013007F1080009F102037860BB60EC
:202C600047F080FC78681FFA88F147F07BFCD7E90282D4F87057D4F86C37786889E794F85F
:202C8000741789F8018009F1030889F80210C7F8088007F108007CE798CF002001297FD95C
:202CA000F0B50378654CC3F34115032D83B084F8BD5803F00F0700F0848013F010031646D4
:202CC00006D0012D6ED0052912D8002003B0F0BD94F89029002AF8D094F89129013202F078
:202CE0000F02BA4255D0184684F8903903B0F0BD437884F88C394388A4F888398588431813
:202D0000811DC02D7ED84E4AC4F8802915444FF0000C0120C4F88459A4F88AC984F8900973
:202D2000AA1A5B1A934284F8917966DB454D002A5CD1B4F98839FA2B53D0414A4249D4F83D
:202D40008039D1F81001C4F880292946151FA2F5A276C4F87057C4F884390025A2F5AA7255
:202D600001ABC4F86C6784F89059C4F8745701952EF03EFF013058D0019B0BB1002098478B
:202D8000D4F86C37C4F870370120C4F86C6703B0F0BD4318D4F88459D4F88029411CBFE7D5
:202DA00000207047022990D045788378A4F88839FF2D1FD1042988D94318B0F80350411D3E
:202DC0009FE70023214984F87C3704F27C7204F27D73C4F87417C4F86C27C4F870370120CD
:202DE00074E7002EA9D005233370A6E7284647F04DFB9EE74318C11C83E712481A4647F074
:202E000045FB62E7124BB4F88809C4F86C37032101334FF6F672A4F87407C4F8703784F835
:202E20007C17A4F87627012050E7D4F86C370222591CC4F86C171A709EE700BF98CF0020D2
:202E400058D8002018D90020F40400200000F6FF14D700202DE9F041684ED6F8E87584B09D
:202E6000044638460D4610F070FC86F8920957B10DF1090202A9384610F099FA002840F08D
:202E80008E8096F892090023ADF808308DF80A301A46431EDBB20021FF20FD2B8DF80C20D5
:202EA000ADF80E108DF80B0003D9002004B0BDE8F0819DF80830042B00F09680052B00F0D7
:202EC0009980032B00F09880022B00F08C80012B08BF042100F088809DF809309DF80A10ED
:202EE000D6F8E805013B0DF10E028DF8093010F0C7F996F89239032B73D0042B0CD1404AEF
:202F00009DF80A000121002301E012F8011F81426DD20133082BF8D1D6F89429029B394FE0
:202F20009A420DF108084FD023680D22591C21601A7023680022591C21601A7023689DF801
:202F40000820591C21601A7023689DF80920591C21601A7023689DF80C20591C21601A7034
:202F600023689DF80A20591C21601A70BDF80E10204647F0F7FA23689DF80B20591C2160E5
:202F800020461A700721FAF78DFE98E8030087E803000120C6F89C5904B0BDE8F08101A960
:202FA000384610F0FBF900283FF46BAF38460DF10A0110F0F9F900283FF463AF019B96F81A
:202FC000920903F0010264E77A68D8F804309A42AAD1D6F89C390C4AEB1A93427FF665AF7C
:202FE000A2E70A4A8CE703218DF8081074E78DF80A3091E70121F7E70221F5E798CF0020A8
:20300000600107082CD9002080841E006C0107082DE9F0412A4C2B4AD4F87036B4F8A07914
:20302000B4F8786682FB0352DB17C3EBA2031FFA83F8474582B00D4603D1B4F8A239B342FA
:2030400033D002680190511C34230160137002680023511C01601370414647F083FA019818
:20306000314647F07FFA019847F6FF7147F07AFA019847F6FF7147F075FA019847F6FF7106
:2030800047F070FA019847F6FF7147F06BFA01980221FAF707FE0120A4F8A089A4F8A2696E
:2030A000C4F8A45902B0BDE8F081D4F8A439064ACB1A9342C5D8002002B0BDE8F08100BF98
:2030C00098CF00206766666680841E00026810B57F21541C0460117002680024511C01602E
:2030E0000E211470FAF7DEFD012010BD2DE9F04FC24B1B68804613F0800083B000F0718120
:20310000BF4B93F8100610F0020000F06A81DFF810B39BF81430052B40F26881DBF8003068
:20312000B84D0093002BB8BF5B42A5FB0342B648B649920D00FB0233C3EB03139B0085FB28
:20314000034502EB8202DC1702EB8202C4EBA55400FB043304EB8204A4B281FB0321DB171B
:20316000C3EBA111BCB10025A94F2E46A7FB0432D20802EB8203A4EB4303E8B2A4469BB227
:2031800080008340BCF1090F94B246EA030605F10105EBD8340489B2B9B100259C4F2E4688
:2031A000A7FB0132D20802EB8203A1EB4303E8B28C469BB280008340BCF1090F91B246EAE8
:2031C000030605F10105EBD83443DBF804E08D4D8D4E8E498EEAEE70A0EBEE70A5FB0032DC
:2031E000920D06FB0200C0EB0010830085FB035002EB8202DD1702EB8202C5EBA05506FBA0
:20320000053305EB8205ADB281FB0321DB17C3EBA111C5B10020DFF8F8C10646ACFB05325E
:20322000D20802EB8203A5EB4303C7B2A9469BB2BF00BB40B9F1090F95B246EA030600F1CA
:203240000100EBD8350489B2C1B10020DFF8C0C10646ACFB0132D20802EB8203A1EB430308
:20326000C7B289469BB2BF00BB40B9F1090F91B246EA030600F10100EBD83543DBF8083089
:20328000634A0193002B1846B8BF5842A2FB0030604E6149030AA6FB0363DB0901FB03F146
:2032A000C1EBD00189B2B9B1002691463746A9FB0132D20802EB8203A1EB4303F0B28C4609
:2032C0009BB280008340BCF1090F91B247EA030706F10106EBD8B9B2BBF81070DFB1002606
:2032E000DFF82CA1B446AAFB0732D20802EB8203A7EB43035FFA86F938469BB24FEA8909C0
:2033000003FA09F3092897B24CEA030C06F10106E9D81FFA8CF7BBF812303D4AA2FB030678
:20332000F608632E28BF6326092B63D9002093468146ABFB0632D20802EB8203A6EB43035D
:203340005FFA80FAB4469BB24FEA8A0A03FA0AF3BCF1090F96B249EA030900F10100E8D88E
:203360005FFA89F9009B019A002BCCBF392338231616BEF1000F26F07F0635DD274A334351
:20338000964543F00206C8BF43F00606D8F800301622581CC8F800001A70D8F80030002239
:2033A000581CC8F800001A70404647F0DBF82146404647F0BFF82946404647F0BBF840467F
:2033C000394647F0CFF8D8F800305A1CC8F8002083F80090D8F800305A1CC8F80020012098
:2033E0001E7003B0BDE8F08F1E43CFE7002003B0BDE8F08F4FF00009B4E700BF4C680020E4
:2034000098CF00206BCA5F6B806967FFD34D6210CDCCCCCCC55A7C0AA0860100FFC99A3BAB
:20342000BC6800202DE9F047AB4B1B68064613F0800084B000F09E80A84B93F8100610F0DD
:20344000020000F09780A64F397D052940F29780632900F292800024DFF898C289B22546B6
:20346000ACFB0132D20802EB8203A1EB4303E0B28E469BB280008340BEF1090F91B245EA25
:20348000030504F10104EBD8EDB2BB68954A82FB0312D917C1EB623189B2002900F0188118
:2034A0004FF0000CDFF84CE26446AEFB0132D20802EB8203A1EB43035FFA8CF088469BB228
:2034C00080008340B8F1090F91B244EA03040CF1010CEAD8E4B2FB8983494FF4F36707FB1F
:2034E00003F7A1FB0737C7F38F1742F20F739F4249D8CFB10020DFF8FCE18446AEFB0732E0
:20350000D20802EB8203A7EB4303C1B2B8469BB289008B40B8F1090F97B24CEA030C00F135
:203520000100EBD81FFA8CF7704BD3E9002313433ED14FF0FF3833681722591C31601A7052
:2035400033680022581C306039461A70304647F009F84146304646F0EDFF33685A1C326031
:203560001D7033685A1C326030461C700621FAF799FB012004B0BDE8F087992585E7002032
:2035800004B0BDE8F0870021DFF868C10F46ACFB0302D20802EB8200A3EB40039BB28B4007
:2035A0000431102947EA030793B2F0D1BFB2BBE701A847F007FC9DF80810002900F08A8096
:2035C0004FF0000CDFF82CE1E046AEFB0132D20802EB8203A1EB43035FFA8CF089469BB2AB
:2035E00080008340B9F1090F91B248EA03080CF1010CEAD84FEA08289DF80910E1B10020B1
:20360000DFF8F0E08446AEFB0132D20802EB8203A1EB43035FFA80F98A469BB24FEA890985
:2036200003FA09F3BAF1090F91B24CEA030C00F10100E8D848EA0C089DF80A104FEA082836
:20364000E1B10020DFF8ACE08446AEFB0132D20802EB8203A1EB43035FFA80F98A469BB2A2
:203660004FEA890903FA09F3BAF1090F91B24CEA030C00F10100E8D848EA0C08BDF80C3052
:203680001B49632BA1FB03214FEA08184FEA51117FF651AF0020DFF85CE08446AEFB013236
:2036A000D20802EB8203A1EB43035FFA80F98A469BB24FEA890903FA09F3BAF1090F91B233
:2036C0004CEA030C00F10100E8D848EA0C0832E70C4600E788468FE74C68002098CF0020BC
:2036E000BC68002089B5F814D34D621040D900201F85EB51CDCCCCCC08B5A0F10103B3FA61
:2037000083F302284FEA531301D0184608BD0F2020F00AF830B9064B93F8863503F00103BE
:20372000184608BDBDE808400F2016F077BF00BF98CF0020014B1B681B6A1847F05C0020A9
:20374000024B186808B1836918477047F05C0020024B186808B1436918477047F05C0020C1
:2037600010B5074C606D40B13AF0B6F894F8513013B180F00100C0B210BD012010BD00BF6D
:20378000B01C002030B40A490A480A78531CDBB20525042B00EBC20400F8325008BF0023C8
:2037A0004FF404520B7062604FF0FF3030BC7047C86D0020CC6D0020037870B4FBB10446DF
:2037C000C0F10106A31914F8015FDBB2002DF9D101335B00DCB2032513800C704D700478F8
:2037E0005CB1022300255A1CD2B2CC548D5410F8014F0233DBB2002CF5D170BC7047022462
:203800002346E8E70B0617D401EB810300EBC30310B400EB81000124002283F8764383F82D
:20382000741383F87523426D5DF8044B136843F4001300201360704701F07F0101EB8103AB
:2038400000EBC303012200EB810083F81C1183F81E2183F81D2182691368002B01DA43F06E
:20386000804343F4001313600020704770B501F07F0505EB850400EBC404282101FB0501E0
:203880000126C4F830310023C4E94A2284F81C5184F81D61C4F8343101F58E711DB9FDF7E5
:2038A00023FE002070BDFDF793FE002070BD00BF2249F8B5D1F8B0390F2B04D05A1CC1F802
:2038C000B0290020F8BD1E4C25780023C1F8B039002DF6D11B4E1C4B3268B2F5006F17D013
:2038E0001B689A4227D017D9C2F50063402B15D9403B02F14005C1F8B4390123237035606A
:2039000092B2402311490A448121FFF7AFFFD8E71B6835607BB12A469B1AE7E74FF00005D8
:2039200002EB0307C1F8B4590CBF02210121376092B22170E6E700232370C2E798CF00209B
:20394000242600200C2600201026002028260020AEE700BFF8B51D4C2378012B03D0022BB6
:2039600009D00020F8BD01461948D0F8B43953B923700020F8BD00231A468121FFF776FF38
:2039800000232370F5E7402B11D9124C2268403B02F14005C0F8B439256092B240230E4C7A
:2039A000084622448121FFF761FF0020F8BD094D2A684FF0000603EB0207C0F8B46908BFC6
:2039C00002202F6092B208BF2070E8E72426002098CF00200C2600202826002038B51346D5
:2039E00002250A46C0E94E3380F811510021FFF73DFF002038BD00BF10B50C7814F0600474
:203A000013D0202C0AD14B78023B092B18D8DFE803F01B21171717171717272E2249012215
:203A2000FFF7DCFF0024204610BD4B78062B24D00A2BF3D01D4B8A78C3F8C029204610BD3D
:203A4000FAF7C6FE0224EEE719490122FFF7C6FF0024E8E717490122FFF7C0FF0024E2E75E
:203A60004B88124A1B0AC2F8BC390024DBE70F4B8A78C3F8B8290024D5E74B881B0A222B40
:203A80000CD0212B04D021462246FFF7A7FFCAE7CA880949092A28BF0922F6E7CA880749A6
:203AA000362A28BF3622F0E758D9002098CF002054D9002050D9002052060020080600207C
:203AC00038B501EB810400EBC4040D46002184F87453C4F88C1384F87513C4F88833C4F88C
:203AE0008023C3782821012B01FB050108BFEDB201F55D7108BFC4F884231DB9FDF7F4FC63
:203B0000002038BDFDF764FD002038BD144B9A6870B5044662B1134A1B7B92F8C4592B433B
:203B200016D081212046FFF76DFE022D09D070BD0C4B93F8C45981212046FFF763FE022D74
:203B4000F5D12046064ABDE870401F230121B7E70121FFF757FE20468121BDE8704051E691
:203B6000A86D002098CF002070B5094A094D1173094B13600021044629700D238121FFF7A4
:203B800075FE2046054ABDE870401F23012197E7086E0020FC6D002055534253A86D002035
:203BA00010B5064B597B0446FAF720FE002800DB10BD20460121BDE81040D5E7A86D002084
:203BC0002DE9F041314D2C7834B1012C01D1FFF7E7FF0020BDE8F0812D4FDFF8D080B0F83B
:203BE000B4337A68C8F804201F2BBA68C8F80820064606D1274B3A689A4202D1797B0129C0
:203C00001AD9254A25491378052401F8334001EBC3000133DBB2042B08BF00234FF4005197
:203C200013701F4B41600222304683F8C429FFF76DFF0020BDE8F081BB7B013B0F2BE0D8F8
:203C4000FAF7D4FD002819DB2B78013B022BC0D9144B1988B1B1BB68D8F8082088F80C4098
:203C60008B4228BF0B46D11A0424C8F808100E4A2C7030468121FFF7F9FDAAE73046FFF75F
:203C800045FFA6E73046FFF76FFFA2E7FC6D0020A86D002055534243C86D0020CC6D002057
:203CA00098CF0020F06D002094900020086E002008B5084B1B78022B07D0033B012B02D83B
:203CC0000021FFF751FF002008BDFFF769FF002008BD00BFFC6D002010B501EB8101084A88
:203CE00000EBC1010446B1F88C131046F4F7FEFA034A204640230121FFF7E2FE002010BD51
:203D000060D90020E8E700BF70B50A7812F060050C46064611D0202D16D1CD88D5B1130607
:203D20002AD52A461F496078F4F782FBE2881D493046FFF753FE00250AE04B780A2B16D0F2
:203D40000B2B0ED0062B03D13046FAF741FD0225284670BD022260781144F4F769FB2846D5
:203D600070BD8B78D3B9104BC3F8085AF0E70F490122FFF733FEEBE70D4964780A4AC1F885
:203D8000C8400321C0E9E45542F8045B2B4680F811110021FFF794FE0025D9E7FAF718FDDD
:203DA000D6E700BF9CCF002098CF0020A0D90020F40400200B7803F00303012B03D0022B1C
:203DC00004D0002070478B881BB915E68B88832BFBD099E710B50223044640228121FDF71E
:203DE000FFFA2046022340220121FDF7F9FA8221204603230822FDF7F3FA064B02229A800B
:203E0000F4F766FB044A204640230121FFF758FE002010BDB001002060D9002038B50922A2
:203E20000D46044603238321FDF7DAFA29462046FFF7D0FF002038BD82B000230168019352
:203E40000B6901930E4B03E00A690192013B13D0019A002AF8DA019A094B42F001020192AB
:203E6000019A0A610A69019203E00A690192013B02D0019AD207F8D4002002B0704700BFB7
:203E8000400D0300436D064A1A61C278012A06D100F2CC5058614FF0802219681A607047C1
:203EA0001800086010B5002304220446194680F811211A46FFF7DAFC2046FFF7E3FF002097
:203EC00010BD00BF10B5044629B990F81131032B0DD0002010BDD0F8E4359B69002BF8D0CB
:203EE00090F81221032AF4D19847002010BDD0F89013D0F87C33994214D9C078D4F88023F8
:203F00000128A1EB030104BFD218C4F880238B4228BF0B46C4F890139BB220460021FFF7AE
:203F2000CFFDD6E7D0F8E4351B691BB190F81221032A03D02046FFF7B5FFCAE79847F9E78C
:203F4000F0B5012190F8D17590F8D36590F8CFC590F8CE5590F8D03590F8D22580F811119F
:203F600090F8CC1585B005EB0C2503EB072302EB062201F01F06AFB292B290F8CD558DF86B
:203F800008109BB2012E0446ADF80A70ADF80C30ADF80E20C0F840218DF8095017D0022E62
:203FA0001FD036B101F08001FFF72CFC002005B0F0BD092D0FD8DFE815F0BF00AC000E00B7
:203FC000D5000E00EA0085000E007700540090F81221032A2FD02046FAF7FAFB002005B0AE
:203FE000F0BD01F060012029DAB234D0012D00F02081032D00F00681002DD7D190F8121103
:020000040801F1
:20400000022900F0DF800329E5D11B0600F14B8102EB820200EBC20393F87633002B00F0F6
:204020004D81BF4B0122C3F81C2ABE4920460222FFF7D4FCBAE7DAB2012ACCD8D0F8E43550
:2040400002A99B689847BDF80E30002BAED12046FFF728FFAAE7D0F8E43502A99B689847B4
:20406000A4E7F9B2AE4D012985F80C1AB3D890F81231022B00F02781032BACD1002900F063
:20408000868190F810110129E1D0D0F8E4355B68984795F80C1A84F810112046FDF70EF961
:2040A0002046FFF7FFFE81E7012A94D190F81231022B00F01781032B8DD100F58871FFF7BF
:2040C0008DFC73E73D0A022DADF8062000F05081032D00F00B81012D7FF47DAFD0F8EC3599
:2040E00080781B680DF106019847BDF80620002A3FF45CAFBDF80E30002B3FF457AF9A42EB
:2041000028BF1A4601462046ADF80620FFF766FC4CE790F81231023B012B3FF65CAF012FB1
:204120007FF444AFD0F8E43500229B68C0F8182102A9204698478AE790F81231023B012B8D
:204140003FF649AF764BD0F818210021C3F8141A12B10222C3F8142A734920460222FFF74A
:204160003DFC23E7012F00F09880022F7FF41EAF13F0FF0F7FF41AAF02691B0A023B52687F
:20418000032B00F21D81DFE803F0393531241A437FF421AF90F81231032B3FF41CAF0369E1
:2041A00007F07F0580F81451196867F30A120A431A60FFF777FE002D00F0E580022384F85B
:2041C0001231F3E651063FF4F1AE1146FFF71AFBECE6052363F30612514B012184F816116F
:2041E0002046C3F8182AFFF75DFEDFE6042363F30612F1E7032363F30612EDE7022363F3F6
:204200000612E9E790F81231022BDBD0032B7FF4E2AE27B9550602D01146FFF7F3FAD4F8CF
:20422000E43502A99B68204698472046FFF73AFEBCE690F812110229C4D003297FF4CBAEBA
:20424000002F7FF4B3AE12F07F013FF400AF180600F1A78002EB820304EBC30304EB81002A
:2042600083F8767383F8741383F87573282303FB0243416D03F55D73DA780B68023A6FF30E
:204280005553012AD4F8E42598BF43F080530B602046936802A99847D9E6D0F8E435C0F86B
:2042A00018719B6844E702F07F0202EB820200EBC20393F81E31002B7FF4B3AE184B002255
:2042C000C3F81C2AB1E600293FF4C1AE0121032380F8101180F81231FCF7F0FF2046FFF7A1
:2042E000E1FD63E61149FFF779FB5FE6FDB2052D3FF671AEDFE805F0342C241C0B03D0F827
:20430000EC3580789B690DF106019847EDE6D0F8EC3580785B690DF106019847E5E600BFB6
:2043200098CF0020B4D90020ACD90020A8D90020D0F8EC3580781B690DF106019847D4E600
:20434000D0F8EC358078DB680DF106019847CCE6D0F8EC3580789B680DF106019847C4E631
:20436000D0F8EC3580785B680DF106019847BCE6D0F8E43580789B6A0DF10601984745709C
:20438000C4F8F005B1E6012384F812310EE60222D0F8E43580F8101180F812215B68984713
:2043A00055E6282202FB014304EB810083F81E7183F81C1183F81D51816903F58E735BE707
:2043C000012363F3061207E770B5044649B990F81131022B1BD094F81631012B0DD000200E
:2043E00070BDD0F8E4355B69002BF8D090F81221032AF4D19847002070BD2A4A2369D2F855
:20440000182A5A60002384F81631002070BDD0F83831D0F82451AB4217D9C278012AD0F8F5
:204420002821A3EB050308BF5219C0F8383108BFC0F828219BB20021FFF718FA00231A4689
:2044400019462046FFF73CFBC5E7D0F83C31B3FBF5F605FB163666B99D420AD8D0F840219B
:20446000934206D233463246FFF700FAC4F84061E4E7D4F8E435DB681BB194F81221032AA6
:204480000CD00023052284F8112119461A462046FFF716FB2046FFF7F5FC9CE72046984707
:2044A000EFE700BF98CF002082B000230193019A094B42F010020192C168019A0A610A698F
:2044C000019203E00A690192013B02D0019AD206F8D4002002B07047400D030082B00023E5
:2044E0000193019A0B4B42F020020192019A61F38A120192C168019A0A610A69019203E01A
:204500000A690192013B02D0019A9206F8D4002002B07047400D0300F8B50B7813F0600517
:204520000C4606461CD0202D17D14A78FE2A44D0FF2A3DD14A88002A56D1CD88002D53D1BE
:204540001B0651D43749384B0D70012183F8C419364A1F23FFF7B4FA00E000252846F8BD8D
:204560004B780A2B4BD00B2B44D0012BF6D191F904308988002B47DBFFF796FF21792A4F31
:204580003046FCF7C9FE0223217940223046FCF727FF97F8C439022B3BD094F90420002A9C
:2045A000DCDA012BDAD030460121FFF7DDFAD5E70225FAF70DF92846F8BD4D88A5B9CC8886
:2045C000012C11D11A060FD5194B1B689B6998471549C0B281F8200A30B1224601F52261C9
:2045E0003046FFF7FBF9B9E730460225FAF7F0F82846F8BD0C4B4A8883F8212AAEE70D4948
:204600000122FFF7EBF9A9E701F07F01FFF766FFB4E730468121FFF7F5F8002387F8C4390C
:204620009CE700BFFC6D002098CF0020A86D0020EC6D0020B9D9002038B50446FCF7A2FEFE
:204640002046022340228121FCF7CAFE2046022340220121FCF7C4FE0C4B0D491B680D4AC5
:2046600000250D701B6882F8C459284698472046FFF71AFF20460121FFF730FF064A204659
:204680001F230121FFF71CFA284638BDEC6D0020FC6D002098CF0020A86D0020012905D08A
:2046A00008B50321FFF71AFF002008BDFFF752B90B88F0B433BB028C4C880E898B88C988A2
:2046C00022F001021204120C0284058B028CADB225F0F30592B22B4322F00A0243EA06136B
:2046E00022439BB242F0010203830284038B23F00C031B041B0C0383038B9BB21943F0BC68
:2047000001837047042B048C2CD0082B4E888A880D89C98851D024F480542404240C0484B4
:20472000838B078C2C0344EA022440F6FF421A4045F6FF733B4043EA063322439BB292B200
:2047400043F4805382830384828B22F440621204120C8283838B9BB243EA01239BB2F0BC20
:204760008383704724F010042404240C4D880F898A88C9880484068B038C12029BB242EAF7
:20478000073423F0A00340F6FF42324043EA051322439BB292B243F0100302830384028B25
:2047A00022F440621204120C0283038B9BB243EA01239BB2F0BC0383704724F480742404F2
:2047C000240C0484848B038CA4B29BB224F0F30423F42063224343EA062342EA05129BB2F0
:2047E00043F4807392B282830384838B23F00C031B041B0C8383838B9BB21943F0BC8183DC
:20480000704700BF214A038890429BB212D002F5806290420ED0B0F1804F0BD0A2F580320E
:20482000904207D002F58062904203D002F58062904203D14A8823F070031343144A9042F4
:2048400018D002F58062904214D030B423F440730C894D6802F56C429BB2234390420C882B
:204860000380C56204850DD18B7A0386012330BC8382704703800B884A68C2620385012335
:2048800083827047034B9842EED0EFE700000140001000400004014000B583B009238DF831
:2048A0000730FCF74DFF8DF807009DF80730012BF7D09DF8070003B05DF804FB82B0064B11
:2048C000002201920193019B03EB80000190019B186802B0704700BF5028004082B0064B75
:2048E000002201920193019B03EB80000190019B196002B0704700BF502800400023C0E913
:204900000033C0E90233C0E90433C0E90633C0E90833C0E90A33C0E90C338363704700BFB6
:204920000B6870B4D1E90524CD682B431343D1E9072523431343D1E909422B43D1E90D65C3
:204940002343134304680B4A334322402B4313430360D1E90B3442690D6922F00702234340
:204960001343D1E9014243614560846070BCC260704700BF3F801CF002683649002310B458
:2049800022F00102212488420260036043608360C3600361446138D02F4B98422ED02F4BA8
:2049A00098423CD02E4B984240D02E4B984232D02D4B984241D02D4B984246D02C4B98423D
:2049C00017D02C4B98423CD02B4B984216D02B4B984224D02A4B984228D02A4B98421AD099
:2049E000294B984229D0294B98422ED0284B984208D14FF03D5243F8AC2C03E04FF4746221
:204A000043F8202C5DF8044B7047224B5DF8044B3D229A607047204A43F8642CF2E74FF442
:204A200074125DF8044B43F8382C70474FF074625DF8044B43F8502C7047184A43F87C2C8A
:204A4000E0E73D2243F8082CDCE7154A43F8942CD8E700BF106002402860024040600240C8
:204A6000586002407060024088600240A0600240B8600240106402402864024040640240FA
:204A8000586402407064024088640240A0640240B8640240006002403D000020400F0020C2
:204AA00000003D20024A536A23EA00005062704700380240024A136A23EA000010627047A1
:204AC00000380240484B98422ED0B0F1804F32D0464B984236D0464B98421ED0454B98424B
:204AE00037D0454B98423BD0444B98423FD0444B98424BD0434B984240D0434B98424CD042
:204B0000424B984251D0424B984256D0414B98425AD0414B98425ED07047404A136A43F06B
:204B2000040313620420C5E73C4A536A43F0010353620120B6E7394A136A43F00103136290
:204B40000120B7E7354A136A43F0020313620220B0E7324A136A43F0080313620820A9E7D0
:204B60002E4A136A43F0100313621020A2E72B4A136A43F02003136220209BE7274A536A1F
:204B800043F4803353624FF480308BE7234A536A43F002035362022084E7204A536A43F40F
:204BA000003353624FF400307CE71C4A536A43F4802353624FF4802074E7184A136A43F035
:204BC00040031362402075E7144A136A43F08003136280206EE7114A136A43F480731362EF
:204BE0004FF4807066E700BF000001400004004000080040000C00400010004000140040B9
:204C00000004014000400140004401400048014000180040001C0040002000400038024032
:204C2000224A936803F00C03042B10B421D0082B22D01F4B03601D4C1E4AA168C1F3031193
:204C4000114491F87011CB404360A168C1F38221114491F8701123FA01F18160A1685DF83A
:204C6000044BC1F342310A4492F87021D340C3607047114B0360DEE7546851685268630250
:204C8000C2F388124CBF0C4B094B01F03F01B3FBF1F303FB02F3054A5268C2F30142013225
:204CA0005200B3FBF2F30360C5E700BF003802400024F400F404002000127A002DE9F047BE
:204CC00000230F6801264FF0030C02E00133102B41D006FA03F232EA0704F7D1D0F800E0D7
:204CE0005C000CFA04F52EEA050EC0F800E091F80490D0F800A009FA04FE09F1FF394EEAA2
:204D00000A0EB9F1010FA846C0F800E06FEA050515D8D0F808E005EA0E0585604D79D0F8C6
:204D200008E0A54045EA0E058560456825EA020242608A7945689A4092B22A434260C26816
:204D400022EA0802C260CA79C568A24001332A43102BC260BDD1BDE8F0870B4B93F8862595
:204D6000D20703D5012283F8222A704793F8222A4AB9D3F8E83533B1044B1A7810445A7834
:204D8000187011445970704798CF0020646D002010B50E4C40F0080284F8842194F9CE2049
:204DA000022A06DD420704D583071CBF012384F8D63005210648FCF7D1FD062184F8850159
:204DC000BDE810400248FCF7B1BD00BFF40400207406002010B5FCF759FDA8B31B4C94F965
:204DE000CE30012B30DD59B3022B2DD094F8D6309BB971B180230521154884F88A31FCF7EE
:204E0000ADFD062184F88B01BDE810401048FCF78DBDBDE810400420BAE7002914BF002059
:204E2000042094F8D1301A0748BF40F002005B0701D411B108B940F00100BDE81040A7E7F9
:204E4000022BD3D10420ECE710BD00BFF40400207A060020F8B5224C04F5C677030A84F86C
:204E6000910105460621384684F89031FCF776FD94F8D13084F89201DB072AD4B4F8D220F3
:204E8000AA4226D1174DD4F88C31C5F8233AC3B285F8293A41F26F714FF6FF738A4218BF66
:204EA0000123134405F62326C3F307220621304685F8272A85F8283AFCF750FD072185F825
:204EC000290A3046FCF732FD052104F29310FCF72DFDBDE8F84004480721FCF727BD00BF44
:204EE000F404002098CF00208006002008B5FCF7CDFC48B1A1F59C53083BB3F57A7F03D2BD
:204F0000BDE808400846A5E708BD2DE9F0476B4E3368002B3AD06A4D6A4C05F1CE0730685F
:204F200033F028F9002833D1674B198809291D4609D95F8864227A43B2FBF1F2452A40F3DB
:204F4000A1811880588094F8613A012B00F0C581022B00F0E08133B95C480521FCF7E6FC2D
:204F6000012384F8613A5A4B1D685A4B1B78002B00F0DB81584B1B68EB1A782B40F2D581C7
:204F8000D4F80006F9F7EEFBC4F8645ABDE8F087306833F0E7F894F82A3A8046052BBED8BA
:204FA000DFE803F00309171D3745AA28B7D1012384F82A3AB3E7552803D1022384F82A3A2D
:204FC000ADE7414A938801339380002384F82A3AA5E7032384F82B0A84F82A3A9FE7132849
:204FE00084F82C0AC4F8440A07DD374AD3880133D380002384F82A3A91E718B9052384F8BE
:205000002A3A8CE70023C4F8483A042384F82A3A85E7D4F8483AE218013382F82D0AD4F8EC
:20502000442AC4F8483A93427FF479AFE6E7D4F8443A2A4803F1020A4FFA8AF1FCF78EFC8A
:20504000804594F82B9A40F01481262015F0E6FA204B48B100221A701B4A538801335380F3
:20506000002384F82A3A5AE71A784A4519D100221A7009F1FF33102B00F2F680DFE813F09C
:2050800030008E008E00DE008E00F400F400F4003000F400F400F400F400F400F400F400A0
:2050A0003000B9F1090F02D0B9F1110F01D1012ADDD0054A538901335381DAE7606D0020D7
:2050C000F404002098CF00208E6D0020870600202C2E00209C6D0020A06D0020C3D90020DD
:2050E000BAF1060F5ADDB9F1010F06D0B9F1090F0CBF4FF002094FF0030994F8300A94F8B5
:20510000311A94F82F2A94F92DEA94F92FCA94F82E3A85F8CE9041EA002109B2900785F84B
:20512000CFE085F8D1C0A5F8D21006D512F00C0F14BF0122002285F8D620B9F1030F13D110
:20514000BAF1090F2ADD94F9332A082AA8BF082222EAE27285F80421002043B29A4200F1F4
:20516000010059DC94F8323AD4F828A0002002469BB25245904657DB7C4B85F8D0001B7872
:20518000232B0BD109EB8903794A03EB83030CEB83031380A2F802E09180D08075497648C5
:2051A0000A2252F078FF10B1002384F8563A714B3A681A607A685A603A891A8194F8563A2C
:2051C0002BBB95F8D6306D4A002B14BF0223012384F8563A95F8D130117884F8581A13F044
:2051E00001031CBFB1FA81F35B09517884F8591AD8B29188927884F8570AA4F85A1A84F87F
:205200005C2A13B109B1A4F85E1A84F8600A0EF00FFF0EF00DFF1FE704EB4308234493F848
:20522000353AA8F8EE3598E704EB48080132B8F82C8052B2984508BF10469AE7BAF1040FB2
:20524000ACDD94F82D2A94F82E3A43EA022359041AB204D5C3F30D03A5F8D4309EE7002A84
:20526000F8DBA5F8D23099E7454A938901339381F2E619F0010F7FF4F3AE414A13890133E9
:205280001381EDE63F4BD3F89821B3F89C11012A1AD141F25632914203D14FF0FF32C3F89E
:2052A0009821D3F89821306802EB820202EB820201EB420189B2A3F89C1103681B699847B7
:2052C00000232B806B803EE60132EAD1B1F5965F04BF0122C3F89821E3E72A4D95F9CE6011
:2052E000002E3FF440AE022E11D14FF48040FFF7B1FD84F8616A95F9CE30012B7FF733AE50
:2053000095F8D130C3F3400385F8D6302BE6032384F8613AEFE71B4BB3F8D430002B3FF4EC
:2053200022AE032384F8613A1DE694F8402094F841309A4204D0FDF759F8C4F8645A25E6FA
:20534000D4F8643AEB1AB3F57A7FBFF41FAE0E4B1B68ED1A952D7FF619AE0C480521FCF76F
:20536000E5FABDE8F047FDF741B800BF1C43002020430020E4D90020C2050020646D00200F
:205380008E6D0020F4040020A06D002087060020104BD3F8E80510B5D8B10F4C217841B1B9
:2053A00062780DF081FFA38883421ABFA08001210021E2885AB141F288339342B8BF134662
:2053C0009A4204D0E380BDE8104045F0E1BE0029F9D110BD98CF0020646D002010B40144B0
:2053E0000446002014F8013B08225840430010F0800F08BF400083F0070314BFD8B2C0B214
:20540000013AF3D18C42EDD15DF8044B704700BF30B54FF4806085B02CF06AFA40B3154CD6
:2054200090F9040094F8683A134A002B18BF08234FF4E1310125CDE90153009100234FF4AB
:2054400080612CF0B6FAFF23E067003818BF012084F8F83484F8083584F8183584F8283503
:2054600084F8383584F8483584F8583584F8683505B030BD98CF0020151C0108374B1B68C0
:2054800013F000635CD02DE9F04F354B1F78B84251D3FF2856D1334B93F8DE30002B47D049
:2054A000DFF8D4A00022CAF86C2ACAF8702ACAF8742AAAF8782A002F4CD00AF59F63104685
:2054C000144611461546164603EB071BB946B3F802C09F8993F8008093F901E061443A4425
:2054E0004645D3E901C738BF464610337545B8BF75469B4509B212B264443844E7D191FB24
:20550000F9F192FBF9F28AF86C6A8AF86D5ACAF8704ACAF8740A144BAAF86E1A1B78114956
:20552000AAF8782A092B4FF0000281F8DE200CD00E48BDE8F08F0E4A02EB0010BDE8F08F6C
:20554000184670470020BDE8F08F0A4B9AF86C2ADA80EDE73A463946DDE700BF4C680020F1
:2055600038490020F40400201C43002004DA002090D400202043002098CF00200268F8B550
:205580003A4E3B4CB6F97C3A511C01607E2111700168054603EBC30384FB0302481CDC1766
:2055A000002328600B70FF20C4EB6204FFF766FF2034304BA4B200284DD01B78B0F90C1074
:2055C00023BB2D4BA1F57A729A4246D82B48B0FBF1F189B2284644F09FFF96F81F367BB16F
:2055E00029F0F0F90146284644F096FF2146284644F092FF28460821F8F754FB0120F8BDE6
:20560000B6F83816284644F087FFEFE71C4B1F78002FD6D01B48002300EB83020133928978
:20562000BB421144F8DB184B9FED186A93F8223007EE103A07EE901AB8EEC77AF8EE676A7B
:20564000C6EE077A67EEA67AFCEEE77A17EE901AB1FBF7F1B5E71B7813B94EF69C21B9E776
:20566000074B1F78002FF8D00146D3E798CF002067666666AD6300201783930300879303AC
:205680003849002018DA0020082F0020000048432DE9F8434A4C427894F8043B02F00F0503
:2056A000C3B9EDB92B46002184F8081BEB1AD9B20E290BD8234493F8201639B102F0F002F7
:2056C000802A4AD0902A5FD0A02A0DD000273846BDE8F8830021AB4284F8081BF6D8E5E76A
:2056E00084F8045B2B46DEE7412966D081F08003042B62D90846FCF7A7FA031D0246DBB2C4
:20570000304884F8083B65F05F0584F8095BFDF707F894F8087B002FD8D0BE1E16F0FF00FF
:2057200024D1FF25A946022756B1DFF89C80464418F8011BD4F82C0B32F020FD4645F7D1F3
:20574000D4F82C0B494632F019FDD4F82C0B294632F014FD3846BDE8F88365F07F05042738
:20576000022684F8095B84F8087B3046164A4FF6FF71104412F8015B491B904289B2F9D1A2
:205780005FFA81F90D0ACFE7412914D081F08003042B10D90846FCF757FA65F06F05062787
:2057A000042684F80B0B84F8095B84F80A1B84F8087B3046DAE70420EFE7082304229FE7A5
:2057C00098CF0020A2DA0020A0DA00200B4B93F85E2612B1B3F830264AB9B3F9DC36084AD0
:2057E000D81782FB0323C0EBA30000B27047D3F8780690FBF2F000B2704700BF98CF0020FB
:2058000067666666F8B5184CC6B205463146D4F8300B32F0B3FC94F8341BD4F8300BC5F332
:2058200007274E40394684F8346B32F0A7FC94F8341BD4F8300BC5F307464F40314684F8E4
:20584000347B32F09BFC94F8341BD4F8300B2D0E4E40294684F8346B32F090FC94F8341B22
:205860004D4084F8345BF8BD98CF002070B50C4DC6B231460446D5F8300B32F07FFC95F86B
:20588000341BD5F8300B240A4E40214685F8346B32F074FC95F8341B4C4085F8344B70BD4F
:2058A00098CF002038B50B4C002305462421D4F8300B84F8343B32F061FCD4F8300B54217D
:2058C00032F05CFCD4F8300B2946BDE8384032F055BC00BF98CF00202DE9F043DFF89493FB
:2058E0002DED028B99F8354B83B00E461546002C00F03982013C89F8354B9FEDD88AD84FE4
:20590000DFF874833378002B62D099F8354B002C5ED135B131F06AFF2B68C01A002880F2CE
:20592000028499F8364B002C40F0A68399F8370B062840F2D781CB4A92F8A53192F8A4110B
:20594000994200F00082D2F8A01199F838CB31F8134064440130013302F5D072A4B2C0B261
:20596000DBB2B4F5E06F89F8370B537100F0D18100F2AA80B4F5806F00F0F88264D9B4F5D5
:20598000A06F00F0CC823CD9B4F5A16F25D8601EC0B2FFF773FDC8B1B0F90C30B24AADF89A
:2059A000014092F82210D9F87C2503EB830303EB830349089B0093FBF1F31021CDF8033009
:2059C0008DF800106846904700233370002D99D103B0BDEC028BBDE8F083B4F5C06FF5D1B1
:2059E000B9F86036002B00F0548328F0F7FF10220024CDF8030006238DF800208DF80140AE
:205A00001FE2B4F5826F00F05082B4F5846F40F0358199F810369A07D8D5B9F81236CDF8C4
:205A200003301021202204238DF800108DF801208DF80230D9F87C356846002498473470D0
:205A4000002D7FF45FAFC3E7B4F5067FBED8B4F5007FC0F02C81A4F50073182BB6D801A225
:205A600052F823F0E15D0108CF5D0108CF5D0108CF5D0108CF5D0108CF5D0108CF5D010844
:205A8000CF5D0108CF5D0108CD590108CD590108CD590108CD590108CD590108CD59010882
:205AA000CD590108AB5D0108955D0108955D0108955D0108955D0108955D0108955D0108C4
:205AC000955D0108955D0108B4F5116F00F0E0815BD8B4F5026F00F0BF8121D9B4F5036FC4
:205AE00000F07282B4F5046F7FF470AFB9F9DC36D9F87C2503EB83035B001020CDF80330E7
:205B0000402108238DF800008DF801108DF802306846002490473470002D7FF4F3AE57E75B
:205B2000B4F5E46F00F07881B4F5006F76D199F8102691077FF54AAF13F0010F4B4B00F0BC
:205B400005835A6882EAE273A3EBE27303EB5303A7FB0313DB08002AACBF43F0004343F03A
:205B60004043102100240822CDF803308DF800108DF80140D9F87C358DF80220684698471A
:205B80003470002D7FF4BEAE22E745F230239C4200F0B1811DD945F240239C4200F02982B9
:205BA00045F250239C427FF411AFD9F87836CDF803301021502252238DF802308DF800104F
:205BC000D9F87C358DF80120684600249847347036E7B4F5376F00F031826FF437616318C3
:205BE000072B3FF6F3AEA4F17100C0B2FFF746FC00283FF4EBAE90F90130CDF80330102314
:205C00008DF80030ADF80140D9F87C356846984700233370002D7FF475AED9E6B4F5E26F98
:205C20007FF4D4AE124B93ED130AD3ED007A20EE270A002420EE080A50F050FF10230722CD
:205C4000CDF803008DF800308DF801308DF80220D9F87C3568469847347092E70000C84234
:205C60001F85EB51F4040020082F0020BC68002018D6002098CF0020C5B3A29140F20143DB
:205C80009C427FF4A3AEB9F97C3ACDF803301021012204238DF802308DF80010D9F87C35B9
:205CA0008DF801206846002498473470C8E6B4F5807F00F01481B4F5887F7FF487AEB9F904
:205CC000DE36CDF80330012210238DF800308DF801308DF80220D9F87C356846002498471D
:205CE0003470ADE60130CD4AC0B292F8AD1192F8AC318B4222D04B1CDBB24900D2F8A84155
:205D0000C74A645A89F8370BB4F5E06F53717FF42FAEC44B93ED120AD3ED007A20EE270AC1
:205D2000002420EE080A50F0D9FE10220723CDF803008DF800208DF8014082E0002182F87C
:205D4000AD110123DAE7B84999F8383B097882F8A5410133DBB201318B4289F8383B00F016
:205D600087810120C1E700283FF4C7AD0378303B012B3FF6C2AD013009F635320621FCF71C
:205D80008DFF99F8353B89F8360B002B3FF4B5AD3470B2E5A4F11100C0B2FFF76FFB002819
:205DA0003FF414AEB0F9023027E799F81F36002B40F0B081B9F83806CDF803001023022285
:205DC0008DF800308DF801308DF8022083E7601EC0B2FFF753FB00283FF4F8AD43680CE775
:205DE000D9F870369149D9F87C2581FB0301DB17C3EBA10300241021CDF8033002238DF825
:205E000000108DF801408DF80230684690473470002D7FF477ADDBE5824B93ED140AD3ED1D
:205E2000007A20EE270A002420EE080A50F056FE102320228DF80030CDF8030007238DF830
:205E400001208DF802306846D9F87C3598473470002D7FF457ADBBE599F810369B077FF586
:205E6000B5AD734AD9F87C359268CDF80320102220218DF8002008228DF801108DF8022020
:205E80006846002498473470002D7FF43BAD9FE528F098FD10230922CDF803008DF8003019
:205EA0008DF801308DF8022015E7D9F8E03613F0200440F0F1805F4B1B681B0640F13981A1
:205EC000102304228DF803408DF804408DF805408DF806408DF800308DF801304AE6D9F8D7
:205EE0003C3BCDF803301022002401238DF800208DF80140A5E7B9F9DA36CDF803301021D7
:205F0000302252238DF802308DF80010D9F87C358DF80120684600249847347090E5FF205D
:205F2000FFF7ACFA00283FF451ADB0F90C304249D9F87C2591F8221003EB830303EB8303E7
:205F40001020490800249B0093FBF1F305218DF80000CDF803308DF801408DF802106846E1
:205F600090473470002D7FF4CDAC31E599F8403B0133DAB2042A00F0D08042F2107389F805
:205F8000402B03FB02F3D9F8442B002A00F0C080023399F88625D207B9F87C2648BF04332E
:205FA000D40748BF0A33900748BF1433D10548BF2833540748BF6433500648BF03F57A637A
:205FC000102100240422CFE599F8103698077FF5FDAC174BD9F87C25D9894FF4F36303FB32
:205FE00001F3A7FB03135B091020CDF80330302187E5B9F9D836CDF80330102140225223EC
:020000040801F1
:206000008DF802308DF80010D9F87C358DF80120684600249847347012E500BFF4040020E9
:206020009C06002018D600203849002067666666BC6800204C680020082F0020FF20FFF7D2
:206040001DFA00283FF4C2AC90F90130CDF80330102170220B238DF802308DF80010D9F8A0
:206060007C358DF801206846002498473470E7E489F8384B012038E65C490620FCF75EFD4D
:20608000002389F8360B337003B0BDEC028BBDE8F083D9F87806AAE4554A99F81016538A67
:2060A000643BC3EB4370C3EBC00388FB03401844DB17C3EB20230933092BA8BF092323EA5A
:2060C000E37303EB830311F0020F03EB830314BF4FF47A7000209B00C90748BF00F5FA608F
:2060E000117DD9F87C259BB203440B44042010218DF80200CDF803308DF800108DF80110BE
:206100006846002490473470002D7FF4FBAB5FE401333EE728F056FC4EE6012389F8403B92
:2061200042F210732FE7347003B0BDEC028BBDE8F08399F81E36002B3FF448AC99F8483BA2
:20614000032B4ED8DFE803F043392A111A6882EAE273A3EBE27303EB5303A7FB0313DB0875
:20616000002AB8BF43F08043FBE4D9F8502B537A907AD17A03F1407303EB0023002203EB73
:20618000014389F8482B10220421CDF803308DF800208DF801208DF802104BE4D9F84C1B2F
:2061A0008A7D087C897A120402EB00220A44591C89F8481B02EB0363E5E7D9F84C1B4A7D67
:2061C000C87B497A120402EB00220A44EFE7D9F84C1B0A7D887B097A120402EB00220A44B8
:2061E000E5E75A1C89F8482B1B06CCE7B11C0108BC68002030B5A0F17D03012B044683B0DC
:206200000D46104608D9214631F0B8FF15B1288804442C8003B030BD7D21019231F0AEFFAC
:20622000019884F0200131F0A9FFEFE730B50F4B85B0D3F8542B00230446C51DADF80E30A1
:2062400014F8010B01920DF10E01FFF7D3FFA542019AF5D10DF10E0015F070FA019A9DF8CB
:206260000E000021FFF7C6FF05B030BD98CF0020044AD2F8583B43F4DF2343F48063C2F853
:20628000583B704798CF0020013070B5094EC4B203E045F0B9FB013448B9E5B2152D2146C8
:2062A0003046F6D9162D04BF034B93F85C5B284670BD00BFF0DA002098CF002000B1D7E7C9
:2062C000044AD2F8583B23F4DF2323F48063C2F8583B704798CF002070B5114C84B0054674
:2062E000D4F8600B0E462BF0C1FA94F8182694F81936003A18BF01220BB142F00802CDE9B6
:20630000016200234FF4964195F9000000911A4608212BF04EFBC4F8600B04B070BD00BF0A
:2063200098CF002010B5064C03E0D4F8600B31F019FFD4F8600B31F01DFF0028F5D110BD3D
:2063400098CF002010B50D4CD4F8643B1B791E3B012B0DD9D4F8600B01213830FFF7BCFFBC
:206360000023C4F8683B84F86C3BBDE81040D9E7D4F8600B012131F0EDFEF1E798CF0020FF
:2063800070B50A4E0546D6F880355E200C469847D6F8803528469847E0B2FBF7A3FCC4F359
:2063A0000720BDE87040FBF79DBC00BF98CF002003682DE9F041002B3D4D3E4F3E4EB8BFD9
:2063C0005B42A5FB0321890D07FB0137C7EB0717BF0096F81A3685FB0725FA170446C2EB6B
:2063E000A555002B57D101EB810101EB810105EB810109B2DFF8BC801320FFF7C1FF2F49D3
:2064000008FB057581FB0531ED17C5EBA11109B21B20FFF7B5FF2368254D002BB4BF532138
:206420004E212320FFF7ACFF636896F81A2683EAE376A6EBE376A5FB0631890D08FB0168E7
:20644000C8EB08184FEA880885FB08354FEAE873C3EBA5552ABB01EB810101EB810105EBF6
:20646000810109B21220FFF78BFF124B134903FB058581FB0531ED17C5EBA11109B21A20DF
:20648000FFF77EFF6368002BBDE8F041B4BF57214521222074E7C1EB011105EB810109B2E4
:2064A000A8E7C1EB011105EB810109B2DAE700BF6BCA5F6B806967FF98CF0020D34D62107B
:2064C0000B2814D810B401EB4103094C01EB83032344184490F8F436934205D0214400233B
:2064E00080F8F42681F8E8365DF8044B7047704798CF0020F0B5444C94F86D3B012B83B012
:2065000005464FD994F86E1B4048DFF810C194F86F7B4A1CA0FB026000F4FE7606EB900001
:206520001944121A5CF8216084F86E2B2FB1D4F8701B04F6743291420DD06EB9344A013388
:20654000A2FB031222F0010101EB52029B1A84F86D3B03B0F0BD2F4E94F8883B93B92E4B6B
:20656000019348F2A501123B15226F46A4F88C1B009384F88E2B29463846B04758B994F8E2
:206580006D3BDBE76F46384611F01CF829463846B0470028F3D094F8881B49B1384610F0D3
:2065A0008BFFECE71D4A52F82360002EC6D0D3E7009E1B4A964214D9013A013E41F2210531
:2065C00012F8013F81EA0321082311F4004F85EA41000ABF490081B289B2013BF5D1964259
:2065E000EED1384643F0BEFF0E49009D6D1A152DA8BF15252A4601F1180051F013FD94F8B9
:206600006D3B84F8B95B99E798CF0020CDCCCCCCABAAAAAAA92A010839DB0020448306087C
:2066200027DB002024DB002070B50C4E054606F6BE31D52244F032FC2C686C6006F6BC31C2
:20664000641A182CA8BF18242960224606F6D43051F0E8FC86F8EC4B70BD00BF98CF002097
:20666000F0B58BB004461F4B1F4A2049009302A81F4B45F007F926680025731C236035706E
:2066800023682922591C21601A702368EA22591C21601A702368C822591C216002A81A70EE
:2066A0004FF03CFA471C02A93A46206851F0BAFC236829461F440C2300E027687A1C013B8B
:2066C00022603970F9D12268511C2160137023680122991821601A7023689B1B33700BB0C1
:2066E000F0BD00BF8FDB00205CFE0608100007080800070870B505682C4E00236A1C0260EF
:206700002B7003682122591C01601A7096F88635DB0704461ED5B6F87C36590510D5244958
:20672000204643F0A1FE96F88635DB071DD523680022591C21601A7023685B1B2B7070BD0E
:206740001A0524D4D80524D4D90724D49A0724D51849E5E7D6F8443B6BB11749204643F04C
:2067600083FE96F88635DB07E1D423682A22591C21601A70DBE7114B1B681806CBD596F874
:20678000103603F00303032BC5D00D49C8E70D49C6E70D49C4E70D49C2E796F8002C0C49E0
:2067A0000C4B002A18BF1946BAE700BF98CF0020380007081C000708280007084C680020BE
:2067C0003000070840000708440007084C000708200007085400070838B50368394D591C98
:2067E000082201601A7003681E22591C01601A70B5F9DA36B3F5E16F044650DDA3F56163F0
:206800001BB2B3F5E16FF9DC07EE903A9FED2E7AF8EEE77A204667EE877AFDEEE77A17EE97
:20682000903A99B243F078FEB5F9D836B3F5E16F3CDDA3F561631BB2B3F5E16FF9DC07EEE2
:20684000903A9FED217AF8EEE77A204667EE877AFDEEE77A17EE903A99B243F05DFEB5F9A2
:20686000DC36B3F5E16F28DDA3F561631BB2B3F5E16FF9DC07EE903A9FED137AF8EEE77AF4
:20688000204667EE877AFDEEE77A17EE903A99B2BDE8384043F040BE03F561631BB213F5F7
:2068A000E16FF9DBB0E703F561631BB213F5E16FF9DBC4E703F561631BB213F5E16FF9DB08
:2068C000D8E700BF98CF002058A08B41026810B40421541C0460117002680B24511C0160E0
:2068E00014705DF8044BC82143F016BE38B50368224D591C0A2201601A7003680822591C23
:2069000001601A7095F81F3604466BB328F05AF81B490530A1FB0031C1F3CF01204643F055
:20692000FBFDD5F87036174AD91782FB0323C1EBA30189B2204643F0EFFD28F04FF8D5F8BC
:20694000785623682A0C591C21601A7023682A0A591C21601A7023685A1C22601D7023684E
:206960005A1C2260187038BDB5F83816044B0531A3FB0131C90843F0CFFDD2E798CF002042
:20698000CDCCCCCC6766666603681122591C70B501601A7003681D4D1D4E5A1C02600222CE
:2069A0001A700446296843F09FFD6968204643F09BFDE98901EBC10189003231A6FB0131C2
:2069C000C1F34F11204643F0A7FD298A01EB8101490089B2204643F09FFD0E4A0E4BD2F811
:2069E0003C1B9942A8BF194621EAE171A6FB0131490901F57A7189B2204643F08DFD236853
:206A00002A7D591C21601A7070BD00BFBC6800201F85EB5198CF002020A10700F8B50B4DEB
:206A20000B4F06462946D52244F038FA34687460A91E641A402CA8BF40243160224607F602
:206A4000044051F0EFFA87F8444CF8BD2E43002098CF002070B5104E104B0A46151D014645
:206A600096F8450C03F83F5C82B003F83D0C7B25C82003F83C0CA3F13B0403F8400C03F84B
:206A80003E5C68460193009443F000FD6846FFF7C5FF02B070BD00BF98CF00206C430020FA
:206AA000F0B5434C94F8483CD90785B0054637D594F8493C0F2B56D900210F463D4B94F822
:206AC000482C3D4843F8400CA3F1400640F6C82CC2F38202712003F8381CA6F804C0B11CEA
:206AE0000393B071373B02A8F271BA22029344F0D5F9029A731CD21A727012F0D1FE02A879
:206B0000FFF78CFF12F0CCFE94F8483CC4F84C5C23F0030343EA470384F8483C05B0F0BDC2
:206B20009A0728D5D4F84C0C2D1AB5F57A6FF5DB94F8493CD4F8500C0F2B97BF1F4A20494E
:206B400002EB8303D969036801911B69984701990620FDF7C3FE94F8483C6FF3410384F879
:206B6000483C05B0F0BD174B93F834301F1E18BF01273946A2E7144B1B685B05CED4114B5A
:206B800093F83430002BC9D00A4B0393C821A3F13F0202A803F8401C0292FFF797FE12F077
:206BA0007FFE02A8FFF73AFF12F07AFEB6E700BF98CF00206C430020C80032EC4483060898
:206BC000A0680600BC6000204C6800202DE9F843254E96F8544C804634BBD6F8B83C6BB310
:206BE00006F658474FF001090DE001352C44EFF31183502282F31288D6F8B82C944220DAA5
:206C0000DBB283F311883319601C93F8585C384429460022FCF742F80028E6D096F8443CAB
:206C2000D3B186F8549CE0E796F8443C33B901463A20FBF783FF044686F8540C2046BDE859
:206C4000F8830022DBB2C6F8B82C96F8544C83F311882046BDE8F88341463A20FBF76EFF65
:206C600086F8540CC1E700BF98CF0020044BD3F8343630EA030314BF01200020704700BF1A
:206C800098CF0020D54A38B50820002382F8AD31FFF7ECFF50B1D2F8A8314FF480640220F0
:206CA0004FF482611C8082F8AD0159804FF40020FFF7DCFF50B192F8AD31D2F8A8115C1C79
:206CC00040F2014082F8AD4121F81300C44991F85D36002B6ED191F85E36002B40F04581DC
:206CE0004FF40070FFF7C2FF50B192F8AD31D2F8A8015D1C4FF4046482F8AD5120F8134047
:206D0000D1F8E016880700F1E180490700F1BB80B44B1B681B066ED492F8AD3182F8AC31B3
:206D20004FF48030002382F8AD3182F8A531FFF79DFF38B1D2F8A03101204FF4047182F82C
:206D4000A50119804FF40040FFF790FF50B192F8A531D2F8A0115C1C4FF4007082F8A54185
:206D600021F813004FF40030FFF780FF50B192F8A531D2F8A0115C1C4FF4A06082F8A54108
:206D800021F813004FF48020FFF770FF50B192F8A531D2F8A0115C1C4FF4376082F8A541F1
:206DA00021F8130092F8A53182F8A431002382F8A53138BD0120FFF759FF00288BD04FF45B
:206DC0008030FFF753FF50B992F8AD31D2F8A8015D1C4FF4047482F8AD5120F8134092F836
:206DE000AD31D2F8A8015D1C4FF4116482F8AD5120F813406FE74FF40050FFF737FF50B118
:206E000092F8AD31D2F8A8115C1C4FF4036082F8AD4121F813004FF48050FFF727FF78B17D
:206E200092F8AD31D2F8A801591C1D46C9B24FF40064023320F8154082F8AD3120F811401A
:206E40004FF48040FFF712FF50B192F8AD31D2F8A8115C1C4FF4846082F8AD4121F8130009
:206E60004FF48060FFF702FF00283FF455AF92F8AD31D2F8A8115C1C4FF4026082F8AD4129
:206E800021F8130048E74FF48060FFF7EFFE50B192F8AD31D2F8A8115C1C4FF4807082F880
:206EA000AD4121F813004FF40060FFF7DFFE00283FF42EAF92F8AD31D2F8A8115C1C4FF464
:206EC000887082F8AD4121F8130021E78020FFF7CDFE50B192F8AD31D2F8A8015D1C45F231
:206EE000302482F8AD5120F813404FF48070FFF7BDFE50B192F8AD31D2F8A8015D1C45F2EB
:206F0000402482F8AD5120F813401020FFF7AEFE50B192F8AD31D2F8A8015D1C4FF4E0647C
:206F200082F8AD5120F813402020FFF79FFE50B192F8AD31D2F8A8015D1C4FF4E26482F843
:206F4000AD5120F813404020FFF790FE00283FF4DCAE92F8AD31D2F8A8015D1C4FF4E46420
:206F600082F8AD5120F81340CFE60220FFF77EFE00283FF4B5AE4FF40040FFF777FE50B930
:206F800092F8AD31D2F8A8015D1C4FF4007482F8AD5120F813400420FFF768FE50B192F8F8
:206FA000AD31D2F8A8015D1C4FF4C06482F8AD5120F813404FF48010FFF758FE00283FF443
:206FC0008FAE92F8AD31D2F8A8015D1C45F2502482F8AD5120F8134082E600BFF404002053
:206FE00098CF00204C68002003685A0607D513F4057F04D007298CBF00200120704703F4C6
:207000008253B3F5825F03BFC81FB0FA80F0400900207047F0B5BD4C94F8BC3C012B85B09C
:2070200000F04F8194F8C90CFCF766FB94F8CA3C834205461FD0002800F0D880D4F8643B6F
:20704000CBB194F8192693F90400002A18BF08224FF4964100230325CDE9015200911A46CF
:2070600008212AF0A6FCC4F8600B20B1FFF76AF9012384F8CA3C94F8CB3C012B00F0C38042
:20708000D4F8D46C3EB1A24B30465978FFF7ACFF002840F0F48094F8D90CFCF72DFB94F83C
:2070A000D83C8342054621D0002800F0F880EEB1337A002B00F01A81964A02EB8303DB6992
:2070C00094F8182696F904000093003A18BF012202210023CDE901121A4610212AF069FC6D
:2070E000C4F8300B10B1012384F8D83CD4F8DC6C3EB1874B30465978FFF776FF002840F045
:20710000AE8094F8E80CFCF7F7FA94F8E03C8342054622D0002800F0CB80F6B1337A002B51
:2071200000F0E7807B4A02EB8303DB6994F8182696F904000093003A18BF01220221002312
:20714000CDE901121A464FF400712AF032FCC4F8E40C10B1012384F8E03C94F8E90CFCF76D
:20716000CBFA94F8EA3C8342054632D098B36A4F41F2EC03D7F8B462E3584FF47A721A6196
:207180003EB34FF48052402130462AF09DFB0546F8B994F8183696F90400002B14BF0921CF
:2071A000082103224FF4E133CDE9012100932A462B464FF480512AF0FCFBC7F8B80240B14F
:2071C0000123C4F82C0B84F8045B87F8BC5284F8EA3C05B0F0BD504ED6F8B8022AF046FBAB
:2071E000C6F8B85284F8EA5C05B0F0BDD4F8600B2AF03CFB94F8CB3CC4F8605B012B84F869
:20720000CA5C7FF43DAF94F8CC0CFCF775FA0546002871D0D4F8543B002B7FF431AFD4F8CA
:20722000D02C002A3FF42CAF94F8195694F8181692F90400002D14BF08220022002908BF9A
:2072400042F0010203254FF46141CDE9015200911A4620212AF0ADFBC4F8540B10E794F851
:20726000E03C002B7FF479AFD4F8C43C002B3FF474AF0122C4F8E43C84F8E02C6DE794F878
:20728000D83C002B7FF432AFD4F8C43C002B3FF42DAF0122C4F8303B84F8D82C26E7D4F8B2
:2072A000300B2AF0E3FAC4F8305B84F8D85C1DE7D4F8E40C2AF0DAFAC4F8E45C84F8E05C43
:2072C0004BE7D4F8C05C124B28465978FFF78CFE20B3D4F80C36002B7FF4A4AED4F8C43CDB
:2072E000002B3FF49FAEC4F80C369BE64FF49643E6E64FF4614319E7D4F8540B00283FF40F
:20730000BFAE2AF0B3FAC4F8545BB9E698CF0020986000204483060890E0002094F8C80CCB
:20732000FCF7EAF90646D8B1D4F80C36002B7FF479AE002D3FF476AE94F8182695F90400EF
:20734000B2FA82F252094FF416510225CDE9015200911A4604212AF02CFBC4F80C0661E66C
:20736000D4F80C0600283FF45DAE2AF07FFAC4F80C6657E6F8B5CC4C94F8BC3C002B00F067
:20738000C18108202AF0B4FAC84DC4F8640B002840D008212AF0A2FA00270346C44984F86B
:2073A000C93C05F530700522C5F8C47236F024FC41F20853012205F53070A5F8C83285F86F
:2073C000CC220DF0D7FE39462B2205F5357050F08AFE48F67C627D26E0233946A5F8D422E6
:2073E00005F540702B2285F8D73285F8FF6250F07AFE48F67C21A0224EF27B0385F82B6314
:2074000085F82E7385F8D763A5F8001385F80323A5F82C3394F8CB3C002B00F05D8110208C
:207420002AF066FA1021C4F8D40C2AF057FAA14B84F8D90C40F23B113A20198094F85D26CD
:2074400018719F214AF21E409971002198601973002A40F00E8194F85E36002B72D1D4F857
:20746000E036580700F1FE80990700F1F2801A0700F1E880904E3068C0F3C010FEF71EFFA0
:207480000020FEF701FF03464FF4007084F85C3B2AF02EFA4FF40071C4F8DC0C2AF01EFAFC
:2074A000D5F8D83384F8E80C002B14BF0123002385F8DC3340F09280D4F8503C002B14BF1B
:2074C0000123002385F8E53343D1D5F828250023C4F8B83C002A00F0DC80012284F8883BF7
:2074E00085F82C25002375487549C4F8783B062236F082FB40F609437048A4F87C3B0DF05C
:2075000039FE4FF480502AF0F3F94FF48051C5F8B4022AF0E3F9D5F834356A4A6A4E84F880
:20752000E90CC4F86C2702F5A070591C0022C4F87007C6F81031C5F8341584F8EA2CBDE8FA
:20754000F84067E5D4F8583B43F00403C4F8583B85E7D4F8E006002310F0020085F8E633E6
:2075600085F8E73340F0E780024694F85D362BB10120FFF77BFB002840F0EF8094F85E3626
:20758000002B40F0E4800820FFF770FB20B1AB18042183F8E813013233681B0600F1FE8016
:2075A0004A4B10219818053300F8011B8342FBD105220921202042F2090385F8ED2385F89D
:2075C000111585F8120542494248A5F81C35042236F012FB3F480DF0CDFD76E794F85D36CB
:2075E0002BB10120FFF742FB002840F0BC8094F85E26002A40F0DF8033681B0600F1B7801A
:20760000D4F8E0164F070CD54FF48060FFF72EFB38B1AB18082183F8E013013285F8E42335
:207620004AE7080705D54FF40070FFF71FFB0028EFD10905F2D54FF40060FFF717FB0028DD
:20764000ECD0E6E7D4F8583B43F48073C4F8583B10E7D4F8582B42F4601242F0C002C4F82B
:20766000582B04E7D4F8582B42F40272C4F8582BFAE6D4F8583B94F85E2643F00201C4F823
:20768000581B002A3FF4EBAE43F03603C4F8583BE5E6D5F83035002B48D0012385F82C3584
:2076A00084F8883B1EE700BF98CF002090E00020A0830608D46800204C6800200CDB002048
:2076C0004884060814D70020F404002078E40020F4830608A4E5002020202AF009F9C4F8EB
:2076E000D00C00283FF49BAE20212AF0F7F8354BC4F87C3584F8CC0CFFF7C4FA012384F82B
:20770000CB3C8CE604202AF0F3F8C4F8C00C00283FF437AE04212AF0E1F82B4A84F8C80C22
:207720000123C4F8802584F8BC3C2AE685F82C3584F8883BE5E64FF46070FFF797FA002896
:207740003FF412AF012085F8E80302460DE70620FFF78CFA00283FF416AFAB18022183F84D
:20776000E81301320FE7012285F8E02344E74FF4A050FFF77BFA20B1AB18022183F8E01354
:2077800001324FF40850FFF771FA00283FF438AFAB18042183F8E013013231E74FF45850EC
:2077A000FFF764FA00283FF4FBAEAB18082183F8E8130132F4E60620FFF758FA0028D2D1C9
:2077C000024619E72D620108112701082DE9F04FBC4C89B005460F46164694F8389530F07D
:2077E00005F88246002028703070D4F84885387018F0010F4AD012F011FF002843D0B24BAF
:20780000D3F8442B002A3ED0970104D5B2F1007F18BF02F17E42D4F8A8159FEDAC7AAAEB09
:20782000010307EE903AF8EE677AF4EEC77AF1EE10FA05DCD4F8AC0501238340134212D135
:2078400011B91923C4F8AC35D4F8AC35C4F8A8A5012001331A2B28BF002300FA03F11142EA
:20786000F7D0C4F8AC35D4F8AC25994B994903EB82032846D3F8582144F004F80223337024
:2078800009B0BDE8F08F0023C4F8A835D4F8B03593B38D4B93F88635D8072DD4D4F8B435A5
:2078A0009FED8D7A03F5921303F57863A3EB0A0307EE903AF8EE677A67EE877AFDEEE77A02
:2078C000B8EEE77A17EE903AF1EE0C7AB4EEE77AF1EE10FA06DB8149284643F0D3FF01233F
:2078E0003370CDE70A212846B3FBF1F201FB12337B4943F0C7FFF2E718F4007F0CD0724B0C
:2079000093F88B3543B17749284643F0BBFF0323337001233B70B3E718F0200F17D01B2082
:2079200012F07CFE98B194F8B83523B16E49284643F0A8FFD3E7644B93F88635D90706D4CD
:207940006A49284643F09EFF0123337098E718F4806F36D094F8B935012B32D15A4BD3F8D6
:20796000E02612F0020F984626D0B3F9DA26B4F9C835D21A6FF463739A4218DB40F28D33DE
:207980009A4217DC0A2392FBF3F25949284643F079FF1EF051FAD8F84C3B93F863300A3BAB
:2079A00023EAE37398429ADB01233B7097E76FF05902EAE75A22E8E74E49284643F062FF59
:2079C000E7E718F4005F0ED012F026F894F84035834208D94849284643F054FF022333707C
:2079E00001233B704CE718F4004F08D0434BB4F99425B3F9B0319A4201DD4149EBE718F4AF
:207A0000804F07D011F0F0FFB4F89235834201D93C49E0E718F0080F04D0B9F1020F01D1F2
:207A2000394971E718F4006FDFF89CA00FD09AF88635DA070BD51BF09DFE40B19AF8103682
:207A4000DB0704D594F805360BB93049C3E718F4805F14D09AF88635D80710D51BF08AFE4A
:207A600068B19AF81036D90709D4D4F80836A3F53713A3F5D863002B01DA2549ABE7BAF8E1
:207A80007C365A0601D52349A5E718F0800F45D0BAF97C0A94F85A3598423FDB03F04CFDD6
:207AA00094F841251C49002A0CBF0D220E220346009228467A2243F0E5FE02233370012334
:207AC0003B70DDE690E0002098CF00200024F4484483060861440708ACC527373EFF06081E
:207AE00049FF060856FF06085800070860FF060872FF06087CFF060883FF0608F404002049
:207B0000150407088CFF060899FF0608A3FF0608AEFF0608B9FF0608C2FF06086C4B1B68C4
:207B20001B017CD518F0400F79D06A4B93F8008004AAC8F109084FEA5808002310462021AD
:207B4000984521D1644940444FF0000B50F0EFFA08F1030859465F4B1B788B4202D9B8F181
:207B60000B0F15D908AB9844002308F8103CBBF1000F54D0594904AA284643F083FE022389
:207B8000337001233B707BE602F8011B0133D7E7CBB2184603910293FDF770FC029B03996D
:207BA00003F1310C9AF8863513F001035FFA8CFC029332D0B4F956E5BEF1FF3F2DD08289EB
:207BC000642312FB03F2464B93F822305B0892FBF3F39E45B4BF6346522394F9542512F15B
:207BE000800F04D090F901E09645A8BF5423029A42B1B4F95825B2F1FF3F03D04068904218
:207C0000A8BF432304AA9C4508F8023018BF0BF1010B013108F101089DE76346DDE7D4F806
:207C2000488518F0040F0BD0B9F1010F08D12D49284643F027FE0223337087F800901FE6D6
:207C400018F4807F08D09AF88635DA0704D5264B1B780BB92549BEE618F4803F0CD09AF827
:207C60008635DB0708D5B4F83C352BB1DAF87826934201DC1E49AEE618F0020F14D09AF8E5
:207C8000863594F8382503F0030313430CD126F099FEBAF86636834206D91649284643F075
:207CA000F1FD01233370EBE518F0100F3FF4E8AD94F83036002B3FF4E3AD0F49284643F077
:207CC000E1FD01233370002384F83036D8E500BF4C68002038490020AF0207086144070895
:207CE000082F0020D1FF06084C690020DDFF0608E9FF0608F2FF0608FEFF060807B50023B1
:207D000000F10D020DF1070140688DF80730FFF75DFD9DF80730084A43B1D2F8343643F42C
:207D20000013C2F8343603B05DF804FBD2F8343623F40013F5E700BF90E00020094BB3F87D
:207D40005626B3F85436801A9B1AC00090FBF3F00628A8BF062020EAE070C0F19600C0B227
:207D6000704700BF98CF002010B5094B0022D3F83C1603F5C863914201D1002010BD13F8EE
:207D8000014B844201D00132F5E70120F6E700BF90E000201D4B2DE9F04303EB81038FB042
:207DA000D3F8C08106460D46B8F1000F2BD0184B03EB41031C22B3F87E460023194604F0AD
:207DC0001F07C4F344190DEB0200A413069350F08AF901228DF80B4006AC8DF81420CDE948
:207DE00003468DF808508DF809708DF80A9002A8C0479DF8142000232AB100944A46394625
:207E000002A803F0FFFE0FB0BDE8F0834483060890E000200A4B03EB4002B2F87E16094A76
:207E200092F8B22102EAD122520707D0D3F83C26511CC3F83C16134483F84006704700BFA1
:207E400090E00020F404002010B5164B42681B7803F00303032B21D1134B1B88DBB1134B13
:207E60001349B3F90030B1F904100A2491FBF4F15B1A1B0103F5B95314334FF4B471B3FB7B
:207E8000F1F3C3F1080303F00F0360331370436800225A7010BD05231370F8E72D23137063
:207EA000F5E700BFA8D50020AAD500202CE9002070D60020436872221A70436873225A707D
:207EC000436874229A7043680022DA7070470F4B4268B3F904300A2193FBF1F31B0110B527
:207EE00003F5B9530A4C4FF4B4711433B3FBF1F303F00F031919E35813604B6853600B7A17
:207F00001372436800225A7210BD00BF70D60020E0070708034B5B7913F0FD0F14BF9E2099
:207F20009D207047CCE50020094B5B7913F0FD0F06D142F210735843064B90FBF3F0704726
:207F4000242358434FF47A7390FBF3F0704700BFCCE5002040D20600054B07EE900A5B798F
:207F6000B8EEE70A1BB9DFED037A20EE270A7047CCE5002048F9514010B50D4B9A78012A5A
:207F80000ED15A68811A00290ADD022199700949B1F866400849B1FBF4F132B10A445A60FB
:207FA0009878013818BF012010BD08445860F7E72CE90020CCE5002040420F00831E00F1A8
:207FC0007A02EA2123F8021F9342FBD14E2243F64913C280CE2243850281CD232322838083
:207FE000A0F87220A0F87830704700BFF8B91D48038903F0010353BB30B4047BACB11A4AD6
:020000040801F1
:2080000002F1F00502E00133A3420ED052F8041B4904F8D590F8F81000EB8101D1F89010B6
:2080200045F823100133A342F0D130BC70470D480289032A4FEA52030AD90A68038102F5E8
:20804000C332A03203F001030A60002BD4D070470B6803F5C333A03348F205020B6002810F
:20806000704700BF2CE900203CE900202DE9F041002839D12C4A107B80B32C4A2C4B92F8EC
:2080800000E092F901C092F90280CEF1FF07AEF17F06FFB2F6B203EB800003F1F0020024ED
:2080A00003E0834202F1040218D053F8041B8904F7D5E1B2A1EB0C0181EAE175A5EBE175A1
:2080C000012D0DDC71B1414514BF394631468342D17004F1010402F10402E6D1BDE8F08152
:2080E0000821F4E77146F2E7104B1A78F02A09D802F10F000C4A18700B6803F582431A33A7
:208100000B60B8E7084A93F90140907B7F2584421D70987805DB4042C0B29870204458701C
:20812000EAE7002CFADAF6E72CE90020A80600203CE90020F0B5374E78B196F88031002B8C
:2081400045D0354A013BDBB286F880311378DC073FD4324B0A681A440A60347B4CB3304B32
:208160002D4F03EB840403F1F001002503E09C4201F104011DD053F8042BC2F303200628DE
:20818000F5D13878C00715D596F8800196F80FE000EB050CBCFBFEF00EFB10C00128CCBFFE
:2081A0000020012058B99C4205F1010501F10401E1D1F0BDE84300F001000028F3D0C2F381
:2081C000834206EB8202D2F890200A60EBE7F37BB7E7D6ED647A134B134CFDEEE77A642075
:2081E00017EE902AA2F57A7200FB02F283FB0230D317C3EBA01303EB4303C3EB031384FBDC
:208200000302DB17C3EB62130533084A92FBF3F3A0E700BF2CE900201ED50020400D030069
:208220003CE90020D34D62101F85EB5140420F00F0B4524C002867D194F8CC01002855D0AE
:208240004F4BD3ED007AB3EE097AF4EEC77AF1EE10FA4DDCBBEE097AF4EEC77AF1EE10FAB9
:208260004CBF08270027D3ED017AB3EE097AF4EEC77AF1EE10FA3DDD47F00107257BADB3D9
:20828000404ADFF80CC102EB850502F1F00014E094F9CF61B142ACBF0221002194F9D06145
:2082A000B3421CDB41F004010F421CBFDCF80C300360954200F1040018D052F8043BD903E4
:2082C000F7D594F9CE6103F00F01B142C3F30313DEDC94F9D061B3424FF00101E2DA94F95D
:2082E000D161B342D8BF41F00801DDE7F0BC70470427B8E7BBEE097AF4EEC77AF1EE10FA5D
:2083000048BF47F00207B9E794F8CD3163B31C4B1D4DD3ED007A93ED017A0A6894F8CC0105
:20832000F0EEE77AB0EEC77AF4EEC77AF1EE10FAB8BFF0EE477AFDEEE77A80F0010017EE3B
:20834000903A193B03EB4303C3EB031385FB0365DB17C3EBE51305330C4DB5FBF3F31A4402
:208360000A6084F8CC0169E70B6894F8CC0103F5433303F5A0730B6060E700BF2CE900200F
:20838000DCD500203CE90020353AFC4440420F0030860608F0B40B4F3E7B86B107F11002CB
:2083A000054607F58077002352F8044B35EA040004BF086847F823000133B342F4D1F0BC71
:2083C000704700BF2CE9002030B42A4B60B92A48027DCAB993F8F9302849203301EB830124
:2083E00030BC4FF4A060D5E793F8D221F2B1013A214883F8D2210A6802F5C32202F5207288
:208400000A60027D002AE5D01D4A12689106E1D51C4A93F8D211127892071AD511BB93F829
:20842000FB301649203301EB8301D9E7124893F8D341057DA54205D8042483F8D32183F8DE
:20844000D241D8E70134012283F8D34183F8D221D1E70029BED193F8FA300849203301EB40
:208460008301BDE793F8F7300449203301EB8301B6E700BF2CE90020BC6800203CE90020F8
:2084800078D60020A8D5002010B450B91E481F4C90F8D4210B6823440B60A2B15DF8044B7A
:2084A00070471B4B1B7813B3012B17D016480B6890F8D421174C82F00102234480F8D42139
:2084C0000B60002AEAD190F8F73013495DF8044B203301EB83014FF440705BE70A480F4CF8
:2084E00090F8D42182F0010280F8D421D2E70B68054A5DF8044B03F5742303F510730120D3
:208500000B6082F8D40170472CE9002040420F00C8E5002048E801003CE9002020A1070019
:208520003C4AA0B992F8D5316BB192F8D6118A081341DB070AD501F00101032A06D8DFE8D3
:2085400002F05048403892F8D73153BB704792F8D631013303F00F0382F8D6313BB192F801
:20856000D531086800F5C330A0300860DCE72A4882F8D531437A002B44D12848C07818B142
:2085800043F0040382F8D53125480078C00730D5244800780028E4D043F0080382F8D531F2
:2085A000DFE792F8E231204901EB83014FF40030F0E61D4B03F13002002914BF19461146F6
:2085C000F4E71A4B03F1180200290CBF19461146ECE7154B03F10802002914BF19461146C0
:2085E000E4E7114B03F11802002914BF19461146DCE70F4800680028CAD043F0010382F89F
:20860000D531C5E70B4B1B78002BB6D0022382F8D531B2E72CE90020ECD5002020D50020A5
:208620001ED5002048E600203086060840860608DCDA0020C8E5002030B4022340F203154B
:208640004FF4FA74322146F20142C37000238580C480018130BC42810380704770B40B4C16
:208660000B490C4B22680E680D6883F8FC01002122F0200283F80012C3F8EC61C3F8F85174
:208680002260C3F8F41170BC704700BF78D600202C2E00202CE9002090F8603043B942691A
:2086A0000121072082F84430A2F8460082F84810704700BF034A0123E021C3735170184694
:2086C000704700BFBCE300204FF0FF30704700BF4FF0FF30704700BF704700BF0020704750
:2086E0000020704770B4067AAEB1427A0B4800212025002352B1142B05DC072903DCC45CB6
:20870000202C18BFC55401339342F4D101318E4200F11500EDD1002070BC7047BFE30020C4
:2087200010B50024C4730121FFF7DCFF024B01225A70204610BD00BFBCE3002070B403987C
:208740000378ABB10C4C02EB4205C5EBC5052544142901F1010406D8072A294403D8CE7802
